:20000000004B00204D420100FDC90110FDC90110FDC90110FDC90110FDC90110FDC90110DB
:1C002000FDC90110FDC90110FDC90110FDC90110FDC90110FDC901103BCA0110A4
:20003C00AD040021490400217D04002181040021110500219105002141060021F8B51047C2
:20005C00F8B50E4600210125AD0430470A48037800F00FF89B070BD0124C2078FF2807D0DF
:20007C00FF2121700E490F24240220436031C882F8BDF8B5014800476B020021E54C000014
:20009C00094801E00848000C064C05492278FF2A01D1CA7A22706031C8827046801C004737
:2000BC0000620840A4060021070F0808F0B4084770B503461546012906D0002906D0114A73
:2000DC002846FFF7BBFF70BD0F4800E00F480524834203D84008641E002CF9DCE340012053
:2000FC0040031818820B012907D00649002380312846FFF7A5FFE0B270BD0249044B6C31C2
:20011C00F6E70000835C0000A0BC862300830D2374060021F8B51A4E0546716B1948CC0942
:20013C00E401002D11D01849097802290FD0007B044372B60120154F4002B8471148203863
:20015C000088C109C90704D016E0C07AF0E7407BEEE70F497463CC61400AC0070CD001208C
:20017C008003316B002D01D0014300E08143084631630749403948630020B84762B6F8BD1C
:20019C0080020021880000219B0200217B3F00004040044010B5224A00215161214989685C
:2001BC00C90009D42149204BCA0598424B6B01D8134300E093434B631D49FFF777FF10BD17
:2001DC0038B51A4D287F002827D11A480088C009C00722D1124C606900281ED1684600F09F
:2001FC0045F868460078012817D168464078102813D208206061686A4009400120600E4ACF
:20021C000021D1620D4A02211160012108432060032108436862206038BD0948804738BDDB
:20023C0000400440180000210000930880020021CF680000680000210011044080E200E050
:20025C00C33B00000749002800D00420064A72B60978C90701D0105800E0802062B640B28C
:20027C00704700006B0200215860044003B40148019001BDA56F00000000000001000300BA
:20029C000A001F005900EB003902EA04F9099712EB1FA132784A0A66FA828C9E63B617C953
:2002BC0064D6EDDEC1E3E0E5FF000000A36100007F1407134D00F1242E1F133FB00A3F000A
:2002DC0007FF0000304000400140034007400F404F40CF40CF41CF43CF47CF4FCF3FCF2F32
:2002FC00CF1FCF0F000000000F00080000003F00000040003F000000040068000E00DC00EB
:20031C00060043001A00050000000000020000003F00000000000400C00000000400C00090
:20033C000000070050C00091007070C00091007082312100319110B10070018101B100A1BC
:20035C008231329110B101911110418141224F40F106007051C0019130181039833108D0BC
:20037C001831416F3100319110B1831414165B680070251050C00091F4C3C0C02014036F0D
:20039C003110410422C082312100319110B163393110410482C082312100319110B163392B
:2003BC003110A2C082312100319110B1501015310514059200703F6452C0311031066131A2
:2003DC00C102426412C13110213971065131E102426400708A65996588C02082503980391F
:2003FC00001E9F4041C001301814181A89C0308260398039001EA94041C001301914191A6E
:20041C003C64369110B1349110B154B0007154A064B0F0800022AF404012B09032B05382CB
:20043C005339533985643F6411C122C1426470C1C26811C1C2C0426470C1C76850C000914B
:20045C00277298921516141642105310F0C12182313131398139313151B070B272652772E4
:20047C00999270B262107310F0C331822131213981391B107265E2C08231608280318039AF
:20049C00020061B00071329110B151A061B0277230C2F36800008012B09032B0007050C01C
:2004BC0000912772999262107310F0C3318221312139813951B070B27E652772989270B21F
:2004DC0042105310F0C1218231313139813931311A107E6551A061B02772B0C018693F64D3
:2004FC0001C122C1426401C1C2C04264151A3C64359110B153828564C012B09032B0007033
:20051C003F6472C281C0426422C111C1426402C011C1426462C031C3426462C311C1426413
:20053C0002C311C14264538253398564E2C347641122404142C281C8426452C211C1426495
:20055C0072C2E1CE426402C281C8426402C201C84264B0C0546900703F6442C201C842645D
:20057C0052C211C0426472C2E1C0426402C001C1426462C001C3426422C101C1426462C333
:20059C0001C1426402C301C1426453828564007061B000711214231C7A4D339110B10070D9
:2005BC00329110B17269007061B000711318321C8649329110B10070339110B17E690070B6
:2005DC00C2C047641510C2C01216476441311514C0C0803105145410A07804040070E6C0D9
:2005FC00863101CC161467106182F0C3010417140070067305720B720E7250B00071818025
:20061C0060B050A092804122C3458080F1C11004301601110114016CD661D761D861D961BF
:20063C00DA61DB61DC61DE61E061E261E461366339639180F2C0210421318280422A1214DF
:20065C00321601112114016CEE610B62F4613963EE610B62F4613963E661E661E661E6610C
:20067C00E661E6619464E661F964E6612A65E6615665E6614667E6611012B0900E720673C6
:20069C00057210123090A761F0CF3C67D4C103C0C0C354644078509150781092607820925B
:2006BC007078309280784092907860923078909110824039F0060110103110140092426735
:2006DC00E661BCA0E2A054A0F08050221546408000222B470D6240A02D828D318D39108240
:2006FC00F1C0100409101A824A391A041082803910040E10AB10BC10C21063642972E0CFDC
:20071C003C6713B003B0C86653B050B054B064B013B0A5661082E0223846AE660071418035
:20073C0001222B47F08010224B46F022184764B03122384263B0CE661082E0223846706654
:20075C00386264B06F818F318F3DD0DFFF923C670071418001222B4764B0F080502265420C
:20077C0063B01182C1226046CE6605671182D122524670665262618172818131813D8231EE
:20079C00823DC0EFF19202933C670B62B081C091D381978290A2D3187F4EF30B1316E31CA8
:2007BC00A44AC391E3813B149062BA1C8B46231E8B4AE31C8B4E90B207228B4290A21B1A02
:2007DC009662E31CA44AC391E3813B18AB1CA04E9B1CA24ABC1CA442B2101082D0229D42D2
:2007FC00F0801022A4466364A566A462AB1094629B10946200703082F1C0100463B00071BC
:20081C00A86ABC10E0B00070B281C291D281018212185181121841828131813D121CBF4AF2
:20083C00E2B032B0B0DFF2923C67F1C72114C34E12C86291729131B0E1B0007008C006C034
:20085C0000C86091709100700182B081C091D0811018518110180614E18042828231823D29
:20087C00201CE44AE2B02122E84632B00510A0DFF5923C672122E842E2A032B03182413951
:20089C00F0C00104011EF642181610C01030081C04476010103C0610F1C76114FA4E16C85E
:2008BC00669171818131813D161C014B769131B006C008C0007061818131813D4082803992
:2008DC000118F11C174B0114B080C0221747BCB033B090EFF1920F933C67007003A063B033
:2008FC0064B0EFB056650071408000222B4764B02A65EFA00071408000222B4764B003B0EB
:20091C003862018262818231823D80EFF19202933C6703A05665E661A2806364E66150B04A
:20093C000071E661E092D08200223D47C0B20070A080F022594330B002C1623101C0A080B2
:20095C00001E5243F0225343A0F56031603953632010101A136F236E11161216546B0070C0
:20097C00B1C700000000000061A500000000000000000000C5950000557601005D1A01003F
:20099C00A97001005169010035690100ED1901000000000000000000511601009131010095
:2009BC00E9450100D1CF00000F7201000E3FA73FAB0C18B82BBC0BDA50E5900AD338D8583A
:2009DC0009CD2CD24008CB24CE3207C920CB2A06C71CC92405C618C82004C518441803C466
:2009FC0014C61C024210C51801C310C416004100C312F6C008C0040093300100ED5C010060
:200A1C00D9C300003D7601001F770100090D0100155D01008D76010099760100937601002B
:150A3C00000000005B770100000000009D090100C80900000F4B
:200A580000FF694501003C0A00005F7C0900001400704C00B0A30800000FF815B1A0B0D28C
:200A780001B14901B700000300FA9803B325057F380000900D0020B421FD83015019AD0056
:200A9800008002AF0304401F01B35801B482B201BC03037005F70810B82084AEB8614E906A
:200AB80055B8D20701FA21FF030F008000230798FFE008003FA7781500BF20930300800575
:200AD800BB7004DE04788001886A03F5F401FF10580000FC0400C4FB2264BDE907180000A4
:200AF80038FF403A00A384060020FF40007F6440400003FF0507B12305330583FF05480A46
:200B18000306B87A02FF009F84020044C703FF0401026384100043FF02B00483880300A3A8
:200B3800FF88FB008460F13588FF601A418C60238202AF00DF7D43C47063C4B0FFC0000024
:200B5800C46FFA03332034730085E63F01856DFF0100393201005377FC024F09E9BF8104FD
:200B7800ED0E01006174F4237000304723BF45ADD000001BB98A2DDF0A7017FFE14F714F00
:200B9800AF121851E1521752B70F0FFFE304D3FFEFD401FF08020020656B0100DBAD6F41F4
:200BB800CF085955413F604087A24AC7AA00B8FFEF2A76F33776FF4301AD077CB0C40DFFBB
:200BD800E0818AF3C5FD0D8AA04000011B00007DC800B002002A00028BB0F7180C0EFFE064
:200BF80026000202DF0000440D0E8CE01200F5028C10E0017002000C00AD030170952B0420
:200C18007122FFE4FEBE7CBF3784840100059540013D5A5E3F34C816002000316639D90421
:200C3800FFE50DF0202898B307C2F1019531693F03FFEF020D200580650E0030FE6F3F31DA
:200C5800FFE1C5A7FFE3FBD571709600E0190020F80175027D017D0608808007F400300842
:200C7800FF2230001E5000A0007F40018002F004E09AF012307F0F117C7D255018A2E00074
:200C98003101BF01115C01B00031A00F260741000D7F13826F1D29F40B300031FC00340474
:200CB80017F00031550C00341400341C003424003403A9FCFFE7B631BDC2FFE802F1FFE1B1
:200CD800A9541CF000315C00346400346CCA00347400347C0034FFEF129C01630020003187
:200CF80093F193A98F26923F14EF91660100C9C1FF0014B2FFE2CCC590CCA1E81ACA33B826
:200D1800C90600F3FFEF0CF00034FFEB1D1E98D070FFEF01052000712E7000316854067058
:200D3800003170003478003480003455880034900034980034A0003495A80034B00034B8E4
:200D5800003476B27F0049903A0F054132DA70FFF0007D000000E61A0020D8003059DC00F3
:200D78007000F1004B00700500927F20010100005C2C0174000044FFF000F30100000700DC
:200D9800B954190020EC01A80252E01A0133340100052000313C0034FFF0009D0000016CEA
:200DB800DC02007200C048EF1800200300C4B958011F0005700100FFF000FD0000046017C7
:200DD8000020241947002001010000310029A80170000031FFF0007B0100000F00F418000B
:200DF80020016100FFF000003D2001004574010049750100003D00000060170020FFF000D0
:200E18000200000039170000000F08000000FFF00001000000FFF00001000004FFF000017D
:200E3800000004FFF0000000580A000008020020690D000044010020910D00000001002081
:200E5800B20D0000A4010020D10D000078010020EE0D0000C80100200C0E0000E40100207C
:200E7800180E0000E81A0020200E000000020020280E0000EC0100202F0E0000F001002031
:080E9800360E0000F8010020F5
:201000003C000000000000000000000034100000000000000000000001000000000000004F
:1C10200000000000000000000000000001000000000000000800000000000000AB
:20103C003400000000000000000000006810000000000000000000000100000000000000E7
:14105C00010000000000000000000000080000000000000077
:2010700030000000000000000000000098100000040000000000000001000000FFFFFFFF87
:10109000FF00000001000000080000000000000048
:2010A0002C0000000000000000000000C4100000040000000000000001000000FFFFFFFF2F
:0C10C000FFFFFFFF080000000000000020
:2010CC0038140000E410000095A1011091A70110A1C2011009B2011041B8011000000000EA
:0810EC00000000002D000000CF
:2010F400280000000000000000000000141100000000000000000000FFFFFFFF0000000093
:081114000800000000000000CB
:20111C00341400003011000065C2011069C101101BC2011091BA011000000000000000006D
:04113C002F00000080
:20114000341400005411000071C20110A5B6011099BF011045B601100000000000000000BD
:04116000300000005B
:201164002400000000000000000000008011000000000000000000000000000008000000AE
:041184000000000067
:20118800240000000000000000000000A41100000000000000000000000000000800000066
:0411A8000000000043
:2011AC00240000000000000000000000C8110000000000000100000000000000080000001D
:0411CC00000000001F
:2011D00000000000681A002004000000000000000000000020000000701000003000000089
:2011F0001C110000701A00200400000000000000000000000C00000030130000180000009D
:2012100040110000781A002004000000000000000000000024000000481300001800000020
:2012300000000000801A002004000000000000000000000010000000A01000002C000000F4
:20125000CC100000881A002004000000000000000000000020000000641100002400000023
:20127000FFFFFFFF901A0020040000000000000000000000280000008811000024000000AF
:20129000FFFFFFFF981A0020040000000000000000000000580000003C1000003400000094
:2012B000FFFFFFFFA01A0020040000000000000000000000100000006013000018000000A9
:2012D000FFFFFFFFA81A00200400000000000000000000001C000000AC110000240000001F
:2012F000FFFFFFFFB01A002004000000000000000000000038000000F41000002800000090
:20131000FFFFFFFFB81A002004000000000000000000000054000000001000003C0000002B
:1813300018000000000000000000000040130000080000000000000032
:1813480018000000000000000000000058130000080000000000000002
:18136000180000000000000000000000701300000800000000000000D2
:0813780002000000F08A0100F0
:041384000100000064
:0413880000000E0053
:04138C0000000F004E
:041390003200000027
:041394000100000054
:04139800E019002038
:04139C00000200004B
:0413A000BD76010015
:0413A400FDC901106E
:0413A8000000000041
:0413AC00000000003D
:0413B0000800000031
:0413B4000000220013
:0413B8002C180020CD
:0413BC00010000002C
:0413C000F8190020F8
:0413C400080000001D
:0413C8000000000021
:0413CC00000000001D
:0413D0000000000019
:0413D400080000000D
:0413D8000000000011
:0413DC00000000000D
:0413E0000100000008
:0413E40024190020A8
:0413E80006000000FB
:0413EC0001000000FC
:0413F000C8160020FB
:0413F40000000000F5
:0413F80000000000F1
:0413FC0000020000EB
:0414000000000000E8
:021406002900BB
:021408000100E1
:02140A002500BB
:02140C002F00AF
:02140E003000AC
:021410002D00AD
:021412000100D7
:0114140001D6
:0814180003000000AC8A010092
:081420000000000000000000C4
:0414280000000100BF
:04142C0000000300B9
:0414300083C4011060
:041434003C14000064
:041438003C14000060
:04143C0000000000AC
:041440008000000028
:041444008000000024
:0414480000000000A0
:04144C00F81900206B
:0414500057720100CE
:041454002000000074
:041458005C8A0100A9
:04145C00A88901005A
:0414600009C30110AB
:04146400E73001006C
:041468002735010023
:04146C0095C801100E
:0414700097C8011008
:041474000000000074
:041478005B8A01008A
:04147C00788801006B
:04148000908801004F
:04148400608801007B
:0214880008005A
:02148A00090057
:02148C0001005D
:02148E0000005C
:01149000015A
:041494000000000054
:041498000000000050
:04149C00000000004C
:0414A0000000000048
:0414A4005F7701006D
:0414A800E54F01000B
:0414AC0005630100D3
:0414B000995301004B
:0414B4009754010048
:0414B800E9580100EE
:0414BC00951801007E
:0414C0006F74010044
:0414C4006D2C01008A
:0414C8000DC801103A
:0414CC001DC8011026
:0414D0000800000010
:0414D40024000000F0
:0414D80018000000F8
:0414DC0028000000E4
:0414E00020000000E8
:0414E4003C000000C8
:0414E8000C000000F4
:0414EC0034000000C8
:2014F000C7482DE9F04F0C4620274FF0000C01211F40ADF14C0D6546DFF81893DFF818837D
:20151000DFF818A3DFF818B30170002F0F93C0490E9205EA020081F800C008BF00287CD136
:201530000E984FF0E047194662460F401040002F08BF002845D10F9E0E9B4FF48601B9F8E4
:20155000B200DFF800C3CDF8289002EA0607002F01EA030108BF00291AD1B94902EA0607C5
:20157000002F01EA030108BF002970D0374643460E9EDC8003F128011881002F81E8C000F1
:2015900004BF311CB1F1806F61D102285FD111E0374643460E9EDC8003F128011881002F2A
:2015B00081E8C00004BF311CB1F5803F4FD1B0F5505F4CD1186A674643693868214698472B
:2015D00043E04646C249B6F9067091F90000BC42A0F10100087017D1328906F1280003C8FD
:2015F000002904BFB0F5803FB2F5505F08D0002904BFB0F1806F022A02D010F079FF03E088
:2016100012F076FA15F022FC524692F90000401E10706FF00101F18015E0B64E3778434621
:201630006FF00100991D08806FB1B3480078832802D08120594608704646316919B160469E
:2016500088472146E7E7CDF82890B9F8B2000F9E0E9A2F46022137401140002F08BF0029C2
:2016700000F07A83A5490B91A64A119243F20141814200F04B83C91C814200F04783944919
:201690000A4691F900104746491E1170B7F906108C4205D043F60401814240F0468342E353
:2016B0004046283090E800032F464FF4820607EA090706EA0800002F08BF002811D15648EA
:2016D000283003C82F464FF400320F400240002F08BF002A02D110F00BFF26E312F008FA52
:2016F00023E328460B9F109097F8380081245D4618B92F780FB115F0D7FD2C70804C002074
:2017100067786081119EE770054635702069DFF8F891017A457A05F0070201EB022135F0AE
:201730007F05A1F104011FFA81F840F0D782B8F5006F80F2D3820A3041460EF09DFFE169DB
:2017500004F114000522083115F0C8FBA8F1030305200D961FFA83F8E27DA57D217E0B9B87
:201770006081C2F3011B93F83860617105EB02255EB161480078862807D1BBF1020F04D153
:2017900005F00700022840F0A982281300F0020ABAF1020F58DAA37805F00700022841D140
:2017B0004E467068002B0C903CD1E16909A801220D3115F093FB062060810C9880478046B2
:2017D0000C96C74F4C48B6683A680078862819D122B915F069FD48463A6886689DF92400BF
:2017F00015F0ADFF9DF924705077002090774046D777B04705F0100010F098F904E0C046C5
:20181000E41A00204046B04715F088F96AE2C046CC1A0020280D002028160020CD1A002085
:201830001C320020344800780026862808BF0126CDF830905EB1002012F0CCF9E77805E0B5
:2018500000000C8C90190020CDF83090A37887B17BB9012F00F03D82022F03D115F0070F0C
:2018700040F03782032F04D105F00700032840F03082280908D315F4405F00F02A82C74800
:201890000778002F00F02582BAF1020F02DAA80A80F01F82C3480078C0F381098611B9F197
:2018B000010F00F01682012E00F01382BBF1030F00F00F82BA48BBF1020F0BD010F80910D2
:2018D000805D4018C7B22EB3E80923D3BF1E0EE0CE1A002000EB09018019097900794018CE
:2018F000C7B2E80912D259EA060313D0BF1CFFB210E0C0462414002020320020EC130020F0
:20191000883100201E3200208C14002059EA060308BF0227C5F3002BA7EB0B008045C0F27B
:20193000D881A8EB07002909584480B2208124BF2521109110994018743080B215F0C0FBA2
:2019500094F80280E060002800F0C381002174220FF013FA0020B8F1000F207103D10D9927
:2019700005F0200008700D9803784FF00008002B52D0BBF1000F4FD1D748008805F0070197
:2019900003291ED18108424609D3554991F82E30A3B90B681BB15B7E33F07F030ED16AB98F
:2019B0008008C24607D3D7498B68887813B1984794F8048010B9BAF1000F02D004202071DD
:2019D00080460B9894F805A090F8383033BBCE49002352460220B8F1000FCB7201F10A0A90
:2019F0008AF80000AAF1020007D000F1020A9AF8001041F010018AF800100A990271052231
:201A1000A1F87820C1F8840014F0F6FB504603210EF032FE94F8048094F805A0E16801F1EF
:201A300074004860886523890B812089A1F85C0028090ED3CBF1030082B2A1F85C20886DA8
:201A5000D44915F04BFAE1688A6DB1F85C00801888655448CF4B0078C0F3011218788D81B3
:201A7000BBF1000F00F0780040EA020048EA00050D744FF0FF038B7318BF4FF0000A81F877
:201A9000306081F83A9081F849A06089002FA0EB0B0085B2658100F01481E069E7802918C0
:201AB0003A460831684615F019FA3E48EE19B5B26581E16800780A7C6E46C0F38103C0F3D8
:201AD000011BC0F38108002B02F0400A4AD0C0F301100023022805D1D0090FD202E0C04694
:201AF000640E00209DF801209DF8000000EB0220A1F844000DF10206A1F84200AD4AB1F88E
:201B10004400B2F84A20824203D04FF6FF72824222D1B8F1030F12D072783078A54B00EB4F
:201B3000022082B24A86B3F84810B61C0120914211D04FF6FF71914218BF00200BE0E06813
:201B50003146323015F0D9FDE0689A4932303F3114F0F2FF08360346002B00F0B580204692
:201B7000E168C07D831125D0BBF1020F03D0087CC00903D309E05AEA080206D172783078F3
:201B9000B61C00EB0220A1F84200032B0CD07078327802EB00220A850CE0C04644120020D9
:201BB000B88A01009F310020E0683146283015F0A4FDE16888890009C0F08380886D3A469A
:201BD000694615F08BF9E068816D79188165E669B0F85C1001227F18A919A0F85C70083194
:201BF0000DF1250015F07AF96F1CBDB26581E1689DF82500896D0870E2689DF825609DF8F0
:201C10002530906D401C9065B2F85C00401CA2F85C0006F0070082F82400C3F3C10182F82C
:201C30002510208992F824708046002F4CD05F4F7F183E78361D8642E68045DCE069291860
:201C50003246083105A815F049F93A789DF817C0111D481980B29DF81450608105EB0C60BA
:201C7000E3689DF8165000EB05409DF81550042900EB052098610BDDE06806A9521E1C3013
:201C900015F02CF93878E3686844C07D83F82600986D05A9324615F021F9E068816D71187C
:201CB0008165B0F85C10A8EB06077118A0F85C10791E89B22181B0F85C2001818918A0F89A
:201CD0005C1000F07FF80DE015F04EFC10F010FC08E015F059FA05E02015002015F054FA0C
:201CF000CDF83090DDF83080D8F804008047E1690A68002313710968E161D8F80810884762
:201D100013E0C046381A00209418002040462A4F00784146401C087097F900003946401E3D
:201D3000087010F0E5FB14F05BFC0A980B9D214F00216FF00106A0F8B21095F83800FE8002
:201D500010B11198007808B915F080F81B481B4990F90000401E0870174890F9000010B97C
:201D7000134800210170154890F90000A0B10F9F0E9A4FF0E040022138401140002808BF9F
:201D900000290DD00D4890F90000002808DC15F08BFA05E09E3100200020014605F0AAFEE1
:201DB0000749002013B00870BDE8F08FA08A0100CA1A002028160020CE1A0020CD1A0020A8
:201DD000E41A00202DE9F04FB84CE0686189E2692589806DADF13C0D0E46891808312A46DF
:201DF00015F07CF8A81986B2E068816D6D188565E0690122311808310CA815F06FF8761C1C
:201E1000B5B20422E06965812918083104A815F065F89DF813109DF8100000EB0160E3687A
:201E30009DF812102D1D00EB01409DF81110658100EB0120049015F061F9D863049814F0EF
:201E5000FDFDA3F84000EA2014F0C5FE0220B849E26808702079117C084310749DF930002C
:201E700015F06DFC82F8460011899DF93000DFF8C4B282F8480002F174009065B2F85C0053
:201E9000401A51684FF0000909185160908982F84790830A18D2030957D310F0070F07D001
:201EB00000F00700032812BF081C5068401C48E05068C17801F00703491001F0380101EB64
:201ED00043014018001D3CE0171C02D115F0ECF9E268B889800A2ED379684878C6112AD1A4
:201EF0003E89796648464D780B7805F07F056D0005EBE3157E2D0DD07F2D09D003F07F0306
:201F10001818801C5B1880B2991C8642EBDC08E0494600E00121801C87F8601080B28642FE
:201F300001DA484605E07968411879603989091A3981A7F86800506E10B1B2F86800B0B198
:201F5000506850619089000916D292F86000002800F0FE80104611F00FFAE268D06C002870
:201F700000F0F680B2F85000002840F0F18015F0E9FA4846E060E0E14846154605904E469F
:201F9000069005A907AB06AA95F824700796284604F0FFFC002840F0D080059A6E69686882
:201FB0002B89311A581A1FFA80F80AB915F07CF9B5F85C0000900196CDF808800698001D9A
:201FD00003900598A969AB6D3A4615300AF060FC002840F0B280B54895F860302E89C15D03
:201FF000701A288113B1284611F0C6F9AE8906F00706032E02D168680078E87395F80F80AF
:20201000732009A913F0BAFE83200DF1320108F09BF8484649460D900AE0C278012A03D174
:20203000002F08BFDC2027D0001D491C0990C9B29DF8320088427FDD09988278032E07D081
:202050000378B3420DD09BF800300BB1022E08D0032EE9D10378032BE6D103465B784345AD
:20207000E2D1BB10B3EBA20F05DA02F0030207F003039A42D1DD48468246059895F80FC0D7
:2020900090F814E04946D84601E0491CC9B28E454CDD07694B00032E03EB070208D1FB5C37
:2020B000032BF2D152786245EFD10AE0883100201278B24205D098F80020002AE5D0022E19
:2020D000E3D10698077D002F08BFBAF1DC0F33D0A869B0F1FF3F27D0712008A913F04EFE13
:2020F000AA69089B484605998B4207D10699064601EB8601C9680D96914213D8401C2C339E
:202110000228F0DB06980D99521CB2F1FF3F00EB8100C26002D107980121817085F8019006
:2021300048460BE0DB2009E0DB2006E0DC2004E01C32002024140020DD206870E2685070CC
:202150009069577850651FB1F22014F044FDE2687C4DDFF8F88195F83800002874D091891D
:20217000794E01F00701022938D1A778002F35D15778002F32D106F11C010888EB6D401CAE
:202190000880506E8DF831900DF131020421984730B94046006818B19DF8311080F8681008
:2021B000E1680DF12E0000906D6E486E4A460BAB2831A84766480078862808D1F08BE76874
:2021D000401CF083B88900F010000FF0AFFC15F0B9F94846E06014F0A1FCB0E05D490F7852
:2021F0004FB35778002F40F0A8809DF83000378C20702379781C002B308402F1280602F13C
:202210001C020CBF4B46082353484946016014F0D5FD0146009351480192038832460D2072
:2022300005F08EFA10B913F0E7FF01E014F014FC5846E268007838B1D5F8801021B110469C
:2022500088475846E26800780A9210B1907BFF286FD0938913F007003DD0401E53D0801E1F
:2022700067D1C3F30130022803D15068007807282FD0108900285CD0104641684A1C4260DF
:202290000F788446C7739CF824608EB9002F50D00A2F4EDA0189324EF01910F8010C8842A2
:2022B0000BD0082F45D1082907D042E0A48A0100C07B00283DD00A283BDA60460189491E3F
:2022D0000181C17B0B3101700A99C87B401CC8731BE0322018E0234E96F871000F280CD03E
:2022F00014F02AFF48B9181300F00200022804DA4046001D01680A98884796F8A7000A9A25
:202310001074152000E0162010700A99454605F1280013F01FF8144E7068804795F830102A
:20233000491C85F83010B1688847202015F00CF84FE70AA812F010FA4BE710F0D9F80FB084
:20235000BDE8F08FEC130020C4180020640E0020203200201E320020981800203212002086
:20237000D4860100A81100208C1400202DE9FE4FE54980460122A1F130000260DF48076825
:20239000002FFCD0DE4ADF4EC027E048E04B17603268920808D2324652F8042C03F14104F3
:2023B000120C42F0F00222704FF0000A8346C1F800A0DFF864C3DBF80810D64D0191880E9A
:2023D00043D2480E41D3802018744FF6D802A3F8512018702868C0F30464162CA8BF203CDF
:2023F0001F460F3F387800F01F001628A8BF2038844223D0624602F1980EDA4ACEF800A0DA
:20241000261A022E05DC16F1020FB8BF6FF0010600E002263018166800F01F06844246F483
:20243000F856A7F866604FF001061660E8D11068374617601068CEF800601068284600680C
:20245000C0F30420162808DB06E0A5F1D0000068C0F30460162800DB203800EB2170401C60
:20247000162805DA10F10A0FB8BF6FF0090000E01520DE4F00F01F0040F4F850A3F8590075
:20249000386880083ABFEA48C0F800A041F04061019E6246A5F13804C80E8F0E80F00100B2
:2024B00000F00100106087F0010000F0010090602068C0F38367C0F38F21B00C23D23046A3
:2024D00040F3072000280BD542425046490805D17F0806BF0127391C4FF6FF71521EF5D195
:2024F000002810DD4FF6FF72490041F001018A4207D27F0047F001070F2F92BF01210F273B
:20251000111C401EF0D141EA0741182012F038FE2068D24E2768C94CA6F10409C0F3870151
:2025300007F0030041EA0021D9F8040040F2FF3253468FB22C21466800972746A7F140005C
:20255000B0470C3D2868C0F30D011C2012F018FEB84955F8080C014000F07C4001431420BF
:2025700012F00EFE55F80C1C01F47C000904090C0143102012F004FE624955F8042C096824
:20259000C2F30350C2F30343490813D2DBF800100D0510EB257003D41028A8BF0F2000E0E8
:2025B0005046090413EB217303D4102BA8BF0F2300E0534643EA001302F47F4002F0FF01CB
:2025D000B8F1220F40EA034041EA000124BF02F0804211430C2012F0D3FD974DB8F1220FD1
:2025F00032BF01202868C0F30070B8F1220F4FEA400040F0200084F8090126BF2868C0F3B5
:20261000407001208E4EB8F1200F40F0100084F8090138BF514606D33168C80C00F44070E7
:20263000C1F384510143282012F0AAFDB8F1200F26BF3068C0F301505046B8F1220F4FEACA
:20265000400040F0600084F80C0126BF2868C0F3C0605046B8F1220F4FEAC00040F08000B0
:2026700084F8010126BF2868C0F345505046B8F1200F4FEA800040F47C40A4F89C0138BFC8
:2026900070490AD3306801038A15920501F47C1100F00F00114341EA0031082012F070FDFA
:2026B0004FF48000A5F1D0012060674A886D40F21E236FF31F40834216D90868030E13F04E
:2026D0000F0F03F00F01C0F3034018BF491E072805D006280EBF0720801C00F00F0041EAA9
:2026F0000011A2F108000170DDF804C0CCF381477F1E13D07F1E3BD036E0C046940222434E
:2027100000600C40B03F005040100940AC3F00501562084088130050000020432846006807
:20273000810C21D24FF480412160D2F80210430AC0F3033703F0800321F08F010B4347EAD8
:202750000301C2F80210D2F80130060A66F30303C2F80130116800F0E70721F0E70147EAC3
:20277000010004E02C2009404FF00040224610603B480068C0F3C0070FB94020A0624FF4A6
:202790000070206428684027C0F3C14040F0300084F8C800CCF3815050B3401E03D0401EC4
:2027B0001FD002211EE0012013F090F90646042031460FF095FF042013F088F98642FAD197
:2027D0002248066826F07F4012F04EFFD9F81400036807214FF06022300E98474FF4806074
:2027F0002060032104200FF07BFF08E000000940042001210FF074FF154812F035FF203DAF
:202810002868144947F6180600F03F0084F8CB0F144B0E80D9F800201868D1680220884753
:2028300011480D4D076001212960BDE8FE8FC04694042A43FCFCFC008C13005040A00C4077
:202850009813005000803F400A600840A83F0050BD37860070B00C4094046042A4010010B0
:20287000B03F00502C20094000600C402DE9F04F0320ADF15C0D12F027FFD14D00240220BD
:2028900005F11C0141F80C4F401E8C60FAD105F14000062701467F1E21F80C4BFBD14FF0AA
:2028B0000808C849A0F80080C74E8160C749361D26F003000B1A2B62A861E861AA6905F150
:2028D0001C09B44607460E46914200F2E581991000EB810121F8044CE8233B804FF6FC7700
:2028F00007EA0C0200F1E803B61A2B6107EA0601EC39A0F8E81020460DF03AFE6861C9496E
:20291000D9F80000DFF8C89228610A6809F10C00026049684160C4498246424613F0B4FCE0
:2029300028B9C24801685246116040685060C048C14FC24EC24BC764BE490665C14A43654D
:20295000C14F816400F1480B8265C04EC765C04B0666816C436609B1204688470FF056F9C3
:202970002146D24E15910C220E9106F120000EF004FACF4F0222ADF8208041F270737762C4
:20299000708CADF82220696AB3621027099740F01900708408A8884700280CBF0A9F271CEA
:2029B0000120ADF82C80696AADF82E000BA888479DF830004D4628700D9969605FB1D0210D
:2029D00039707C70B870FC703C713946BC600220FC6011F09BFFB749182001220DF0F4F918
:2029F000E220514614F050FC182012F07BFB68706868B246CAF808000BF02EFC0AF1700034
:202A1000AD4EA860DAF80870C6F824B0AB4DB76005F10C0105F118000DF00EF8A8600D206F
:202A300014F030FB00B1A0460E2014F02BFB08B948F01008A249A86814F05AFDA149C8222D
:202A500005F1240011F034FA9F48B8F1100F68604BD113F07DF8706A002846D0C268002AA6
:202A700043D006278DF810700220ADF8120004ADADF8144095E80300904725468DF81070B7
:202A90000320ADF81200706AC268ADF8145004AB93E8030090476D1CB5F5FA7FF3DB756AE2
:202AB0008DF81070042004ABADF81200EA68ADF8144093E8030090478DF81070052004ABFE
:202AD000756AADF81200EA68ADF8144093E80300904704AD8DF81070706AADF81270C268CF
:202AF000ADF8144095E803009047DFF8E09109F1140009F108010CF09FFFC9F80400204658
:202B100014F014FD25464FF006084FF0040B1490A9F1020707F8024F02207870284614F077
:202B300076FD0146149AD9F80400C9B212F072F96D1C022DEEDB664909F120004FF4FA7267
:202B500011F0B6F9706A00284FD00769DFF884916FB10096494612A80A688988026012AD95
:202B7000818095E8030001232246B847706A00283BD0C26852B1494612A80B6889880360CF
:202B900012AF818097E803009047706A68B307695FB38DF80880ADF80A8010A8ADF80C40AE
:202BB00002AD009095E8030022460223ADF84020B847756ABDF840006F69B080AFB109E090
:202BD0008C140020D164010021320020004B0020101A0020BDF8400002AD401CADF84000E2
:202BF00095E80300022210ABB8472DA014F0F4FA706A00283ED00769002F3BD08DF81880D1
:202C1000ADF81AB00EA8ADF81C4006AD009095E8030022465B46B847E0B90E981930159086
:202C300028E0C046C8FF0100D88A0100F0120050080200209D9E0000A9450100A12A0100D9
:202C5000F5140100110C010051020100FD0D0100B93601008DF818802046776AADF81AB01A
:202C700006ADADF81C407C690F9095E803005A460FABA04715980E900DF008FFE0200E21CD
:202C900013F0DCFF13F078FE0AF10200012113F09DFE01F093F9FCE722F8024B14E6C04649
:202CB00054492053656E736F7200C0469012002020BF020009890000A41000201417002073
:202CD000955201006D6D0100056F0100A8170020D9020100FE8A01002DE9F04FADF18C0DDC
:202CF0001C911E93CC491D920A6806460DF156000260496841603046694612F0A3F90028F1
:202D10001F9004BF0020229000F0F78102200027B61CDFF84CB32090D34D2297304602A95C
:202D300010F0A7FB5FEA000900F0E48122990EA816220EF022F89DF809707F1E00F08280DC
:202D50007F1E40F0CF81B9F10A0F40F3D681B61C316804A80160361D318805AF42F20B0082
:202D700039800DF1160110F005FEBDF81600BDF81410884200F3C181B61C16F8010B16F8D5
:202D9000017B16F8014B8DF8380016F8011B8DF839700EAA8DF83A40304605F01FFBBF49F4
:202DB00009780028064400F0A8811F9C012904F1020400F091814FF400500DF14E0110F035
:202DD000D9FD0DF14E000DF15601082213F05CFA40B11C990DF14E00082213F055FA002853
:202DF00040F07A8142F2010004A907F0FFF842F20B0005A907F0FAF842F205000EA907F00B
:202E1000F5F80DF1390142F2060007F0EFF80DF13A0142F2070007F0E9F80DF13B0142F2AB
:202E3000090007F0E3F89DF83B0028B1022840F0538142F2030001E042F20D000FA907F0C8
:202E5000D5F849E1B9F1040F40F35781B61C16F8010B16F8017B16F8014B8DF8380016F808
:202E7000011B8DF839700EAA8DF83A40304605F0B5FA0028064400F040811C9806A909F0A8
:202E9000A7F99DF83600002840F00A819DF83B0000287AD195F82D70002F00F0FD8095F83E
:202EB0002F00874207D095F888000A2801D10AF063F9686B1EE06F6B4FF400500DF15E0129
:202ED00010F058FD13F0DCFA4FF0FF08229C2190A24695F82D00A04240DC686BB8F1FF0FD5
:202EF00008D008EB88040019007912F0FDFA686B071923D195F82D300746002B08BF229C12
:202F100019D05846229C40681946D8467F1F7F1DFA782AB1491E04F10104F8D17F1D0AE000
:202F3000804795F82F10491C85F82F10D8F80810884795F82D30A34200F094801C980BF094
:202F50008BFF38710120F870FC788DF8364038798DF83700229B8DF82330A1E0387910F002
:202F7000F3FE014608220DF15E0013F08DF940B138880104219814F0CEFB82453CBF824634
:202F9000A046641C7F1DA4B2A3E795F82C70002F00F0828095F82E00874207D095F8880085
:202FB0000A2801D10AF0E8F8286B1EE02F6B4FF400500DF1660110F0DDFC13F061FA4FF08A
:202FD000FF08229C2190A24695F82C00A0424DDC286BB8F1FF0F08D04FEA48140019C07FB0
:202FF00012F082FA286B071925D195F82C300746002B08BF229C1CD0DBF80400229C1946D4
:20301000D846203F2037BA7F42B1491E04F10104F8D120370DE0C046C88A0100804795F885
:203030002E10491C85F82E10D8F80810884795F82C30A34216D02299384620220DF09DFEA4
:203050001C980BF009FFF8770123FF2039462022BB770446787206A8FC720CF021FB1FE09D
:203070008C140020612055E0A42E0020F87F10F06BFE014608220DF1660013F005F938B139
:203090007968219814F047FB82453CBF8246A046641C2037A4B297E764203BE0ED13002066
:2030B0009DF836000EA9162240F004008DF8360008A80CF0F5FA1F9C9DF83B00A41C40B180
:2030D0009DF84D700FA839460FF024FE3F1A8DF8357006A80FF0AEF820984844801C80B24F
:2030F000209003E01F9C4E44B61CA41C209884423FF714AE2098022803DC229A672011467D
:2031100004E01F9A911C121A2298921C1D9B19801E990A8023B0BDE8F08F70472DE9F04F2C
:203130000F46C64E42680168ADF14C0D726080687162C54CB06077B1C1487A68C761BD69FD
:203150004262BA68026225B1BE4D14302860BA690260F86820604FF008084FF0010AADF8E5
:20317000188006A8ADF81AA08847B84D9DF81C10089B69706B6108B113F056FB3868804749
:20319000706880474FF400578346ADF800801E200197716AADF802006846884711F076FDAF
:2031B0002068406880472068C16810A888472068836810AA002001469847606008B913F0D9
:2031D00033FB13F047FDA248A34FA24A2861A34C1760A4495460A24BD160A34FA448936023
:2031F000A24C1761A34F546100F118013964BA64A14B3B651439796403F140029F4B7B613B
:2032100003F16A01B9619E4BFA649F497B629D4B19609E4959603B669D4999600024AC6068
:2032300080F838409B49D9609B4999619B4999629B499C4A99639D4B13619D4B53619D4B0E
:20325000D3619D4B13629D4B1C635C634FF0FF0983F8389083F83B4083F83C4083F83D4038
:20327000AF49C0F89C10904B53601123BB81944AC263944B0364944A4264944B8364944A73
:20329000C264944B0365944A4265944B8365944AC265944B0366944A4266944B8366944AEC
:2032B000C266944B0367944A4267944B8367944AC267944BC0F88030934AC0F88420934BD8
:2032D000C0F88830924AC0F88C20924BC0F89030914AC0F89420914BC0F89830914A1460E7
:2032F000914B83F800A05C80022012F04BFE0222E862494614F027FAE81C0222494614F0A1
:2033100022FA022012F03EFE8849086008680222214614F018FA11A80FA911F0D3FCE86A44
:203330009DF84410421C01709DF8440010703C709DF84400A87013F063F8A861716AADF8E8
:2033500008801420ADF80A0002A888471527ADF810800398ADF81270716AE86104A88847A7
:20337000744F05983C70801E2862734B1C70704D6C70AC7040F60D00EC6013F0A1FE40F2A7
:20339000FF7907468DF8284009A94246ADF82A909DF829002F6100F0F0008DF82900286965
:2033B000099713F09BFD2C62EF616448A0F8009011F0B2F9624D2878012803D0204601466C
:2033D00004F098FB5F4804705F4F3C702878012803D02046014604F08DFBB1685846884796
:2033F00002F046FC13F026FD5848007811F07EFB5046214604F07EFB11F04EF9544804700F
:203410002878012803D02046014604F073FB0FF0A1F81820ADF830804E4FADF832004E4DBD
:203430000D97716A0E950CA8884708B113F03CFF01F074FD13B0BDE8F08FC0468C140020D1
:20345000281600205C1700200432002064180020C73C0100B030002055870000B1270100C0
:20347000A7670100DDC0000055DF000055100100EC1300201415002038300020AE830100D4
:2034900029E300001C31002049AF0000B1A20000A9370100054F010011280100BDEB000040
:2034B000F3760100640E0020AD6D00004DCC0000CD5E0100650F0100854A0100EC17002039
:2034D000E9F7000075750000251301008D5001007580000061EA0000614C0000E92C0000F9
:2034F00095FF0000A97E000069CB000045700100FD9F000085390100C560010011D40000B1
:2035100011B500001DAE0000E367010001E90000C9350100A1600100B54001003129010083
:203530007D740100003200206C0A0020242D0020883100201C3200201E320020F00D00205C
:20355000E41A002020320020183200204F1200201D320020E7F70000DC1900202DE9FF4722
:20357000D64C0F460546F80B80F08B81B80880F07881F80A80F05181DFF84483DFF844A331
:20359000B80F80F0D080207A002854D1380954D3002525700126A671284612F0C1FFD14804
:2035B00013F06AFFD0492A4604F1580014F0A8F804F1400090E8000313F05AFD2379B0EBD4
:2035D00008004FEA103071EB09010905012B40EA0100E0640DD194F85010B0EBC12F08D816
:2035F000E07830B904F1D4004FF0005113F0BEFC17E040F609002671BC49208504F12803CD
:2036100094F83500E57000F0F00040F0010084F8350094F834000B6000F0F00084F8340007
:20363000E5622846294604F1400282E80300E06427F008074DE1380972D2B80B5ED2780B1F
:20365000C0F04781AE69CEB14046B04216D0A86843681BB105F1200199424DD1407B10F09C
:203670000F0F0BD1688C40F60901814206D128466FF4807100224FF00073B04704F1580098
:203690005146002214F03CF8A96800264FF0010840F602026672088884F80080824207D071
:2036B0000A8B4FF61F60104040F43470088306E00A8A4FF61F60104040F4347008826E741C
:2036D00013F0D6FCD4F83C21E36804F59E719A4208BFB046A56C45B1854226BF281A401E9D
:2036F000401B01EB8801000B8860A664192013F033FE27F48057ECE01846A9E704F11800C7
:2037100014F013F8061C08D0706830B17568F068B6F9241000222023A84727F40057D8E041
:203730000020207284E7A968088840F60209814507D00A8B4FF61F60104040F434700883D1
:2037500006E00A8A4FF61F60104040F43470088204F1400090E80C00002B08BF002A1AD0AA
:20377000042012F0B3F9B0B1266C13F081FC864226BF801B401E801B000BE860E968688A1D
:20379000401840F6C411E860814203D340F2EE22824200D9E960AE699EB14046B04210D0EF
:2037B00094F8350010F00F0F0BD1698C09F10700884206D128466FF4807100224FF0007311
:2037D000B04704F158005146002213F099FFB4F8AC004FF6FF71814209D10220ADF80000D0
:2037F000684612F0F3FABDF80800A4F8AC000120207013F0B3F84FF00008192084F8058037
:2038100013F0AAFD6E692EB1414628464FF080630A46B04727F000575BE014F077F8054673
:2038300004F1140013F081FF061C15D0E06810B1703012F035FFF068E060284614F062F8A2
:2038500013F016FCA0642A4813F016FE4FF4006104F1D40013F08AFB002027F4806720720D
:2038700037E004F12005284613F05FFF07F0B6FD284613F05AFF27F0020708B147F00207AB
:2038900027E014F043F8014604F11C0013F04DFF0646B569A80817D2B6B125EA0500B0619C
:2038B000084614F02FF8706888B185B12A46F068B6F9241075680023A84708E0700A00201C
:2038D000738000009DBA0000084614F01BF827F4804727B104F1D400394613F047FB009052
:2038F000BDE8FF8791E70000796101000010044045A90000B0B50446BC480768ADF1480DE3
:20391000002F00F0AC812078401E112800F2A781DFE810F06E0156013C0127011F010801E7
:20393000F100E300C300B2008D005D0053004200A5012A001C001200F86B002800F08F8126
:20395000684621460CF0ACFBF96B86E1386C002800F085816846002101220DF00EFA607843
:203970008DF80000396C78E1F86A002800F07781684600210E220DF000FAA11C684613F0DE
:2039900005FAA57BA1890022ADF80A1005B101228DF80C20F96A61E1B86B002800F05F81A3
:2039B0006846002102220DF0E8F9A5788DF8015060788DF80000B96B4FE1786B002800F087
:2039D0004E81684621460CF06BFB796B45E1386B08B36846002114220DF0CFF9A5788DF8BD
:2039F0000150A3680193A289ADF80820A17B8DF80A1060788DF80000E57B8DF80B50237CD8
:203A10008DF80C3094F911208DF80D2061690491396B684688476068002800F0208101461D
:203A3000F22008700020487010F070FF17E1B86A002800F014816846002124220DF09DF936
:203A50006078A11C8DF800000DF1020013F09EF904F10C0103A813F099F9257EE08A04F15E
:203A700019018DF818500B22ADF816000DF119000BF016FEB96AF0E0786A002800F0EF80C5
:203A90006846002102220DF078F9A5788DF8015060788DF80000796ADFE0386A002800F009
:203AB000DE806846002112220DF067F9658862796078ADF8025023798DF80520E11D8DF8D8
:203AD0000000A5798DF804300B220DF107008DF806500BF0E5FD396ABFE0F869002800F05A
:203AF000BE806846002101220DF047F960788DF80000F969B1E0B86910B120460FF066FC50
:203B1000A07D002800F0AB80A07820B9A069002800F0A58003E0A069002800F0A08012F0D8
:203B30004FFC9CE07869002800F099806846002113220DF022F96D46A01C01684068296077
:203B50000B22686004F10A0102A80BF0A9FD796983E03869002800F0828020460BF07CF840
:203B70007DE0F86800287AD0684600210E220DF004F96078A11C8DF800000DF1020013F0F0
:203B900005F9A089ADF80C00F96866E0B868002865D06846002114220DF0EFF8A01C01680B
:203BB0006D46296040686860A07A0B2204F10B018DF808000DF109000BF072FDB9684CE0B6
:203BD000786800284BD06846002110220DF0D5F860786588211D8DF800000B22ADF802503B
:203BF00001A80BF05DFD796837E0C046181A00203868A0B36846002119220DF0BEF8A01CFB
:203C100001686D46296040686860A07A410824BF01218DF80810810824BF01218DF809104E
:203C3000C10824BF01218DF80A10010924BF01218DF80B10C10924BF01218DF80C1030F0C8
:203C50007F001CBF01208DF80D000B220DF10E0004F10B010BF024FD39686846884712B011
:203C7000B0BD70472DE9F04FDFF8B4C292F808B009AF88460646ADF1240D049338F07F0548
:203C9000039206BF604600884FF6FF700590F08A800934BF002008203076F08AC00834BF2A
:203CB000102080207076F08A400903D260460E30007800E00020B076F08A41082CBF202432
:203CD0000024000928BF44F010047568002108F07F08307D06916D1E02280EDB0C2808DC01
:203CF0000C2803D1022044F40854069044F0030404E00D280CBF02200120044396F88800A1
:203D100008B144F00804210900D328B1DFF89C9299F89C3013B908B1DF203BE121096DD358
:203D300096F88950DFF888A206F1240133891AF8052007910AEB0001097908908918491D4D
:203D5000C9B2C918B1F5006F80F2268100284CD0049A039906F1800009F0FAFE079900281B
:203D700008603FD0806AB0F1FF3F39D070680023401E8DB196F88A10524600F80119515DD3
:203D9000491EC9B241B1721892F87F20491EC9B2002900F80129F6D1079970660968896ABE
:203DB000B162090E00F8011996F82A1000F8011996F82910089A00F8011996F8281005F0A7
:203DD000030500F8011902F0070141EAC501017071683289091AC9B270608918318105E023
:203DF000DB2700E0F3277770D7E00023F08A7370C00828BF44F0100475686D1E336DA3B93E
:203E1000B36D93B999F8B510012903D13089B0F5EE7F06DA200904D202290AD144F4005496
:203E300001E044F48054012002E044F408540220069044EA8834B8F1020FA4B20AD0B8F1B9
:203E5000030F10D1ED1F09F1A801284613F055FC6D1E08E0B9F88E00001205F8010999F892
:203E70008E0005F80109069802280CD0B8F1000F15D0BBF1000F0CD004990598814208D1EF
:203E900044F040040BE0BBF1000F08D1B8F1000F05D00599081205F8010905F8011944EA8A
:203EB0008B24BBF1020FA4B209D0BBF1030F0ED10399ED1F284613F020FC6D1E07E0039977
:203ED0000888001205F80109087805F80109BBF1000F05D00498011205F8011905F8010945
:203EF0003878F8B933480178307D0D2814D068B9306D28B999F87800411C89F878100AE09F
:203F100099F89D00411C89F89D1004E099F88600411C89F88610014605F8011904E0C04621
:203F30003212002044F48074201205F801092C7070683189401B7560C0B2401830812009A6
:203F500027D3B06D00B130621B48007810B1307D0D281ED1726A12F1150002D113F0A4F923
:203F7000726A916A481C9062306A3289B162471B0092D21B019090B20290706A96F8882046
:203F90002B46153007F0DAFB00281CBF7070071C07D10020707005E0E5277770F32012F0C4
:203FB0001AFEF8B209B0BDE8F08FC046A8110020A08A01008D310020241400202DE9F041CB
:203FD000CB4CCC4DDFF834836088ADF1600D4108C0F08C800CA808A90DF0C0FF012879D187
:203FF000404624300068D8B10769CFB1062002268DF808000022ADF80A600FABADF80C205F
:2040100002AE009396E803000C23B84740B9BDF83C006084109F67621198A06213F014F89E
:204030009DF82D00012805D002202077BDF82210A1820AE0032009AF20773A6804F11401E5
:204050000A6078684860BDF82210BDF8200009AA00230EF0C1FC011C02D0A1A013F02FFBB4
:20407000022011F0ABF9BDF830009DF82C7028870DA985F83A7005F1480013F0C3FABDF814
:20409000320005F13E0609A9A5F84600304613F0B9FABDF82200298FA887502012F0C2FDF4
:2040B000B5F84610532012F0BDFD4A20314613F0EBF895F83A10E12012F0C0FDA98F4B20BD
:2040D00012F0B0FD05F10800102112F07FFC0120207005E0012011F071F9002013F068F8D0
:2040F000A01C012112F064FC2046408880080DD3606A11F019FB11F055FE00B2A081E08173
:2041100001F0E0FEA01C022112F052FC2889410805D305F10800012112F04AFC288981081D
:2041300005D305F10800022112F042FC288901094BD395F8540005F1080600283DD0401EE5
:2041500039D0401E02D0401E33D039E095F85010472012F073FD95F85110542012F06EFD07
:20417000A98F4B2012F05EFD298F502012F05AFD0927032395F83A008DF8597016AA8DF8FE
:204190005A305D498DF8580001278DF85B7018200BF01AFEB4F84E00B4F84C1088420FD193
:2041B00095F8520001280BD13046202112F00EFC06E0032002E0022000E001200EF006F83E
:2041D0003046082112F0F4FB2889410911D395F8520005F10806032818BF042802D1A86D67
:2041F00011F08AFA10F0FAFC3046102112F0E0FB2889810907D30CF0D9FF05F10800202188
:2042100012F0D6FB2889C10907D30CF0FBFA05F10800402112F0CCFB2889400A0DD395F8E5
:20423000550012F0C5FF41F2883011F095FA05F108004FF4807112F0BBFB4546E8884008AB
:204250000DD368780026000904D3A878012801D110F098FB6E70A81D012112F0A9FB608887
:20427000002839D10A200825254CADF812004FF0FF37ADF81050616A059704A888470028F9
:204290002AD10720ADF84850616AADF84A0012A88847149E1596F8B91A499DF84E20087878
:2042B00090420ED19DF84C004A78824206D089684B6C33B100213246984702E03046FFF7AE
:2042D00019FB159840B1ADF818500320ADF81A00616A079606A8884718B0BDE8F081C04664
:2042F00041757468204572726F723A20307800C090120020481300204D760100A41000205B
:204310008C140020101A00202DE9F04F09AFADF13C0D08900A92388809911E46ADF81800E0
:20433000101C08BF002000F08481002700F101094FF0FF3A4FF0010BB8466CE1252940F0B7
:2043500063811078521C0A922D2818BFADF8068005D15846551CADF8060010780A95302871
:204370001CBF4246434605D10A9908785A465B46491C0A912A28CDF80080554616D1306856
:2043900004930A99CDF808A0C01C4B1C20F00300001D306050F8044C0A93002C08780094EE
:2043B00018D5ADF806B06442009413E044460AE0610001EBC40140180A99A0F130040878B2
:2043D0000094491C0A91302801DB3A28F0DBCDF808A004932E282BD10A9908782A2801F11B
:2043F00001010A9111D13068CDF80880C01C20F00300001D306050F8045C002D48BF454646
:2044100008782B46491C0A9111E0454643460AE0690001EBC50140180A99A0F13005087850
:204430002B46491C0A91302801DB3A28F0DB02930AB1224604926C2804D04C2818BFADF8F4
:20445000048005D10A990878ADF804B0491C0A910BA9CDF80C800FAB07916428059300F00B
:204470008B80692800F08880BDF818C0752872D078286ED06F286AD0702850D063283DD02D
:2044900073281ED009980A990128A1F101010A9115D96B490C68B5F1FF3F03D0A84288BFE9
:2044B0006D1C00D8099D029508A80AA932466B46A047C7190A99039801F1010974E04046E7
:2044D0002AE030680A99C01C20F00300001D306050F8040CBCF1000F01F10109014608B9D3
:2044F00055A00146079112F045FE0390B5F1FF3F5BD0A842C4BF281C039056E03068C01C03
:2045100020F00300001D306010F8040C5D468DF82C000A990395584601F1010945E008203D
:2045300035680490E81C20F00300001D306050F8041C082210230FA80DF030FB401E0790DD
:20455000402101700A99079801F1010929E0082302E0102300E00A230A99306801F10109AE
:20457000C01C20F00300001D306050F8041CAA42BCBF2A1C049210E00A99306801F10109BD
:20459000C01C20F00300001D306050F8041CAA42BCBF2A1C04926FF009030FA80DF0FEFAAD
:2045B0000790059D281A0390009C241ABDF8065000945DB906E008A8202109AA11F078FB50
:2045D000009C7F1C641E0094F5D503980546401E039075B9BDF80600E8B10098401E0090D5
:2045F00019D408A8202109AA11F062FB00987F1CF4E70798411C0791017809AA08A811F03D
:2046100057FB03987F1CE1E708A809AA11F050FB7F1C09F101094A460A9812F8011C401C37
:2046300000290A907FF48AAE089808B14146017038460FB0BDE8F08F286E756C6C2900C07E
:20465000208B0100BA492DE9F84F00254820C1F8F35FB84CC1F8FF0F94F8E200002800F055
:204670006381012800F02F81B34E02283CD0032840F05A8151F8310CD4F8B8100029A0F538
:20469000C060C4F8D400B8BF49420028B8BF4042814226DA4FF08057D7F8A4014568B4F891
:2046B000BC0030214FF47F42082300903046A847D7F8A4014568B4F8C00004214FF4F802CA
:2046D000122300903046A847D7F8A401B4F8D070456820214FF440620A2330460097A84744
:2046F000012584F8D8501AE151F8318C12F0EEFE2F4600B901273946904F38680028FCD0A9
:20471000B146012609F10409D9F82CA03E6009B112F0E2FECAF30720C4F8BC0012F0D6FE5B
:20473000AA4600B9B2463B68002BFCD0D9F800B0BAF1000F3E6001D012F0CEFECBF3844034
:20475000C4F8C00012F0C2FEAA4600B9B2463B68002BFCD0D9F81C90BAF1000F3E6001D02A
:2047700012F0BAFEC9F38120C4F8D000B8F5C061C4F8B81000F09C8094F8D80068B9C4F8E7
:20479000D410D4F8C000C4F8C800D4F8BC70C4F8C470D4F8D030C4F8CC30D4F8D410D4F82D
:2047B000BC30002954BF02206FF0010004F1C802176801EB41014018411000EB917107EB4B
:2047D000A1001060D4F8C810C4F8C43000291CDD1E293CDDD4F8CC0030B93429B4BF153943
:2047F0001E21C4F8C81025E02A29BABFD4F8C8000B381E20C4F8C800D4F8C4003F28B4BF02
:20481000401C3F20C4F8C4001FE0D4F8CC00032812D011F10B0FC6BFD4F8C8000B30301CED
:20483000C4F8C800D4F8C4000028C4BF401E051CC4F8C450032508E011F1150FC6BFD4F8D3
:20485000C8001530301CC4F8C800C4F8CC504FF08057D7F8A401B4F8C43030214FF47F4214
:204870004568354800930823A847D7F8A40104214FF40032112345682F480096A847B4F8BA
:20489000C860D7F8A40104214FF4F8021223456829480096A847D7F8A40120214FF4406298
:2048B0000A23B4F8CC60456823480096A84701E084F8D85040F2FF50404502D8801C4045C0
:2048D0002DD208202EE051F8311C1D4F4BF2F5204843060A3868C0F3814001280AD111F08B
:2048F00061FA10F06DF812F0FDFD3111C010484306EBE03694F8E50030B91248006820F01C
:204910007F408019460801E084F8E5500E48310C0660012741600D4D8760287808B90B20C0
:2049300000E0052084F8E40004F090F9BDE8F88F39400C40940F002000A00C4000800C4019
:20495000B43F0050102009403C600C408E8A01002DE9F04FAF4E82463068ADF1140D08B958
:2049700012F0A2FCAC490120AC4F08703978012902D0002103F0BEF830680489456812F0B3
:20499000B6FEDFF89C922888000937D399F83800002833D031684A6A4F6E906AC846B0F1E4
:2049B000FF3F25D027B3431C93628862030E07F80139306890F82A0007F80109306890F8DF
:2049D000290007F80109306890F8280038703268106A00940190401B201A80B20290916A18
:2049F000506A92F888202B46153006F0A7FE00E0DB20D8F87C10002840F000812146284685
:204A10000BF03AFE642003A90FF0E6F9854999F838700878884637B98348007809F0C0FF05
:204A3000012805D0E6E009F0BBFF012840F0E280DFF8F8C1A01C241D6D1EA1B2ACF87800AD
:204A5000C1F3022040F0080005F8010929709DF80C70CCF88450002F4FF00005ACF86A501E
:204A70000CBF49F24E0047F60E206446C4F8C0006F4EC4F8800070688047B3466D4E049061
:204A9000BAF1010F6BD0BAF1040F68D0BAF1000F65D094F84000BAF1050F04F13007C0F3C1
:204AB000C0003ED0E8200DF10D010FF095F999F8380030B39DF80D00032822D1787B3B7C61
:204AD00000F0F00007F1110140F00300787343F018003874F4200FF07FF9D9F89C00804708
:204AF000A064306A544BD0F808C06586294602208DE80300D8F80C002A463946E047374676
:204B100067E0306A87684C4BA4F86A50294602208DE80300D8F80C002A4604F16801B84716
:204B3000EDE728B9787B00F0F00040F0010004E0787B00F0F00040F003007873B146294671
:204B5000D9F820003E4B8668658602208DE80300D8F80C002A463946B0474E46CFE794F8C0
:204B70003D0000F0F00040F0030084F83D0094F8400004F130018A46113140F0180084F854
:204B90004000F4200FF028F999F83800002808BF4FF4FA5002D0D9F89C0080472949A064D0
:204BB0003746D8F80C000B783E6A43B9A4F84E5002212A468DE8060004F14C0105E065860B
:204BD00002212A468DE8060051462A461A4BB568A8471A490880DBF80810002808D41A4A01
:204BF00092F900006834401C10700498FC600DE0049888471A200BF077FC08E0002908BFD2
:204C1000E420F8D0114A00201070E420884705B0BDE8F08F640E0020CB1A0020E41A00205C
:204C3000EC130020841900204F120020280D00208C14002028160020399D000094180020F2
:204C500091C90000C6180020CD1A0020203200202DE9F04F002898461546ADF12C0D00F0F6
:204C7000F58011F47C1F40F0EE8011F00F0F00F0ED8007460591002006900A904FF0000A79
:204C90000990544608944FF0010BCDF810B0044650460790059805990BEA000021EA0B01A7
:204CB0004FEA4B0B401E059100F0AD80401E69D0801E56D0001F40F0C08005B12F660720E8
:204CD000152642F2D002022307F8010B01A907F8016BA2F1CF0007F8013B0EF04BFE6846AC
:204CF00003A90AF04FFB8B48019A018842F2D0064FF47A63701890FBF3F0009B3E46C018A6
:204D10000090824206D8801ABDF80C300090581CADF80C00009B5008514681460904180497
:204D3000030C19430004534610EB090041EB0A0102F02CFA0090BDF80C309DF80C009DF851
:204D500000209DF8011006F8010B181206F8010B9DF8023006F8012B9DF803200934BF1D7D
:204D70004BE00220152607F8010B042307F8016BB8F1000F07F8013B0CBF099898F800000F
:204D9000241D57E01DB1EF6595F86B0006900520152642F2D002049B07F8010B0DF10E01BE
:204DB00007F8016BA2F1CC0007F8013B0EF0E2FD02A80FF06FFD5848029AB0F8B61042F20E
:204DD000D00670189DF80E604FF47A6390FBF3F150189DF80E30069AE41D000200EB6600A4
:204DF000B0FBF3F03E4602903F1D06F8012B9DF808109DF809309DF80A2006F8011B06F827
:204E1000013B327018E00320152607F8010BB8F1000F07F8016B034607F8013B04BF0A9837
:204E300007F8010B05D098F8000007F8010B98F80100641D07F8010BA4B2059800287FF43C
:204E500029AF264661E011F00F0F01D000205DE080468A4602264FF4803908F1020509EAC3
:204E70000A002AEA090A4FEA4909B0F580301AD0B0F5803014D0B0F500300ED0B0F58020F6
:204E900009D0B0F5002004D0B0F580102AD1072404E0062402E0052400E00424002704E009
:204EB0000224012701E001242746A81C214600F047FC47B104F00F04C0F30A0141EAC421F6
:204ED00041F4004105E004F07F0400F0FF0141EA042105F8011B36180912B61C2970B6B25B
:204EF00045196D1CBAF1000FB9D1022ED8BF00260BDDB01E4FF6FE7708F8010BB819C0F38A
:204F1000022040F0A00088F8000030460BB0BDE8F08FC0469E2E0020E82D00202DE9F04F3E
:204F3000AC4C04F128000068ADF1240D0FF0D4FA08B111F06BFCA248DFF89CA2DFF888B217
:204F50000068A24E089011F031F811F059FAE569A769B5F57A7F13D0C01B4FF47A720023C2
:204F7000A5FB000102F012F980464FF47A72002311F0D8FF2A46002302F008F9C01901E053
:204F9000A0EB0708A0618D488C49006820F00200086070688047DBF80010DBF804304546C6
:204FB0006918B1F57A7F0DD34FF47A72B1FBF2F2D2184FF47A73CBF804201F46B1FBF7F227
:204FD0005A43891ACBF80010B168884770688047DAF8041002466818B168CAF80400104644
:204FF0008847DAF8000000285FD007464FF00009706880474FF000081FFAA5F3079083B9AA
:205010005FFA95F36BB93979E8B2884204DD79682846884209D20AE03879E9B2401A387157
:2050300008E079682846884201D3414601E07968091A7960B88878B9FB8853B9FB6843B1EF
:205050003B8933B1B87A19460AF0FAF8F8687860B88808B9FB880BB13B896BB9B9F1000F02
:2050700004BF3868CAF8000003D03868C9F800003868B846074601E0B9463F68B16807989D
:205090008847B8F1000F0ED0B8F8043043B9B8F806302BB998F80A00B8F808100AF0D0F8CD
:2050B000404611F07DF9002FA2D144484349006840F002000860E06828B3804723E015F82D
:2050D000060C2169A5F10C07032819D0E16A9DF816000978884210D115F8080C10F09CFB8D
:2050F000B979012903D0022908BFA87000E02870002029460DF0B4FB05E011F087FB02E06A
:2051100009B12846884708200727ADF81000716AADF8127004A88847069D0028CFD0294825
:2051300000680088C8B1706880472649096800220D880A80B1688847089A0020294620708D
:2051500090470546FF202070706880471D4909680A8815430D80B168884710F027FF074626
:20517000B7F1FF3F1CD0706807B9194F216AB94238BF0F1C80471C230546626AADF80230B1
:205190000820ADF80000716A019268468847A16A3846491CA1620FF0D7FBB168284688472F
:2051B00008200A27ADF808004FF0FF35ADF80A70716A039502A88847C5E6C04610E000E0DA
:2051D0000C8B0100242D0020501A00208C1400208EC2F52864180020FC3100202DE9F04FC1
:2051F0008146002000212022ADF1540D009003A80BF0C3FDD9F82400B9F8221001236A46B4
:2052100007F08EFD0024A046002876D10098002873D006467079042869D100200190F188BB
:20523000B06801AA002307F07BFD00285FD1019800285CD007467879BD68001F3AD0401EDA
:2052500004D0401E2FD0401E10D04AE0F888202847DC03A8002120220BF08FFDFA8803A8F8
:2052700029460AF01DFA44F002043AE00BA86B682968436005F1080201600DAB1168506846
:20529000196002F10805586029686B680FAA083553602846116011AB026841681A6044F064
:2052B000080459601DE029880DF10A0044F00404018016E0298802A80180BDF8081042F2D3
:2052D0000E0012F071F815F8028F44F0010408F00100C8F3800BC8F3401A1390C8F3400379
:2052F00014933F68002FA6D1019811F08EFE3668002E8FD1009811F088FE99F82870634D60
:20531000022F18D0A008C0F0BC805F4903A8202210F0BAFF002840F0B480012F04D1E87891
:20533000401CE87099F82870032F04D12879401C287199F82870002F4DD1A86A401CA862F5
:20535000600820D3B8F1000F04D105F13E00494612F058F942F20F00414612F02CF81399A3
:2053700042F20A0012F027F8149942F2100012F022F842F21100594612F01DF842F2120070
:20539000514612F018F84FF40050494612F0BBF9B9F81A10502011F045FCB9F81A00B9F873
:2053B0000010D9F82C304A460DF016FBB9F81A004946288705F13E0012F024F9687801289D
:2053D0005AD0002001210CF075F941F2707003210CF070F950E0022F4ED1E00805D3BDF856
:2053F0000A1042F2140011F0DFFF200913D342F215000BA912F087F942F216000DA912F0CC
:2054100082F942F217000FA912F07DF942F2180011A912F078F9286B4946401C28634FF4C1
:20543000005012F070F9002003210CF043F96878012821D0012000276870154C6F7104F1D5
:20545000E000064611F060FF012802D1304612F070F911F0E5FD074611F0E2FD42F210710E
:2054700000EB07200DF02CFA206A01F57A6112F0EDF8304612F05BF9D5F8981009B148461C
:20549000884715B0BDE8F08F8586010048130020A41000202DE9F04706460020ADF1380D4D
:2054B000DFF89092ADF80C00A0480F460168A34D097D252900F00E81006805A96C3006F0A1
:2054D00087FE002818BFC0B240F02D8197480068C18AC9080DD3007D03280AD09DF81F006F
:2054F00038B99DF820004C463870B5342070002019E101A804A909F045FFA5F12F018A4600
:2055100091F82F30019A3468DAF808104FF47A78404641F208155843891A08FB120008FB11
:2055300001F1001B091B8D42C8BF002965DC854205DD002803DD346804F5915434609DF816
:205550001F00002857D042F204000DF135010EF011FA10F0A5FF044606980DA9241A42F2A4
:2055700006000EF007FA9DF834109DF81D00FF2904BF0A218DF83410FF2808BF0A209DF8FF
:2055900034206B499DF81C30B4FBF1F1801880B24843991008FB01F1814298BF081C2D180B
:2055B00005A810F02AFD9DF81C203468C446B0FBF2F15143411A8BB20CFB02F26146594398
:2055D000531A521A1B1B121B954201D9002A08D56942994216D2002B14D5B5FBFCF109B2ED
:2055F00003E06900B1FBFCF189B232684FF4916303FB012405E0002004E0306841F630346B
:205610002418346005460DF1120102A809F0BAFE0298DAF80810B4FBF8F210180290814259
:2056300003D99AF82F30834204D94B4603F15804267836BB9DF81C0055190004A84298BF17
:205650002D1A9DF81F00002808BF9DF8200016D09DF81C00B5FBF0F084B29DF833000EF078
:2056700073FB9DF83120014620460EF0B1FC044610F0B0FC024608A920460EF0F7FA4C4698
:205690000DE0814204D8BDF81200401CADF812004C46BDF8120094F85B100CF066F9387041
:2056B000224E84F8B5003068007D05287FF41FAF2148007800287FF41AAF387803A9ADF870
:2056D0000C0042F20C0004F091FCBDF80C00A4F8B0000CE768460DF10E0109F053FE306850
:2056F000009A2B7841F208144FF47A7101FB0202009259438A1A944210DCA1F5FA61914288
:20571000BCBF00F5FA6030604C4694F85B10208F0CF02BF901460020397002E039784C4692
:20573000652084F8B5100EB0BDE8F087640E0020A0860100E82D0020351200205F2F0020B6
:20575000F0B504460846ADF16C0D401E6BD0401E0DD0801E00F00381401E00F0E980401EEA
:2057700000F0DB80401E00F0A88000203CE142F2010007A90EF0FEF842F20B0008A90EF054
:20579000F9F842F206000DF165010EF0F3F842F207000DF166010EF0EDF842F2050019A903
:2057B0000EF0E8F804A809F0A7FC05460DF1670142F209000EF0DEF89DF86700002808BF06
:2057D000002303D0022010F0FDF8034607A8006808A920600988271D3C46B81C218005F05A
:2057F00007079DF865609DF864109DF8662000F8011B9DF8674000F8016B03F0030600F865
:20581000012B620747EA926104AC41EA8611012700F8011B9DF8672000942946019706F064
:205830004FFE0A3099E042F206000DF165010EF0A1F842F207000DF166010EF09BF842F2BE
:20585000040019A90EF096F804A809F055FC05460DF1670142F208000EF08CF89DF8670085
:20587000002808BF002303D0012010F0ABF803469DF864009DF8657004F8010B9DF8666060
:2058900004F8017B9DF867209DF86770790704F8016B03F0030705F0070646EA916004AE3E
:2058B00040EA8710294604F8010B002700962046019706F005FE001D4FE042F2150011A99D
:2058D0000EF058F813AD42F2160029460EF052F815AE42F2170031460EF04CF817AF42F2E8
:2058F000180039460EF046F811A801682160406860606A6804F108035A602868186030688E
:2059100003F10801086074684C60386801F1080528607A686A60202066E042F214000DF1EB
:2059300022010EF027F8BDF8221002200A1258E009A8002120220BF020FA42F2130009A998
:205950000EF018F809A811F015FC024609A9204609F0A6FE09A811F00DFC80B244E042F224
:205970000E0002A90EF006F80DF10A0142F20F000EF000F80DF10B0142F20A000DF0FAFFE2
:2059900003A942F210000DF0F5FF0DF10D0142F211000DF0EFFF0DF10E0142F212000DF08A
:2059B000E9FFBDF808009DF80B209DF80C709DF80D609DF80E509DF80A1004F8010B02F0C3
:2059D0000102001204F8010B07F0010042EA400206F0010042EA800205F0070042EA401215
:2059F000042004F8011B22701BB0F0BD2DE9F04F06469E48001D0068ADF1340D80470B9004
:205A10000AA9822004F0A0FB9DF8280018BB00248DF828404FF6FF75ADF804509DF8280082
:205A3000ADF80650FF2108228DF8000002A811F08AFE8DF81840D420694601F06FFF9DF8E5
:205A50002800401CC0B28DF828003228E4DB82200AA901F063FF0020DFF808A2DFF80882D0
:205A70008DF8280081469DF828008DF8019069468DF80000D02004F067FB01274D46E8B9F9
:205A90009DF80B30012B07D19DF80A0020B90DF1020011F00BFA88B9747B002C0CBF052256
:205AB00009224F469C4209D10DF1020006F10E0110F0A6FD002818BF012507D1002F40F059
:205AD000BF801DB9707F002800F0BA804C469DF828008DF8214008A98DF82000D12004F0F0
:205AF00033FB002832D19DF82200FF282ED08DF800006946D42004F027FB002833D102A84D
:205B1000311D082210F07CFD00B330887788ADF80400ADF8067045B1307B9DF82810B769C8
:205B30008DF818000DEB81010F61D420694601F0F5FE75B1307F9DF82310884209D08DF882
:205B5000230008A9D12001F0E9FE02E0641C322CBDDB322C74D14F468DF80070D420694670
:205B700004F0F2FA28B1DAF808100B988847192074E002AB184611F099F94C4600B101246D
:205B90002046341D30B918462146082210F038FD00284AD030887388327BADF804009DF851
:205BB0002810ADF80630002D8DF818200DEB810000F110000CBF4946B1690822016002A8B5
:205BD000214611F08BF998F8380030B1D8F888201AB19DF80010204690474C469DF82800AC
:205BF0008DF8214008A98DF82000D12004F0ACFAE82807D09DF82200FF2803D0641C322C58
:205C1000ECDB10E09DF800008DF82490337F8DF8220069468DF82330D42001F07FFE08A9FC
:205C3000D12001F07BFE322C02DB7F1C322F93DB322F05D1DAF808100B9888471A200DE09A
:205C50009DF82800401CC0B202288DF82800FFF60AAFDAF808100B98884748460DB0BDE8D8
:205C7000F08FC0468C140020EC1300208C1400202DE9FF47854FDFF830828C4CF8680028D7
:205C90003ED18F4D8249843D2868814210D0814981420DD0804981420AD08049814207D017
:205CB0007F49814204D07F49814201D011F0FCFA10F0D6FD29684FF0FF32012805D1C1F39B
:205CD0000330083805D0C01F01D0012A01D1012000E00020F8700EF03FFC142804D1404666
:205CF00000F1E001C0F8A4100FF08AFF216A19B911F0DAFA2046016A096A07F11000884781
:205D1000632002A90EF068F8DFF8A49109F1B70000780FF05FFF06464046D0F8981090F88B
:205D30009D20B0F896C041F00F0102F03F02C0F898102CF0070C80F89D204CF0010CA0F87F
:205D500096C0B37A4FF0000A00F188057BB99DF8083002F0C0023F3303F03F0313436B7557
:205D7000EB8A4FF6C0721A4042F018020DE09DF8083002F0C00203F03F0313436B75EB8A33
:205D90004FF6E0721A4042F02002EA82307B052814BF2420292088F89C00F27A307B401D7A
:205DB0005043E2690A230CF0010C90FBF3F0C0044CEA1040E881F07A1923800390FBF3F007
:205DD00060F31C212961288B117D4FF6F77361F3020003EA00012883107D00F008000843EA
:205DF000288399F9A6000DF05DFEA8F8A200716833683089401EA8F88AA0414303EB5100FE
:205E10004FF47A71B0FBF1F0A8F8A800C8F88CA0687B00F0F00040F00100687311F098FB21
:205E3000A0B9F07A234A99F8B730B1FBF0F01070F07A022BB1FBF0F0C0B2B1FBF0F0787095
:205E500004D11D4802214170A8260670F86850B9206A0668616A194807F110032A46B047E1
:205E70003C4605460DE050460BF028F9206A86684FF002098DE80006F868524629461346A9
:205E9000B047E5600090BDE8FF87C0468419002000F0022000F0012000F000200080022063
:205EB0000080012000800020280D002028160020A8110020C8190020C4180020282D002093
:205ED00018130050F0B500214422ADF1540D02A80AF053FFF22013A911F0CEF9834DBDF8FB
:205EF0004C0013A9A5F86800F32011F0C5F9BDF84C000DF10901A5F86A00E22011F0ACF9FB
:205F1000688CADF81200410806D305F10C01096805A80160BDF81200810805D3291D098823
:205F300006A80180BDF81200C10807D305F1100109680DF11A000160BDF81200010908D31B
:205F50000DF11E0005F14C01242209F0A9FBBDF81200400903D3A86A12906F6A1197644828
:205F7000007800280CBF0121002101200BF026FFBDF8120041082CBF0F240B24810824BF59
:205F9000A41CA4B2C10824BF241DA4B2010924BF2434A4B2400924BF0834A4B220460FF0DA
:205FB000D9FE071C00F09F8005260DF1090100F8016B0A68026049684160BDF812100830FC
:205FD00011F0AEFABDF81210844648080BD3BDF81410604611F0A4FABDF8161011F0A0FAA5
:205FF000BDF812108446880807D3BDF81810604611F096FABDF812108446C8080BD3BDF86E
:206010001A10604611F08CFABDF81C1011F088FA8446BDF81210374A9388080949D3BDF896
:206030001E10604611F07CFABDF8201011F078FABDF8221011F074FABDF8241011F070FA03
:20605000BDF8261011F06CFABDF8281011F068FABDF82A1011F064FABDF82C1011F060FAF4
:20607000BDF82E1011F05CFABDF8301011F058FABDF8321011F054FABDF8341011F050FAF4
:20609000BDF8361011F04CFABDF8381011F048FABDF83A1011F044FABDF83C1011F040FAF4
:2060B000194611F03DFA117811F03AFABDF812108446480906D3119960460EF0CAFD1299F0
:2060D0000EF0C7FD05F11401224630463B4605F0F1F80820ADF80260074D01972968ADF855
:2060F00000006846884715B0F0BDC04690120020AA170020A4100020B01400202DE9F04FEB
:206110000128ADF1140D40F0F180DFF81882D8F8DC00012840F0E7800220C8F8DC0011F04A
:20613000EDFB029001200EF011F9061C06D00120C8F8DC00029811F0DDFBD9E011F0D6FBF9
:2061500003906D484FF00009C0F8009001200FF0BDFC012818BFCDF8009004D148460DF0C9
:2061700063F8012000906548654FC0F800903868112011F0C9F900280CBF4F4601271020E6
:2061900011F0C2F908B147F002070F2011F0BCF908B147F004070B2011F0B6F928B1594805
:2061B0000068594D016B288888470A2011F0ACF94D4600B101254FF0805B28460BF5DC75C3
:2061D00020B12868514C016B208888475048012404602868816947F0200088474D48046014
:2061F00011F08CF900F001010191400814D24A4811F019F98246BAF1040FF8D0BAF1010FA9
:2062100005D1DBF8D80142684348032190474349086820F003000860484600F085F83848CA
:206230002B680068986B8047019801280DD0BAF1010F05D1DBF8D801426837482146904746
:206250003649086840F0030008602C48046028684169384688470B2011F056F920B1286869
:20627000294BC16A188888470A2011F04DF920B12868264BC16A188888472548046003222D
:20629000C8F8DC20234BC3F800902868416B384688470128F9D104200EF058F80546184FD9
:2062B00015481F490460386808688009FCD30098012802D120460CF0B7FF11F00DF9082062
:2062D0000EF044F807460398C8F8DC4011F00AFB0CF0B0FB029811F00DFB57EA050018BF43
:2062F0004FF0FF3604E06FF0040601E06FF00106304605B0BDE8F08F0C400940000222433B
:206310002C200940B8010010428801003E88010028200860800104430040034024220840F4
:2063300014100940940F00202DE9F047DFF80CA20746AAF13500DFF8F8810068800880F07E
:20635000E7800FF02FFD814908310B6800261C17641C990D0AD2C0F13E0110F10A0F4FEA87
:20637000E101D8BF08218C42B8BF0C1CDFF8C4C1990E0FD2590E0DD36246143A1168C1F3B0
:2063900004211629A8BF20391268C2F30462162A0EDB0CE0634AD2F87C11C1F304611629C3
:2063B000A8BF20391268C2F30442162A00DB203A61189146162905DA11F10A0FB8BF6FF0C4
:2063D000090100E01521584C584D01F01F0242F4F85222802A6812F0030F18BF0126D20892
:2063F00028BF46F002060FB146F00406424692F90740041B052C04DA9479B44208BF9188FD
:2064100066D00F28A0F10F0827DB08EB0014A4F1F0084FEA282EBEF1070F88BF4FF0070ED2
:206430007546062D88BF06255CF82570042404EB850465462C59E41B04F0FF05F70824BF5A
:20645000C4F307273D44B70824BFC4F307473D44770828BF05EB146501E00025AE465CF881
:206470002EC0F7080CF0FF0424BFCCF307273C44B70824BFCCF307473C44770828BF04EB4C
:206490001C64ADB2A8EB0E27B9EB010105FB07F505F1800504EB1524D8BF012103F0FF0352
:2064B00034254D43A9B259434FF6FF73B1FBF4F18B4238BF191C802889B2918005DA10F1D7
:2064D000800FB8BF6FF07F0000E07F20D0719671194800681F2910604FF0000008D340F234
:2064F000FF128A4206D24908401C8A42FBD301E01F219180124F0F39090940EAC10047EA87
:206510000001CAF8FB1F0026CAF8FF6FBDE8F0870C490D4F424608200F60921D1070BDE878
:20653000F087C0463C1100506E620840242208400C3200209C13005008200940350009403F
:2065500000E7A48030100940FDFDA400AC3F00502DE9FE4F0646824AF07B20B91146491C43
:206570000978022908DB012803D110460078022802DBF120BDE8FE8F346AB6F8289096F8D5
:20659000347096F835B0B58B4FF000085FEA040A17D0744890F83830002B2ED0016D0029A3
:2065B0002BD004F0FF0088476E49096D04B20AF47F008847001900B2001D00B2C43084B21B
:2065D00000E0C4240DB12D1DADB267480078012809D147B16548C11991F8048010F80B00B3
:2065F0002418641DA4B205EB090020184044801C80B20FF037FE071C02D11A20BDE8FE8F5F
:2066100008EB09002B193881002D07EB030078600EBF0020E019801C00217422C7F8A000DF
:2066300007F10C0011F08FF84C442D1907F13C00FF211022A7F84C5011F085F807F12C0085
:206650000F21102211F07FF800243C707C707868716A328D09F024F807F1800006F12C0169
:206670000B2209F01DF807F18C00314610F0A6FA7089A7F89600307B87F89800707B06F162
:206690000E0587F899002A6869460A60AB888B80AA798A719DF800102046012908BF01209B
:2066B0009DF80110012908BF40F004009DF80210012908BF40F008009DF80310012908BF96
:2066D00040F010009DF80410012908BF40F020009DF80510012908BF40F040009DF80610CA
:2066F000012908BF40F08000A7F89A00707D87F89C00B07D87F89D00B28BA7F8A42022B1EC
:20671000D7F8A000B16908F0CBFFB07F87F8A600306AC7F8A800B7F8A400C0B1D7F8A00096
:20673000A8B17868401E7860F82101707868401E78600470B7F8A410B7F8A4607868401A76
:20675000786039897018801C38817868B8650848007839460CF084F82046BDE8FE8FC04658
:20677000920E0020EC13002044120020A08A0100141500202DE9F043002B08BF002A10D1FA
:206790000029BCBF00204FF0004106DB50EA01071CBF6FF000006FF000410AF0BAFDBDE852
:2067B000F0835FEA530898EA610803D50026404266EB01015FF0000913F0004E03D0002652
:2067D000524266EB03031C461546002C08BF8D429CBF2C1C0025070C47EA01470E0CB442DB
:2067F00008BFBD429EBF240444EA15442D04070A47EA01670E0AB44208BFBD429EBF240285
:2068100044EA15642D02470847EAC1774E08B44208BFBD4200F29280870847EA81778E0876
:20683000B44208BFBD427BD8C70847EA4177CE08B44208BFBD4265D8070947EA01770E09E2
:20685000B44208BFBD424FD8470947EAC1674E09B44208BFBD4239D8870947EA81678E0938
:20687000B44208BFBD4223D8C70947EA4167CE09B44208BFBD420DD8E60146EA5566EF016E
:20689000B14208BFB84201D3C01BB14159EB09094EEB0E0EA60146EA9566AF01B14208BFAC
:2068B000B84201D3C01BB14159EB09094EEB0E0E660146EAD5666F01B14208BFB84201D3B8
:2068D000C01BB14159EB09094EEB0E0E260146EA15762F01B14208BFB84201D3C01BB141C9
:2068F00059EB09094EEB0E0EE60046EA5576EF00B14208BFB84201D3C01BB14159EB090962
:206910004EEB0E0EA60046EA9576AF00B14208BFB84201D3C01BB14159EB09094EEB0E0E82
:20693000660046EAD5766F00B14208BFB84201D3C01BB14159EB09094EEB0E0EA14208BF4D
:20695000A84201D3401BA14159EB09094EEB0E0EA34208BFAA423EBF2D0A45EA0465240AEF
:206970008AD373464A465FEA080803D50026404266EB01015FEA480803D50026524266EBB9
:2069900003031E4617460B46024631463846BDE8F0832DE9F043044694F830900F46984668
:2069B00015468B20ADF1340D0DF10A0103F0CCFB8A20694603F0C8FB94F8250000283ED128
:2069D000B9F1000F19D1BDF80A104FF6FE70884205DCBDF80A1088422FD1694615E0B4F8EE
:2069F00044009DF80A608DF80C0000128DF80D00BDF80A008DF80E601BE0B9F1020F09D0CE
:206A1000B9F1030F19D104F1280103A810F075FE092612E0207CC00934BFB4F84200B4F871
:206A300044008DF80C0000128DF80D00208D8DF80E00001205268DF80F00002013E002287F
:206A50000CBF05260926012818BF04F11C0104D1892006A903F078FB06A9324603A810F08A
:206A70003DFA94F8260006EB0D01C8723A4603A831460AF013FC002840F08E80B9F1000F1A
:206A900019D1BDF80A104FF6FE70884205DCBDF80A1088422FD1694615E0B4F844009DF80D
:206AB0000A608DF8200000128DF82100BDF80A008DF822601BE0B9F1020F09D0B9F1030FEE
:206AD00019D104F1280108A810F017FE082012E0207CC00934BFB4F84200B4F844008DF804
:206AF000200000128DF82100208D8DF8220000128DF8230004203E6881460BA9822003F0C6
:206B100023FB9DF82C10307B8142D8BF9DF82C00002841D007460024722029460FF02EF9DF
:206B3000B0689DF82C102018C8F80000007881422EDD2B68C10001EB0011D8F80000C9181C
:206B500029604278012A1FD0807828BBB9F1040F06D0091D08A80FF0EFFF012816D017E091
:206B700008884B888DF82800042208A98DF82A3000128DF8290018128DF82B000AA80FF0F4
:206B90003FFD012802D003E0807828B9002004E07F1E04F10304BFD1F3200DB0BDE8F083DD
:206BB0002DE9F047064637680C465FEA0208ADF1180D14BF00214FF0FF3107F148008146BB
:206BD00010F08CFE002808BF0B2000F0DF80002565707148FC60B8F1010F057004D06570CC
:206BF0000220FC600EF070FD2078012840F29080801E012857D9801E01282CD9801E01280F
:206C100000F2B88010F082FE8246A078009021782846062908BF0120019001200290A068E0
:206C3000228A6368E16806F061FE0746504610F069FE002F40F0A080B8F1000F02D010F0DC
:206C5000B1F802E030460FF0EBF9002800F0878010F069FD21E010F059FE012782460097DC
:206C7000A168A278606824782B46042C08BF3B1C08F094FA0746504610F044FE002F7BD198
:206C9000B8F1000F02D010F08DF802E030460FF0C7F9002863D00EF09FFC3E49C1F8B05189
:206CB0000D60074668E010F031FE8246E08A0090E0680190208B0290A0780390207D0490DF
:206CD0000121059122782846022A08BF081CA368E178626802F0F2FD0746504610F012FECB
:206CF000002F49D1B8F1000F02D010F05BF802E030460FF095F9002831D00EF09DFC071C96
:206D10003AD1E078A168E28A236909F0FDFEC8E710F0FCFD8246E08A0090E0680190208B1D
:206D30000290A0780390207D049001200590277807B90546E1786268A368284602F07CFE6D
:206D50000746504610F0DEFDB7B9B8F1000F02D010F028F802E030460FF062F908B91420A4
:206D700014E00EF051FC071C06D1E07821690CF04BFC96E74FF0FF37B8F1010F02D0022006
:206D90000EF08AFC484610F0A5FD384606B0BDE8F087C046504502401A3200202DE9FE4F33
:206DB000794C074694F83D00002800F0DA80DFF8DC81B7F84210B8F88A00884240F0D180BC
:206DD00007F128000FF08EF8002800F0CA80002598F88D0084F83D5010B102200FF0F0FB84
:206DF0006148007810B101200FF0EAFB387C400905D310200FF0E4FB802010F0A5FA20203A
:206E10000DF056FE594E06F120000CF03DFD7A6851781078334600EB0120C0F30321C0F3DB
:206E3000003684F8391000F00F0184F83A60C0F3031684F83E1098F8B30088F890600F28B1
:206E500004D0884202DDD67806B9014688F8711098F871A083F84050BAF10F0F09D194F875
:206E70003B0002287DD10EF041FA07F071FBBDE8FE8F3F480078012803D00120294600F006
:206E900039FE43484068804700900FF0D9F93948DFF80091DFF8E0B0066898F8712099F8E0
:206EB0000030D9F80400311A980091FBF0F05BF822100DF091FCC9F804605BF82A0001912B
:206ED0002E4EB060F0600CF05FFE019831680EF027FA09F081FA2E4900988968884794F84D
:206EF0003B0002280DD127480CF0CEFC98F8712034F812004FF470719140091A21480FF02B
:206F10002DF898F89030388929460FF028FA20630F2B14D098F8711094F83900994208D071
:206F3000401C6FF00F0598408101A1EB80016D1805E0401C98408501A5EB8005A03D65632D
:206F5000022004F1200584F8380028460CF09CFC0B48A062616B28460FF000F8102010F079
:206F7000F3F9BDE8FE8FC046773000201C310020E41A002060160020E8880100241A002026
:206F9000910701002C310020EC170020A81100208C140020C81900202DE9F04F7A4C80462D
:206FB00008460026ADF1440D0028089004F105010E701ABF006800684FF0FF30B8F11D0F39
:206FD0000C900CBF1E201D20099009F0DBFD24224046314610F090F915250D9605210E96E2
:206FF00020460F96C0880A9104460B94A1427EDA65484779002F6AD1641F404602AAA4B28D
:2070100021460AF079FCBDF814709DF81130781D1FFA80FAD80951D233F07F035AD0029AE4
:207030000C98904256D0099829460AF095FA002850DC8EB9611E40463A4689B20FF080FA37
:2070500050B90299E01B80B2B1F5805F0B9041D10F904FF0040906E0A9460AEB0500B9F1B9
:20707000000F85B236D007EB09001FFA80FB2146052206AB40460FF094FD099806AA5946E0
:207090000CF0ECFF26B90E98401C80B20E9006E0E01B81B209984A4653460CF0DDFA0D98F2
:2070B0009DF818205946401C22F0400280B20D9009988DF8182010F01FF90BE098080CD2F6
:2070D000544507DA3049052048710F4638714FF0FF3056E0E41BA4B204E0404621460DF00A
:2070F00025F804460A98A04282DB2748C0880B99761C0446022E0A91FFF678AF0C98B0F1D5
:20711000FF3F14D020480899C58008890090C86801908A88CB880868099904F055FF1A48EC
:207130000D9E0746C588FC80701C80B20D900F98C0B101460C2202AB40460FF032FD0D9F89
:2071500002980E9EC5F5805404210C22ADF80E4002ABADF81070401C02900998ADF812608D
:207170000AF034FA09980CF051FC074840790028ADD10548C580404609F004FDC5F580579C
:2071900038B211B0BDE8F08F441A00202DE9F0411C4615468C4208BF854282BF00230022AC
:2071B000E5E0002C08BF002D0AD100290EBF00286FF000006FF0000100F0E1F8BDE8F08143
:2071D0005FF000085FF0000E002C08BF8D429CBF2C1C0025070C47EA01470E0CB44208BFFE
:2071F000BD429EBF5FEA044444EA15445FEA0545070A47EA01670E0AB44208BFBD429EBF9D
:207210005FEA042444EA15645FEA0525470847EAC1774E08B44208BFBD4200F29380870875
:2072300047EA81778E08B44208BFBD427CD8C70847EA4177CE08B44208BFBD4266D80709D7
:2072500047EA01770E09B44208BFBD4250D8470947EAC1674E09B44208BFBD423AD887091C
:2072700047EA81678E09B44208BFBD4224D8C70947EA4167CE09B44208BFBD420DD8E6018E
:2072900046EA5566EF01B14208BFB84201D3C01BB14158EB08085EEB0E0EA60146EA956624
:2072B0004FEA8517B14208BFB84201D3C01BB14158EB08084EEB0E0E660146EAD5666F01AA
:2072D000B14208BFB84201D3C01BB14158EB08084EEB0E0E260146EA15762F01B14208BFD5
:2072F000B84201D3C01BB14158EB08085EEB0E0EE60046EA5576EF00B14208BFB84201D3D3
:20731000C01BB14158EB08084EEB0E0EA60046EA9576AF00B14208BFB84201D3C01BB14103
:2073300058EB08084EEB0E0E660046EAD5766F00B14208BFB84201D3C01BB14158EB08089D
:207350005EEB0E0EA14208BFA84201D3401BA14158EB08085EEB0E0EA34208BFAA423EBFC6
:207370002D0A45EA0465240A89D3734642461E4617460B46024631463846BDE8F081704747
:207390002DE9F04306467078ADF1140D002840F0D78096F8961002291CBF0329E82096F8F6
:2073B0008B108029C8BFE82096F88C10092901DB0A2900DDE82096F88D10002900F0BF8017
:2073D000042980F2BC80002840F0BA80614C04F1B7000078884204D006F18D01E82001F043
:2073F0005FFF06F18C01E72001F05AFF06F18B01E12001F055FF06F19801502001F050FF41
:2074100096F8960002280CD04FF6FE70A4F8840006F18E0104F17A0010F06FF906F18E0578
:2074300004E006F18E052888A4F884004A4806F180010B220FF052FD4FF001080220A6F871
:2074500016802946307501A80FF0B8FB96F89A70B6F89890706806F19A01002FA0F101007E
:2074700070600CBF002040464F780FB140F002008F780FB140F00400CF780FB140F00800C8
:207490000F790FB140F040004F790FB140F0800071684A1E7260314B0870377D7168002533
:2074B000481C3062781E087030893565801C30811878B565A0B30427F08A86F8695006F148
:2074D0008E0186F86B70C00934BF94F8890094F8B20086F86A0006F16C0010F00EF9204CE7
:2074F000206810F47F0F0CD086F82C70206806F12C01424600F47F003063304602F01CF9B5
:20751000206810F0FF0F0BD02A2086F83C00206806F13C0100F0FF003064304606F0AEFC91
:2075300000953046832101AA4B46FCF79BFB071C02D1304606F02EFE381C01D106E0E82025
:2075500070701820307030460BF068FC05B0BDE8F083C046A81100206C30002024140020CE
:2075700010870100F0B542F20400ADF11C0D0DF115010CF0FFF942F2050005A90CF0FAF9E1
:20759000664C67489DF81510A0666420414321666449C4F884109DF814104843E0676248F9
:2075B000C4F8A0006148007880B942F2020069460CF0E0F968460EF0E3FE04F15C000BF072
:2075D0008BFD04F134000BF0CFFF27E042F2030069460CF0CFF90EF0FDFC05466846294611
:2075F0000BF098FB2D1A04F1780084F85B500BF073FD04F134000BF019FD012742F202000F
:20761000694684F854700CF0B5F968460EF0B8FE04F15C000BF060FD84F85870E8200DF16C
:2076300016010CF0D9FB9DF81600032804BF012084F8B40094F8B80000286DD13C4D002115
:20765000302205F1080009F098FB20460021332209F093FB3748E861374F6F6105F11000B7
:207670000BF03AFD42F21B000DF117010CF082F99DF817000DF1170185F82C0042F21C0031
:207690000CF078F99DF817109DF8170085F82D1095F82C10012641B148010EF073FC286328
:2076B00008B910F036F895F82D0040B100EB800080B20EF067FC686308B910F02AF81F490C
:2076D00005F138000A270A684B6802607F1E436000F10800F7D1002195F82C7085F8881054
:2076F00047B1286BFF220346C2777F1E997703F12000F8D195F82D7047B1686BFF22034663
:2077100002717F1ED97003F10500F8D12846062209F033FB84F8B86007B0F0BDE82D002054
:2077300039390100F5F200009F760100ED130020A42E002075B00000002A7515D08A010083
:207750002DE9FE4F0CAF8A4699460446D7F804B00292594603F0C2FA06466A480578002EF4
:2077700000F0CB803888F082DFF8AC8134751DB1012C04BF1520307506F1800059460B2204
:207790000FF0ACFB012C04D00D2C1CBF7068401C00D170683062002598F838003565002800
:2077B000B56543D0DFF864B1052C18BF012C38D14FF0040AF18A86F86BA0534886F869503F
:2077D000C90938BF29380078029986F86A0006F16C000FF092FF0BEB8407386810F47F0FCE
:2077F0000CD086F82CA0386806F12C01012200F47F003063304601F09FFF386810F0FF0FB3
:207810004FF0030A0BD02A2086F83C00386806F13C0100F0FF003064304606F02FFB98F8B0
:20783000380018B1D8F898100D2C13D00095029A4B4630465146FCF715FA071C5ED1E41F7D
:20785000012C03D8707E40F020007076304606F0A1FC53E005205C4686F86B00343409B1DE
:20787000FF208847206810F0F70F12D02A2086F83C0098F80120206806F13C01012A00F00E
:20789000FF0030641CBF20F008003064304606F0F5FA0095029A4B4630460321FCF7E2F939
:2078B000071C2BD11A4806603489756801A964200CF092FA174E6D1E231DA01C99B2A6F8AC
:2078D0007800C1F3022040F0080005F801090A1F297091B2AA1CC6F88450104608F0CCFE96
:2078F0009DF8040000280CBF49F24E0047F60E20C6F8C000C6F8800000E01A27F8B2BDE8CC
:20791000FE8FC046241400205A1200200887010098180020280D0020EC1300202DE9F041C5
:20793000724B734ADFF8C0810C46D128014610DCD12879D0713800F0B280401E00F0AA80A2
:20795000401E00F0A380113810D04C3800F0878007E0D23853D0401E40D0401E33D0401EC1
:2079700028D008460FF05DFC0B2802D1F420BDE8F0815B4D05EB8005A97809B9E87850B1C8
:20799000E878884208BFFB2000F0A880227891426ADC904268DB534E7068804729786A7828
:2079B00007464046401821460FF098FAB1683846884792E02178022956DA1846641C0422C4
:2079D00000EB810086E0207832284DDA1746C100241D182201EB001178187BE02678304617
:2079F000022841DA2C2505FB0680611C102239300FF074FA616905FB0680C1646DE022787A
:207A10006178022A30DA02292EDA40462C2301EB42064F1C03FB0205022285F8387000EB67
:207A3000460000F5DE7018E022786178022A1BDA322919DA2C23404603FB020595F830300C
:207A50009942A4BF4B1C85F83030322303FB021101EB4101032240189030A41C3AE0207851
:207A70006778022800DA17B1E820BDE8F08141462C22C5197E1C02FB00136A0083F8286063
:207A900002EBC50288180A227C30E6E72CB3184608221FE00CB310464FF496621AE0B4B9C0
:207AB000404600F17C04A0F1080200F1900300F5DE71022042F82C4F9360401E116104F1CD
:207AD0000A0403F1960301F10401F3D105E040465822243021460FF001FA0020BDE8F08170
:207AF000247901008C140020A021002014280020642300202DE9FF47604C804660680F4649
:207B10008047A246674E684D654C8146B8F1010F5AD00FF0A7F9002851D0594800780028B8
:207B30004DD158480078002849D157480078002845D156480078002841D1554800780028DB
:207B50003DD154480078002839D153480078002835D152480078002831D1002009F0EAFA47
:207B700068BB207858BB012FA0461FD04F4F326AE86897F90010344611F1020F05D0926B99
:207B900097F900109047E868226A494E96F9001011F1020F05D0926B96F900109047E868A1
:207BB000226A6FF001013170397003E00C35203628683268012188F80010D1698847DAF84D
:207BD00008104846884755E0012009F0B3FADAF8081048468847207801283DD1DFF8D490D3
:207BF00099F8BA000028FBD1306A436CE868022102AA98479DF80800A84660B199F8BA0008
:207C100048B92078012827D10020012F207023D00FF034F920E0DAF804008047264F022166
:207C3000814600222170306A7A81244B85688DE80600D8F80C0008373946A847002801D5C7
:207C50000FF032FB1E4991F90000401C0870DAF80810F7604846884720781A4D022803D188
:207C7000287808B10FF020FB2878012802D020780228FCD00090BDE8FF87C0468C140020D7
:207C90001C3200201E320020203200201D3200201F320020CA1A0020CB1A0020CC1A002095
:207CB000E51A00202816002084190020C81A0020C91A0020282D0020280D0020DD2E01009F
:207CD000CD1A0020E41A00202DE9F843644C0746207808B10FF0E8FAA0460120614988F8BE
:207CF00000000978012902D00021FFF703FF5F4D60495F485C4C012F2A68D1F800900078A7
:207D1000A77035D9BF1E52D07F1E13D07F1E02D0781E47D043E092F86900207192F86A00F8
:207D3000E0700020607102F0A3FE2A68002A64D1BDE8F883002860D0564ED6F8981021B10A
:207D5000032088472A6896F83800002855D0776D002F52D0D06D20B102210023B8472A6862
:207D7000776D106E002848D008210023B84743E000202071D18A4048C90934BF90F8891069
:207D900090F8B210E170A77837B990F867701FB10229C4BF0220E07002F06AFE2CE00FF075
:207DB00083FA29E0002020710FF0D5FC24E0334F38788600D9F83C00804779683C22401A83
:207DD000B0FBF6F0B0FBF2F151436278401A9101A1EB8201091AD9F83C003C318FB2804766
:207DF000274906FB0700086791F8740000F0F00040F0020081F874002A682248007878B9EB
:207E100012B90FF051FA2A685168087800F02000E0718878A0710878800901D20FF09EFB8C
:207E3000A078042819D0184D68688047A17802290CD016490F7817B915490F7837B1022143
:207E500088F80010A9688847BDE8F883832188F80010A96888470EF033FCBDE8F883C0461B
:207E700020320020E41A0020C4180020640E00202414002048160020A8110020C819002024
:207E9000280D0020183200208C1400201C3200201E320020EC1300202DE9F04389461446E4
:207EB0000546ADF12C0D69460DF0CCF85FEA000800F0C480AD1C0226284602A90BF0D9FAC3
:207ED000071C00F0BB809DF80900814509D0F6197D1908F10200B61CAD1CB6B2B042EBDCAB
:207EF000ACE0401E05F1020500F08B80401E52D0801E38D0401E2BD0401E24D0401E18BF8A
:207F1000622040F0AB80202F40F0988028686F6805F10801206004F10806676001F108052E
:207F30000A684B68326004F1100773602A6868683A6005F108067860306804F118010860B5
:207F500073684B6089E0022F78D12888208084E0202F73DC20460021202208F00EFF3A4608
:207F70002046294677E0042F68D12888AD1C208015F8010BA070287800F00100E070287896
:207F9000C0F3400020712878C0F38000607128784011A07161E00A2F50DD0DF112000021CF
:207FB000162208F0EAFE28682D1D20602988271D42F20B00398004A90BF0DCFCBDF810000D
:207FD000A18888423ADCA81C10F8011BA17110F8011BE17110F8011B217210F8011B012319
:207FF000C1F3C202A2720DF1120200F0F7F928B39DF82700A0819DF81670E78104F11000B3
:2080100026E0042F1ADD0DF112000021162208F0B4FE15F8010B207015F8010B607015F86E
:20803000010BA07015F8011B0DF112020023C1F3C2002071284600F0D1F908B967200DE052
:208050009DF82700E0809DF81670278104F10A000DF11601112207F023FB00200BB0BDE855
:20807000F083FEE72DE9F04F674C2068ADF12C0D002840F0C58004F124063068002800F0C5
:20809000BF8062480078022800F0BA80614D281D006880470A90606AB046074678B35C4E7D
:2080B0004FF0000A4FF01D093B7D0820711E11F8012F9A421ED0401EF9D1404639465246CB
:2080D0000CF050FD787E30F07F0005D194F82F00401E84F82F0004E094F82E00401E84F8A0
:2080F0002E0087F8019057F80CBC384609F0FAFD5F4602E0BA4657F80C7C002FD4D1352026
:2081100007F0B6FB444EA968002849D1452007F0AFFBA96800283DD1D8F8000038B1017D3E
:20813000252904D050F80C0C0028F8D110E078B196F8580050B3684601A907F023F93748D0
:2081500000990078001F884213D8012086F85500152007F08DFBA96848B10A98884720687F
:208170000DF106016C3004F033F858B10FE00A9845E0252007F07CFBA9680A98884700201B
:2081900086F855000420FFF79FFD39E0192001F04DF935E00A98884708200BF0F9FD2FE00F
:2081B0000A98884796F8B400A8B10EF049F9317800290EBF0921491EC9B201EB81017118C1
:2081D000D1F802100FF0A7FA42F21071814284BF6431081A00D800206968002808BF0620C4
:2081F000DBD0C6F8980088470446D6F8A010D6F8980006F1A8020CF0A9FFA96820468847E6
:208210000BB0BDE8F08FC046640E00207F160020E08A01008C140020E82D00205F2F002014
:20823000BCB50546694800880021820804D2B5F89A20D20828BFE82110F0600F04D1B5F896
:208250009A00800828BFE8212889B0F5006FA8BFE82195F8980030B995F89400002808BFA9
:20827000F52100F0AF80002940F0AC80DFF860E1D5F8A870DFF860C19EF8381017B9012967
:2082900003D028E0002900F09C80D5F8A81060468D3041F002010778C5F8A8101FB141F0AD
:2082B0000801C5F8A810D5F8A81011F0FF0F05D02A2085F83C0001F0FF072F6411F47F0FA7
:2082D00007D00420D5F8A87085F82C0007F47F0028639EF83810002059B33E4995F89470DE
:2082F0000B6804226FB925232B750968C98AC90934BF9CF889109CF8B21085F86A10891C1D
:2083100008E015212975D98AC90934BF9CF889109CF8B21085F86A1085F86B2005F18C075E
:2083300085F869003B6805F16C010B607A684A6001E00121297595F89C70EF760446AC6550
:20835000B5F89A102C6595F89D30E9826A682B7795F82C702A620F2F09D00246B5F8A40087
:2083700005F12C0100B90122284601F0E5F928BB95F83C10FF2901D1AF6D27B105F13C01D4
:20839000284605F07BFDC8B9009495F89810B5F8963005F18C022846FBF764FC071C0CD1F1
:2083B0002889B0F5006F03DA284605F0F3FE04E0E5206870284609F095FC3846011C01D191
:2083D000BCBD1821284607F049FDBCBD20150020EC130020640E0020A81100202DE9F04F83
:2083F000154601F00708C1F3C2074FEAA119044683460C22ADF1240D0021684608F0BDFC12
:208410006248B8F1000F36D0B8F1010F7ED1228801A9A6780A80E41C8E7014F8011B01F0C9
:208430000F018DF8081022880DF10A031A80BDF80A30A41C4FF0000C6B75019ECDF818C01A
:208450004168B14207D1017A9DF80820914202D14189994208D006990C30491C0629069137
:20847000EED96046614601E0017840788DF800108DF8010022E014F8013B14F8016B8DF864
:20849000003000228DF801600C38079210F80C1F994202D14178B14207D00799491C06291F
:2084B0000791F3D91046014603E04168027A4089687501918DF80820ADF80A0003A806F06E
:2084D0001BFE9DF800109DF80100B8F1000F11D0B8F1010F1AD1019904989DF808209DF873
:2084F0001460484086EA02010918BDF80A20BDF8160004E09DF80C2051409DF80D205040AA
:20851000401803D1EF701FB1022F05D0002039E02188281DA41C0180B9F1010F27D0B9F127
:20853000020F2CD1BDF80A10281DC91DCA10214607F0B6F8BDF80A00C11D04EBE104F0B12B
:20855000401E811000EB5171C910C9B26D182B798710012600EB577121F00701401AC0B29C
:20857000401C06FA00F0FF301840287107E0291D20460AF055FF207804EB8004641CA4EB84
:208590000B04A0B209B0BDE8F08FC046D41500202DE9F04FADF1840D209002F005FB0EF05A
:2085B0005FF90026012804D10EF090FB022808BF01265B490868C0F38150012806D151F8AD
:2085D0000C0C0127010E07FA01F00643554800780DF0A6FD544D2C46286038B1FF2204F1B2
:2085F000400107467F1E01F8012BFBD1209909684FF0000901F0FF02FE2A1DD0DDF880C0C1
:2086100001F0FF074A460123FF2F0ED0B84203D903FA07F73E4201D002207EE001F0FF0100
:2086300047EA0909611881F840205CF8041F521C01F0FF07FE2FE7D1092005F049FD2098B8
:20865000002124220823606017A80FF03FF94FF0010804F1240017AA8DF8748041460FF0A1
:2086700031F9236843B3002794354FF0040BBA4608FA07F0064219D119EA000F04BF07F00A
:20869000FF0141F4C04105D0E019209B90F8401053F82110254804F025FCF8B24FF0FF311C
:2086B0000EF016F92368C5F800A001E0C5F800B07F1C2D1D9F42DBD301A8002130220823AC
:2086D0000FF0FCF81A4E30780025102101AB0990184A009504F108000FF0ECF80DA8282216
:2086F000082329460FF0E2F80DAA7068124914952B46139004F160000FF0D4F80F4951F88F
:208710000D0C474620F4F85040F4005041F80D0C0B4EC1F8FF7F2846376021B0BDE8F08FE7
:20873000B43F0050193200204C2B0020007FC767E88A0100FD680100814101000D30094015
:20875000080009402DE9F843644C002605466676687D0628A4BFE8216176A97D0E2903DDD7
:2087700003281CBFE8216176032805D15C48008840083CBFE820607695F8280008B1E8203F
:208790006076E87D092801DB0A2801DDE8206076287E08B1042801DBE820607604F118073A
:2087B000294638460CF056FE291D112207F12C0006F076FF95F8280004F11809002804BFAE
:2087D00084F86060A87D04D095F8290084F86000688DA4F85600687E84F85800A87EDFF824
:2087F000048184F85900E87E822784F85A00287F98F8A76084F85B0098F8B63084F85C7057
:20881000394F84F85D6005F11D01E763042684F8406098F8B72084F85E3009F1490084F8B3
:208830005F200B220EF05AFB607E00284ED1687800284BD1287EA77E8DF800000FB1EA20C6
:20885000607605F11701E72000F02AFD94F8600028B1287E022808BF01208DF8000098F874
:20887000B7009DF80010884203D0E820694600F017FDA77E1E4C601C007808B10EF014FDE9
:20889000B8F88A0019490880C7B1032F12D0052F05D0012F03D0022F01D00EF005FD0220E8
:2088B00060700BF039FF4FF6FF70A8F88A001149088005E00BF030FF032000E001206070E2
:2088D0002720287030460DF07BFE01E02A20287028460AF0A3FABDE8F883C046B0300020CF
:2088F00020150020A8110020597301008C19002088310020721600202DE9FE4F544E0746D5
:20891000301D00688047534C00258346A01C05701FB10DF075F90AF045F994F83800B046E0
:2089300010B1E06B00B1804709F014FEDFF8749109F11C0090F900000EF0F4FB0DF0FAFA3F
:208950000EF0E6FB0EF06AFA0EF05CFADFF808A107270AF1240656F8040B00B180477F1E2D
:20897000F9D13E480560456005614FF470018160C1600AF1040007680FB10BF0EDFE3848DD
:208990004E4600688AF80E508A3EC0B112E048460CF0E8FA029002A80BF0DEFE21E04846B2
:2089B0000CF0E0FA019001A80BF0D6FE14E068460BF0D2FE07F054FD00280090F7D1294822
:2089D0000078012803D028460146FFF793F82648264F057007F12409786A0028DFD109F1AC
:2089F0000409B86A0028D2D17D62BD622048A06187F82E501F4BE36187F82F501E4A226271
:208A10001E4961621E4B87F830501E4AA362204BE2621D4963601F4A21631C4FA260204BAA
:208A300065701D4967631D4FE16058462761D8F808106361884706F18D01522000F030FCC0
:208A500096F8A7000AF0F8FE2846BDE8FE8FC0468C140020EC13002014150020241A0020B5
:208A7000242D0020E41A00201B320020640E00200FEB0000ED7601009D6101003182000048
:208A900039D30000916501003973010031B60000D7BF00009DB100003533010075F5000078
:208AB0009D240100321200202DE9F041071CADF1200D00F0C180F86B002800F0BD80B7F8B3
:208AD0004020002A00F0B880007817F130014FF0000603D097F83810052902D0002E00F016
:208AF000AB80584C401E2BD0801E18D0C01E40F0A380012A40F0A080514C0725E0788DF866
:208B10001C5000280CBF0121311C3046E17009F055F9E07802228DF81D0028460BE0012AC7
:208B300040F08A80B4F854000122401CA4F8540004208DF81C00394607AB02F0BBFB7BE083
:208B5000684631460C2208F018F9B7F840000B284CD1FD6B15F8010B84F820002B786878CA
:208B7000AD1C03EB002328460EF039FA8046281D0EF035FA0546387A2077022806D03968FF
:208B900004F1140001607A68426001E03888A08203F00100190928BF40F00800590928BF96
:208BB00040F010006084834218BF0226B8F57A7FADF8020008D32448404505D3C4F824806C
:208BD00040460CF0B1FD00E00226606AB5F57A7F019007D342F21070A84203D3A5620EF0FC
:208BF00033FA00E00226A06A029000E0012602258DF8016068468DF800500AF02DFF0DF1D9
:208C10000D009DF801108DF80C500EF089FCBDF802100EF085FC01990CF01BF802990CF0A7
:208C300018F839460D2203AB284602F043FBB4F85A00401CA4F85A0008B0BDE8F081C046EE
:208C5000A410002090120020407E05002DE9F843634C5C4D5C4EDFF87881604F94F8E41059
:208C70000846401E0B2864D8DFE800F07E2C43062343062343067967042907D001220A290D
:208C900045F8212C14BF0220032004E0202045F8210C0120024684F8E200002045F8390C2B
:208CB0000827C5F8FF7FC5F8F37F45F8392CBDE8F883052914BF09200620002784F8E40072
:208CD000376078E094F8E170383D0120002FC5F81B0004BF0620002102D00021F1600320AA
:208CF00084F8E400032045F8010C31603068800861D294F8E4103548012703290ED000681C
:208D1000456800216022052300914046A84794F8E400062814BF0A200720CFE70068456838
:208D3000002160220523022000904046A8470420C4E70EF0B3FDBDE8F8832648264F00268B
:208D5000012506600E203D6004F036FE02200CF0A3FC84F8E45084F8E360BDE8F883002018
:208D700038600C25786024E04FF08059D9F8A0010168202088472C3D0F2045F8010C41F623
:208D90001D56C5F80360D9F8A401466800214FF4C0720723022540460095B047D9F8A4019D
:208DB000C66800214FF4C07207234046B0470120386084F8E45004F178000EF06BFDBDE857
:208DD000F883C04639400C4038600C40A401001000A00C402C500C4004800C4034600C4040
:208DF000940F00202DE9F04304466668A7680D46ADF1340D0EF08AFD3178012903D10EF0D4
:208E100081FD0020A9E04FF0010886F800800EF079FD287870706878B07068687060A86831
:208E3000B060E868F06028693061287D3075687D7075A87DB075A869B061287F3077687F9B
:208E50007077A87FB0774FF00009C6F82090C6F830904D4675627563B562B56386F82C502E
:208E7000102386F83C3086F82D5086F83D50786805F02EF9204605F0AFFA204606F028FE3D
:208E900070B937480068C16838688847786804F093FD0EF03BFD35700EF034FD2C465BE0FF
:208EB00001A82946302208230EF008FD0694387BCDF800902B4A0990B96801AB06F1800016
:208ED0000EF0F8FC01A82946282208230EF0EEFC05942549386901AA2B46079006F19C002D
:208EF0000EF0E0FC01A82946242208230EF0EEFC8DF81C80B07838B906F1D000294601AAFC
:208F10000EF0E0FC19483061707838B906F1EC00294601AA0EF0D6FC1548F06001A829460A
:208F3000242208230EF0B2FC0695ADF814501149079406F584700A2201AB0EF0A3FCB969E5
:208F5000FA6906F140000EF063F90B4A06F16C00042123460CF062FF20460DB0BDE8F0832F
:208F7000D0010010B5BB00005D4E01007D7601007576010001FF0000797301002DE9FE43C0
:208F9000604C614D0E46B00959D35D4800F1280980464DE00178D0290EDBD02909D181784D
:208FB0003970C17879700179B97085687D60C168B9600EF03FF947E004F10805286009F047
:208FD0002DFF28460BF0C8FB3EE0884798F83010491E88F83010A9688847009801788DF8CF
:208FF0000410A0604778CFB1DC2F0DD0DD2F0BD0E42F09D0F32F07D0DE2F05D0DF2F03D097
:20901000E82F18BFDB2F0BD104F08EF99DF80400162805D168460BF09FFB01E009F0FEFE2B
:209030009DF80400162803D004F108000BF094FB48460BF097FF002869680090C5D1F00BB6
:20905000A846C00305D0314F07F00AFA00280090A0D1700905D32E208DF8040001A809F00C
:20907000DDFE700805D325208DF8040001A809F0D5FEB00805D326208DF8040001A809F071
:20909000CDFEF00805D327208DF8040001A809F0C5FE300905D329208DF8040001A809F06B
:2090B000BDFEF00908D300208DF805002D278DF8047001A809F0B2FE300A08D300208DF80E
:2090D000050030278DF8047001A809F0A7FE6068D8F8041080B18847616800270091D8F8E7
:2090F000081067608847009804F10806306009F095FE30460BF030FB0020BDE8FE83C04613
:20911000640E0020141500208C140020381A00202DE9F04F0746880FADF1140DC0F0B28058
:20913000002009F04FFE5B4D4FF000081C35C5F80080564845F81C0C01200DF0F1F9564893
:209150000EF09AF955482838BC6890F8342040F60A06C34600F1280189468246A0F82A802F
:2091700090F835300E8002F0F002C0F82CB003F0F00180F8342041F00101A4F802809AF859
:20919000042080F83510012A01D17B7CABB1B8680088A6F10801814205D0218B4FF60F406E
:2091B0000840208304E0218A4FF60F4008402082B86887F8118004F04BF8B868694604F07D
:2091D00089F968460EF090F83346D91F4A1C00E03446666836B13088834203D0814218BFF9
:2091F0008242F5D1C4F80490607B00F0F00060730AF114000EF099FA80680088814220D034
:2092100082421ED03E8C0EB397F82C0097F82D60C7F824B000F0F00087F82C0006F0F00026
:2092300040F0010087F82D0007F12003CAF82C3099F80D00A7F8228000F0F00089F80D00BB
:2092500004E0D9460AF1400080E8000328680028FCD0C5F8008001200CF038FC012808D042
:20927000607B00F0F00040F00100607308480EF003F9B9680A8A4FF6FF3010400882B868B2
:2092900045F81C0C05B0BDE8F08FC04601010E04592B0100001004406D350000980A002029
:2092B0002DE9F0475E4E80460F46B8F1450F07D106F13004342220460DF010FEF466ACE0DD
:2092D0000DF05AFA3A2808BFF42000F0A780554C04EB8004A07810B9E178002938D0E17801
:2092F000814208BFFB2000F09980B8F1580F25D0B8F1600F1BD0B8F1E00F0FD0B8F1E80F91
:2093100005D03A78904220DC91421EDB20E006F1B7003978007881421AD17EE097F90000A9
:209330000AF0C0FB4FF6FF7181420ED010E038880A280ADBB0F5804F07DA09E038888F2896
:2093500003DB46F2B041814202DAE820BDE8F087354D6868804721786278824606F1640084
:209370008146401839460DF0B9FDA96850468847404650384FD0801E37D0401E48D08D3809
:2093900041D0401E28D0401E3AD0801F45D16868804704460DF04EFDFCF76AFC96F9A60082
:2093B0000DF0C0FE0CF0C6FD0DF0B2FE0DF036FD0DF028FDA9682046884796F8A7000AF0AF
:2093D0003BFA09F129015220FFF76AFF0EF0C0F818BB09F0BFF820E096F8A7000AF02CFAC5
:2093F00001281AD01A20BDE8F08796F88D0018B902200BF05DFB10E002200DF09DFF0CE0FC
:209410000DF000FD09E096F9A6000DF08BFE04E00DF004FD01E00DF07BFE0020BDE8F08729
:20943000A81100202C8201008C1400202DE9F8435B4D804695F83800002798B12A6F8AB10C
:20945000D5F8900070B142F21A0069469047D5F89000804730B19DF8000018B1B8F1E10FAE
:2094700008BF01274F4A02F1B70000780CF0B2FB407B02280CBF052601264D4C206800283E
:2094900000F08B80B8F1000F91466ED0B8F11B0F02D1017D052968D1B8F1E90F25D027BBF1
:2094B000B8F1E10F16D10DF0D9FD90B12068C18AC9080FD299F89810817699F886104A1CC6
:2094D00089F88620406881703046FEF7FDFBBDE8F8832068B8F11C0F16D1216A002949D029
:2094F000884700202060BDE8F883F1200DF073FB2768B87E50B90DF0B1FD20B12068C18A34
:20951000C90801D2D6E7206847462FE07868398907F0B2F878680088000905D395F8380065
:2095300010B10BF001FB2768F88AC00811D3387E00F07F003876387D032803D1787E40F0F9
:2095500004007876F0200DF046FBE168206888470FE015490126B87E0E70401EB876F02057
:209570000DF039FB11480078AFE70027477008F0B9FB2068C08A000A0AD395F8380018B96A
:2095900099F8A7000AF058F999F9A6000DF0CAFD0020206010200DF0D7FEBDE8F883C04674
:2095B000EC130020A811002018320020C6180020640E00202DE9FE4F5E4C814604F1140AC2
:2095D00050460EF0B2F890468B46074608F0010000900EF09BF98425BBF1FF3F019017D122
:2095F000A6692EB1A069C068814508BFA0690DD00EF08CF9DAF800608AE0F168894540F053
:2096100086800EF07FF9301C00F08780B0F924B058460CF0C9FA00287FD0A16981425CD031
:20963000B84217D104F1B0000DF03AF860690068606197F82700394640F0040087F8270063
:209650000AF10C000BF004FE5FEA980021D3676901221AE00FB905B31CE0396888423AD142
:2096700004F1B0000DF01CF839680868386091F8270040F0040081F827000AF10C000BF0F5
:20969000E7FD5FEA980004D300224846394608F001FD002501980EF035F9A179627A607940
:2096B00041EA0203184310D1012939D0012A37D026691D480DF0E0FE022104F1D4000DF011
:2096D00055FC30460DF0D8FE2AE004F1D40002210DF04CFC24E03F68BCE7009F90F82720E9
:2096F000012505FA07F13E1C41EA020180F8271014BF0E480E480CF069FB5FEA980004D36F
:20971000616948462A4608F0C5FC002505E03668002E7FF472AF0EF0F5F801980EF0F2F8E2
:209730002846BDE8FE8FC0466D3500000100020401000104700A00202DE9FE4F0746104624
:20975000002F00910CBF4FF0E80B4FF0000B002900F0AB80BBF1000F40F0A98060B17868A9
:20977000401E7860F82101707868401E7860002606703889801C3881009C4FF000094FF02E
:20979000020ADFF83081CDF80490083C14F8080F00F00F010F2900F08580012820D00428F3
:2097B0007AD1454D95F83800002875D0296D60688847061C26D03889B7F84C103018801C95
:2097D00081421FDB78686D6D6168019B3A46801BA847B8B178683D89801B786076195AE048
:2097F0000098019E042309EB0001C91C11F8010FFF2841D021283DD13889B7F84C200B3062
:20981000824202DA1A20BDE8FE8F7868B8F8A020401E7860121202707868401E786098F86A
:20983000A02002707868401E7860019D057098F8A2007A68107098F89E2078681201401E8A
:20985000786042F00F02027098F890C098F871207868401E786042EA0C1202707868401E5A
:209870007860212505707868F61DB6B2401E7860052505705B1EB9D17868C6F30121401EF9
:20989000786041F0880101707868401E7860067038893618B61C3E81BAF1010A09F10809C8
:2098B0007FF474AF7868B86501E04FF0E80B5846BDE8FE8FA8110020EC1300202DE9F04FD5
:2098D0008A4609AF4FF08051ADF11C0D90463D69059001F5D8700490D1F8B001D7F808B035
:2098F0004169069327208847524C4FF00309143CC4F884970126C4F87C67C4F88097022034
:20991000C4F8FC06F868C4F8080430460DF0D1FED4F808040008F8D2D4F88C07800F28BF90
:20993000B14655D2681E41460C238DF800000DF1010011F8012B5B1E00F8012BF9D1022D6E
:2099500019BF0020011C98F80C1000208DF80D108DF80E008DF80F000099C4F83C15019B0B
:20997000C4F84035029AC4F84425039BC4F848353968BAF1020F4FEAC542A1EB0A08A2F53C
:20999000002106D34FEA4A52A2F580026FF315021143264A0A43C4F84C258246C4F85085BF
:2099B000BBF1000FC4F854A5214DC4F858B511D02E6078682060C4F808B030460DF079FEC3
:2099D000D4F88C078008F8D3D4F88C07000801D3CA4627E0C4F88497D4F88C0710F0030F2B
:2099F000FAD1D4F8800720F00200C4F880073F7D47B1049F3868016A272088473868016962
:209A100027208847C4F87C670598C4F8806748B12E6006982060C4F80880C5F800642062B5
:209A3000C4F82880504607B0BDE8F08FC801042000004842184002402DE9F04F894609AF54
:209A50004FF08051ADF1240D9246059038683D69079001F5D8700490D1F8B001D7F808B0FA
:209A70004169069327208847504C4FF00308143CC4F884870126C4F87C67C4F880870220D5
:209A9000C4F8FC06F868C4F8080430460DF011FED4F808040008F8D2D4F88C07800F28BFCF
:209AB000B04653D2681E51460C238DF800000DF1010011F8012B5B1E00F8012BF9D1022DE0
:209AD00019BF0020011C9AF80C1000208DF80D10019B8DF80E0000998DF80F00029AC4F83D
:209AF0003C15B9F1020FC4F84035039BC4F844254FEAC542C4F84835A2F5002106D34FEA13
:209B10004952A2F580026FF315021143254A079D0A43C4F84C258146C4F85055BBF1000F44
:209B3000C4F85495204DC4F858B511D02E6078682060C4F808B030460DF0BBFDD4F88C076D
:209B50008008F8D3D4F88C07000801D3C14624E0C4F88487D4F88C0710F0030FFAD1D4F88D
:209B7000800720F00200C4F880073F7D47B1049F3868016A27208847386801692720884761
:209B90000598C4F8806740B12E6006982060C5F800642062079FA760A762484609B0BDE893
:209BB000F08FC046CC01042000004842184002402DE9FE4F524D286808B90DF075FB554C9A
:209BD00004F13800DFF83C91DFF840A1DFF8408107789FB94D46686880474B490F7847B938
:209BF0005246A96817782FB983234246137088476DE0A96802234246137075E0D4F898105E
:209C100009B104208847676D2A685FB1D06D20B102210023B8472A68676D106E10B10821F0
:209C30000023B8473C4E306A3C4F016CF86888474D46834668688047029033480578002DFD
:209C500048D150460078002844D1D4F8841000208847F42001A90AF0BFF89DF90400304DBB
:209C700058451ADC6B79C3B9D9F8081002988847A878042801D00DF017FB042140466F79D0
:209C90000170D4F88410781C687109B1032088470320688100F006FD27E083214046346AFC
:209CB0000170636CF8686A4600219847B6F90400BDF90010884214BF0020012007F0FEF9FF
:209CD000D9F80810029888470835287838700CF0F7FC0AE0022140460170D9F80810029827
:209CF0008847D4F88410042088470E480078012803D000200146FDF7FDFEBDE8FE8FC046DA
:209D1000640E00208C1400201C3200201E32002020320020EC130020281600208419002057
:209D3000C4180020E41A00202DE9F8434F4E84460120002430704E48504D04704D48DFF849
:209D50003881047005F14E00008804EA0307B146002F4FF0020606EA020608BF002E14D1C3
:209D70004FF0E04720461F401040002F08BF002803D11D2006F0B8FB54E0454695F9000033
:209D9000401E28700DF086F84CE0424692F900303C4E5B1E137043F20842824207D06F8E36
:209DB000931C834203D0BA4218BFBB4217D1304608300068826C60469047008843F603014E
:209DD00081420BD0204601F0F7FF98F9000000283FD098F90000002838DD42E06F8EB5F826
:209DF0006A1043F60400884205D0B84203D0B5F84E20904203D12248007803281AD1B1F5D1
:209E1000505F05D0080B0BD31D2006F06DFB07E01D480168304601F5C071016005F070F812
:209E30000DF014F898F9000098B198F9000000280CDD16E0022811D0204601F0BDFF98F9E8
:209E5000000030B198F9000000280ADC0DF02CFA07E020460146FDF74DFE02E0204606F03E
:209E700043FB89F80040BDE8F883C046E41A0020CC1A0020CB1A0020CD1A0020280D002028
:209E9000C6180020401600200C0100212DE9F041554C2079ADF1400D032818BF607140F0A1
:209EB0009E8000256571A84601A824220823294684F804800DF00AFD032001A98DF81C0090
:209ED0002A4601200DF0DAFC1D27A0602E46A5700AAB3846414604220CF063FE9DF8281037
:209EF000E378A52907D19DF82900FE2803DC9DF82B20962A09D0242902D0B72918D11FE02E
:209F10003E46EBB99DF8290019E0B5B1984203DAFE2B18BF01280BD1984203DD012B08BF83
:209F3000FE2805D0284606F02DFE9DF8290004E0384606F027FEA57802E03D46A570E07065
:209F50007F1C1E2FC4DD8DB926B91D2009F05EFD042015E0A67030464FF480510AF0E6F821
:209F7000E08041463046FDF717F80AE01EB1304606F008FEA57828464FF480510AF0D6F8DF
:209F9000E0800AAF174D00970EA82968AE8801600EAB868093E8030042460C2306F030FEA7
:209FB000E6880A2809D1384641460C2206F0E5FE40F6EF70801BADF82E00BDF82C000EAF6A
:209FD000401CADF82C002968AE8839600EABBE8093E803000C220AAB06F032F9607910B0D2
:209FF000BDE8F081F88A0100441A00202DE9F84F0F4605460CF0FBFB4FF6FF71814208BF0C
:20A01000682000F096804C4C410001EBC0002418D4F8026016B9D4F80630F3B1D4F806105C
:20A03000B14208BF692000F084806078401E0FD0401E07D0801E10D13868864273D881429A
:20A0500071D30AE0388886426DD881426BD304E03878864267D8814265D3384E7068804739
:20A0700042F20208B346DFF8D8A00090A5EB0800012816D9113831D1207862785646002190
:20A09000301806F07AFE637838460DF073F8834298BF181C02D938460DF06CF80246304671
:20A0B0001EE00BF097FF06463846314608F032FE361A5FFA86F9DBF80860B9F1000F30D07C
:20A0D000207862783946504405F0EAFA1D484146A94218BF401C80F8009008E050466278A8
:20A0F00021784018394605F0DBFADBF8086008F11900A84204BF00208AF8870008F11A00E0
:20A11000A84213D19AF887009AF886104218322A01DC08430AD102208AF8860030278AF864
:20A1300087700098B0476A20BDE8F88F0098B0470020BDE8F88FC046548001008C1400205D
:20A15000302F0020422E00202DE9F0410C4601467138022840F29680133824D04D4F4C3886
:20A170007AD0401E61D0401E48D0401E36D0401E29D0401E1AD008460DF053F806460B2E62
:20A1900011D0424D6868804741498046B000425CBF1840184278394620460CF09FFEA96892
:20A1B000404688470CE0F420BDE8F0812278022A68DA3949601C01EB820104220CF08EFE01
:20A1D0000020BDE8F081217832295BDA334FCA00201D02EB0112B9181822EFE72678022ED8
:20A1F00050DA2C25601C05FB0671102239310CF075FE05FB0670C06C6061E1E720780228E9
:20A2100040DA2C2101FB0070667890F83800B04238DD23786278394602EB430201EB420161
:20A23000022201F5DE71A01CC8E72078022829DA2C2101FB0070667890F83000B04221DD36
:20A25000227860783223394603FB020000EB4000032209189031E6E72078022812DA2C21AE
:20A2700001FB0070667890F82800B0420ADD6278207839468018420002EBC00289180A22B4
:20A290007C31D0E7E820BDE8F081C0468C14002024790100A02100201428002064230020E4
:20A2B0002DE9F0434D4CDFF8388194F83F600027ADF1140D002E57D198F86660002E53D00E
:20A2D000C768007A454600F00701C0F3021900E0BF1C0E46701EC1B24EB17A783878B5F816
:20A2F0008E6000EB0220B042F2D1022710E005F16406443600E008374846411E5FFA81F9CC
:20A31000A0B3304639460CF017FC0028F3D0032794F83F0040F0040084F83F0002A80BF062
:20A33000F5FD01200CF04CF904F134018720FFF70BFF04F13C018520FFF706FF04F13D01E3
:20A350008620FFF701FF04F13E018820FFF7FCFE0120009004F134060196B5F88A30394628
:20A3700002AA0520FDF7ECF9002F33D198F871100F292FD0404690F890208A422AD090F89C
:20A390008D0038BB1748007820BB17480078012803D001200021FDF7ADFB144C60688047DB
:20A3B0002146134C94F83B20022A11D194F83820FF2A0DD00F4A176857B9576A47B989684E
:20A3D000884704F1200009F05FFA06F0D9F901E08968884705B0BDE8F083C0463830002073
:20A3F000A811002022150020E41A00208C140020EC170020640E00202DE9F04F474C6068DA
:20A41000ADF1140D8047464A92461178DFF8148102919AF80020A168A146012A0CD00124E8
:20A430008AF80040884798F80000012805D020460021FDF75FFB00E088473C4C3A4DDFF883
:20A45000F0B0E06805F1B001814206D1594691F90000002818BF00274AD1D9F804008047BD
:20A4700000270390374EA5F8B27006F138000578002D07BF4FF48600391C2E482021226ACE
:20A4900095688DE8030031492B4A2C4B10683A46A847D9F808506080002827D45946767831
:20A4B00091F90000264B294A401C087093F90000E260401C187006B18027234EA08FB6F8EC
:20A4D0008E304FF67F7101400F433843A087B6F88A00082204F13F0706F1A801A4F84A0021
:20A4F0003846A4F848300CF0F9FC01270398A847D9F804008047D9F8081017B9029A8AF8A4
:20A510000020884798F80000012803D000200146FDF7F0FA384605B0BDE8F08F8C14002054
:20A53000CA1A0020E41A0020280D002028160020CE1A002000004F8C90190020F114000085
:20A55000CD1A0020EC130020A8110020D80D00202DE9F84F994692468B4606460DF0D6F9EA
:20A570004D4C0090B4F92610B4F924000AAF401A40F6F871014008297ADAB4F92400401C49
:20A590006FF31F30A084B4F924800BF0DBFD054606F170000CF084F8C5F808B085F826A0D0
:20A5B000C5F80490A5F824803C48EE6097E80C00202100271940104005F1100383E8030014
:20A5D00004F1140085F827700368002B43D129460AF03EFE002844D0A6F8B88095F8270039
:20A5F00040F0800085F8270086F8BA70E07920B1207810B1E7710120207200980DF082F9B1
:20A61000A069002844D12078F0B9607901283FD00DF07CF90646A07988B9A86807F0A0FED5
:20A6300040B930460DF06EF904F1D40004210CF09DFC2DE004F1B0000DF02CF902E018499D
:20A6500001200870304621E001200CF087F919200CF082FE1CE004F1140029460AF0F8FD25
:20A6700048B9B4F9240000F6FF706FF31F30A0846FF0010809E0A6F8B88095F8270040F0B3
:20A69000800085F8270086F8BA7000980DF03AF94046BDE8F88FC046700A0020F1EFFF9F46
:20A6B000173200202DE9FC414648474C474F48490378A57862893878042D6DD101F13C06B0
:20A6D0003578884605F0F005357000268E63414908335A43424391F838500092002D50D072
:20A6F0000D46AA6F002A4CD0EB6F002B49D004F10801684690478446374BE178DFF8E8E033
:20A7100020791A68BCF1650F31D0BCF1000F28D1107D052811D13148017871B9186890F877
:20A730002C00042809D119686D6D906D096B3346A847002808BF1A2016D0294D6868804787
:20A7500028490E68002E08BFA96807D0A96804F10C02964213D03668002EFAD18847387840
:20A770000FE0704606706046FEF760FE22E082F8690082F86A107046E96F06701C2088474D
:20A7900018E01A49009E04F10C076161B6FBF0F138460CF08BF90DE091F83C4008338000A9
:20A7B0005A43884604F0F0045043886344F0030481F83C4098F8740000F0F00088F87400B0
:20A7D000BDE8FC8185190020C4180020C8190020280D0020EC130020640E0020351200201F
:20A7F0008C140020241A002020320020C19B00002DE9F04706464FF00108ADF1600D092246
:20A81000B07D8DF84C8006F117018DF84D000DF14E000CF063FB464D68688047814616A973
:20A830008120FFF791FC707D002854D09DF85800022817DA042000238DF80300347D8DF89E
:20A8500002809DF858708DF8013069468DF80040781C8DF85800D220FDF760F8812016A9D0
:20A87000FDF75CF800274FF0FF0A3C46307D8DF8217008A980F001008DF82000D120FFF71E
:20A8900063FCC0B99DF82200FF2814D08DF800006946D420FFF758FC20B1A968484688475D
:20A8B000192042E0307D69460DEB80000461D420FDF734F801E08DF822A08DF82440307D22
:20A8D0008DF8234008A98DF82000D120FDF726F87F1C322FCADB307D00279DF84D208DF82B
:20A8F00040000DF14E018DF841700DF142000CF0F5FA8DF84B80D02010A9FDF70FF8071C43
:20A910000FD1307D314610228DF828000DF129000CF0E4FA30690AA90F90D320FCF7FEFF75
:20A930000746A96848468847F8B218B0BDE8F0878C1400202DE9FF410546080BC0F0868094
:20A95000484E4449002401272246347006F1580077720CF0D5FE40480CF08EFDF068416855
:20A970008868B04608B9C86828B13F483F491C38C46150310160384608F024FA374E346000
:20A99000374846F81C0CA9684C80AA68128840F60200904205D00B8B4FF60F421A400A8347
:20A9B00004E00B8A4FF60F421A400A8200F1080C6F74ACF10702531C00E039464F6837B197
:20A9D0003888844503D0824218BF8342F5D127464F60487B00F0F00040F00100487308F141
:20A9F00014000CF0A2FE8068008882421BD0834219D0288CC8B195F82C006C8495F82D300A
:20AA10006F6200F0F00085F82C0003F0F00040F0010085F82D0005F120024A60487B00F099
:20AA3000F000487301E0C8F84840A868694602F051FD68460CF058FCA86802F009FC306896
:20AA50000028FCD03460A86846F81C0C0090BDE8FF81C046156A01006D3500001C1004409B
:20AA700001010E04700A00201C100440010007062DE9F84300204A4C8DF800000CF0CCFD49
:20AA9000E278484E414DDFF80C91012191404FF6FF725218024096F83800628120B3326F42
:20AAB00012B342F21A0069469047374827790378A3B19FB99DF8003083B1D6F8940068B133
:20AAD00080474946491C2A78097830B1678908314A43B0FBF2F0C019608127799DF8001065
:20AAF000608907FB01006081A078002847D1284F386AC06B80474E46804664892978707846
:20AB10003B6A08304443D86B8F0080476968224D2A787578214E3C23401AB0FBF7F103FAA1
:20AB300002F0B1FBF0F205F108034243891AB1FBF3F25A43891A05F10803691A641896F8FD
:20AB5000581096F83C5098B2083401F0F00107FB048341F0020107FB0032736596F87440F0
:20AB700086F8581005F0F000B26340F0020086F83C0004F0F00086F87400BDE8F883FFF70D
:20AB900091FDBDE8F883C04618320020C8190020281600208419002038120020280D0020AC
:20ABB000C4180020EC1300202DE9F0434A4D95F8E700ADF12C0D00287AD13F4F387B012466
:20ABD0000021242285F8E7407E6885F8E6000823C5F80C6101A80CF059FE002605F10C0098
:20ABF000069601ABADF814603449079632460CF049FE334905F1300001AB32460CF042FE0D
:20AC1000304905F1540001AB32460CF03BFEB96820468847DFF8BC802B4808F104037A7B37
:20AC300000781868C0F3815922B1B9F1030F04D185F8E140B9F1030F1ED0B9F1020F1BD02D
:20AC5000B9F1010F2DD14FF08059D9F8A4011F4F456831464FF040521C23032000903846CB
:20AC7000A847D9F8A40131464FF400720923456800943846A84714E002200AF025FDB9F17D
:20AC9000030F0CBF4FF47A7142F21071104800685435B1FBF0F128460CF0ECFD28460CF051
:20ACB000F9FD40460068C00802D230460AF00CFD0BB00020BDE8F083808A0100BFBC000012
:20ACD00099080100610301001932002000A00C40108B0100B03F0050940F00202DE9F84F0B
:20ACF00005464448DFF8109183462E18093699F8380034788846B0B1D9F8501099B10BEB92
:20AD10008507786B00F0FF0088478246D9F85010786B00F47F008847504480B218B13178A0
:20AD30004018001DC4B238481230007801280CD198F808704FB1314898F80930C1190E792D
:20AD5000C05C0019401DC4B200E000260D2D09D106EB0408B8F1F80FD8BF294F1CDD0CF010
:20AD7000A3FA05E030198046801C0BF07BFA074697B902200BF076FA011C0AD00BEB05000A
:20AD900090F825001A2708701E4E4F70307807F067FD0020BDE8F88F08F102023846002127
:20ADB0000CF0D1FC07F10C00002174220CF0CBFC07F13C00FF2110220CF0C5FC07F12C00D5
:20ADD0000F2110220CF0BFFCE0197860022D3E810BDB0B2D09DA7868401E78606D1E057074
:20ADF0003889641EE4B2401C3881A7F84C403846BDE8F88FD4860100EC130020A08A0100DB
:20AE1000980E0020141500203212002046492DE9F0410A680646ADF1280D08A80260496885
:20AE30004160424C94F8B30006F12805002877D07078002874D1706E002871D0012102AA97
:20AE500005F0A0F800286BD19DF80800B073F06C38B1294605AA0DF11603F7F73DFF002865
:20AE70005ED10DF116000090706E294605AB01F073FE002854D12E48007801284DD04FF4CC
:20AE9000005006A908F076FD06A808A908220BF0FBF930B106A8294608220BF0F5F9002887
:20AEB0003BD194F85900002837D0A66CB4F8445042F2010004A908F05DFD049A4FF00041BE
:20AED0000020E2FB0610061C206D0CF08FF987190498B84202D86D1C3F1AADB2154E706890
:20AEF00080475FFA80F8206CB84204D1208FA84208BF002708D027642587002084F83500E8
:20AF10000BF0CEFA0127E064B168404688470FB106F000FA012084F85800002084F85900EA
:20AF30000AB0BDE8F081C046C08A0100E82D0020ED1300208C1400202DE9F84F0646307979
:20AF50008028D4BF0020E82071790027092901DB0A2900DDE820B179002975D0042973DA35
:20AF7000002871D1DFF8F48098F871000F286BD0B8F88A104FF6FF70884265D0B8F8841058
:20AF9000884261D0F079314C01280BD040B1FF285AD194F83B00002856D101252F4602E0E6
:20AFB000012500E00225DFF8A8A00AF12000834608F06AFC0AF1100008F066FC04F1200079
:20AFD00008F062FCDFF8989009F1040000688047204B84F83B500246FF21002060631D689D
:20AFF00084F83810002D0CBF0121011C012F84F83D10554684F83C7008BF032085F84000E3
:20B010004846816810468847B11DE820FEF748F9711DE720FEF744F9311DE120FEF740F934
:20B0300094F83D00012802D120200CF085F90A4898F871104FF47077A86207FA01F000F206
:20B05000636158460BF032FDBDE8F88FEC1700201C310020640E002075210100A811002096
:20B070008C1400202DE9FE4F0BF00AFA434C04F1080202901168E0604FF40050491C11605C
:20B09000694608F077FCDFF8FCA0DFF8FC9094F82F0000285FD0666B94F82D0000254FF0B0
:20B0B000FF0BA0462F4654E0B07F800821D3F07F08F04AFE0146082268460BF0E5F8C0B125
:20B0D000716802980CF027FB2D49814211D8F07FB7770AF009FA86F81FB0DAF8000080472D
:20B0F00094F82E3013B15B1E84F82E30D9F80810884798F82C006D1C2036ADB236E0F0780F
:20B11000800822D3307908F01FFE0146082268460BF0BAF8C8B13088010402980CF0FBFA57
:20B130001749814211D83079F7700AF0DDF986F804B0DAF80000804794F82F3013B15B1E20
:20B1500084F82F30D9F80810884798F82D006D1CADB2A842D3DC94F82E0048B1A046266BE4
:20B1700098F82C0000254FF0FF0B2F46A8429BDC04F1100007F0B0FFBDE8FE8FA42E0020F0
:20B1900000A493D6901400208C1400202DE9F04105466C78ADF1180D002C7CD14248B5F825
:20B1B00096100088884218BFE82405F18C0101A80F460BF003FD01A80AF094FE3B4B40B974
:20B1D00095F8990040B1A3F13800007820B9E82461E0002085F89900002C5CD195F8990029
:20B1F00000280CBF0120052004262E753946E8820DF10E000BF0E2FC686895F89840401ED8
:20B210006860411E6960B5F8968004702F7D69680024481C2862781E087028892C651A7886
:20B23000AC65801C288142B305F16C0005F18C010CF063FA1E4F85F86B60386810F47F0F8E
:20B250000CD085F82C60386805F12C01012200F47F0028632846FEF76FFA386810F0FF0F9B
:20B270000BD02A2085F83C00386805F13C0100F0FF002864284602F001FE0094284603210D
:20B290000DF10E024346F8F7EDFC041C02D1284602F080FF2CB16C701A202870284607F06D
:20B2B000BDFD06B0BDE8F0813212002024140020188701002DE9F04F0C4692468046994678
:20B2D00000213822ADF13C0D684605F056FD20686D4628606068686020892881207A03289C
:20B2F00004D0022003268DF80C0002E003268DF80C60374C207818B104F12C000BF0B4FFDF
:20B31000A08DADF80A0060781F28B4BF411C00210027B8F1050F617040F080000BD0B8F148
:20B33000040F05D0B8F1020F08BF40F0600004E040F0200001E040F040008DF80D00ADF848
:20B3500028A04FF0010BCDF8249022498DF80EB00A680BA802604968416005238DF8356088
:20B37000B8F1050F8DF83660B4F850008DF8343012D0B4F85600B8F1040F08D0B8F1020FCE
:20B390000ED1B4F85C00401CA4F85C0008E0401C80B2A4F8560003E0401C80B2A4F850009D
:20B3B0000D4918206A4604F00FFDC0B258B1B8F1050F09D1606A0AF0B7F9B4F85000401C61
:20B3D000A4F8500000E05F4638460FB0BDE8F08F901200205986010061650000F8B5071C53
:20B3F00000F08880B86840F6030120264A1C02E04068761EF6B260B15EB10388994218BF1C
:20B410009A42F5D1F9681CC820311CC149C881E849007868BA690025BD6138B397F827005D
:20B4300042F00202002300F00700401E09D0401E04D0801E08D14FF0805304E04FF08043D4
:20B4500001E04FF000532A4697F82700000908D397F8270010F0070F03D04FF080702A4324
:20B4700003437C68F868B7F92410A0470CF04EFA214C0646B4F92600401C6FF31F30E08426
:20B4900004F12000016881F827500BF09DFD30460CF038FAB4F92400B4F92610884229D17D
:20B4B000F86890F8BA0000280CBF0520072005F0A1F8F86890F8BA60BEB90668AEB1E2687D
:20B4D0000E4912680968B2F1FF3F13D0B6FBF1F2012A8CBFB6FBF1F1012170300CF0CAF938
:20B4F000F86870300CF0D6F9F8BD80F8BA50012008F060FEF8BDC046700A0020108B0100D2
:20B510002DE9F041414C0746206800287BD0DFF80081002F18BFE92F17D10AF081FF45469C
:20B53000297801EB81016918C1F8020095F8B560287800EB800029184E702878401C287070
:20B55000C0B20A28A4BF00202870324D68681C2F32D0314E4FB1F079032806D1E12F04D0B2
:20B57000002088F8B200072000E0052008F010FC2468F07903280ED06CB1002084F8690019
:20B59000E18A2648C90938BF2938007884F86A003846FDF74BFF98F85700012833D168689A
:20B5B0008047044606F03EFCA96820468847002088F85700BDE8F08180470646A96894F837
:20B5D0002F0002281ADA216804F124000BF028F894F82F00A968401C84F82F003046884739
:20B5F0002068007D252819BF012088F85600012088F8550000202060BDE8F0813046884729
:20B61000F120FDF713FFBDE8F081C046640E0020E82D00208C140020781600205A12002026
:20B630004549B0B5044601F13800007800287FD094F88B00002871D13520207504F18D01B6
:20B65000112204F16C000BF049FC04F13C00FF2110220CF078F804F12C000F2110220CF098
:20B6700072F894F88C0004F13C0500283ED0401E29D0401E14D0401E58D12A2028700227A1
:20B690002764042305F8103C4FF410222263032184F86B10204606F0C1FF071C3BD137E028
:20B6B0002A200A272870042327644FF44C1205F8103C02212263204684F86B1006F0AEFF23
:20B6D000071C28D124E02A2002272870042327644FF4102205F8103C01212263204684F836
:20B6F0006B1006F09BFF071C15D111E02A2002272870042327644FF4502205F8103C002159
:20B710002263204684F86B1006F088FF071C02D1204602F03FFD381C0BD1B0BD01280AD18F
:20B73000886C8047002808BF002002D0192000E018200BF00BFDB0BDEC1300202DE9F04F28
:20B7500009AF9A4616468846ADF1440D3C893D88D7F8049010900020AC428DF83C0001DAF1
:20B77000CA4501D30BF0A0FD002E6AD03748875D042EA4EB07044FF00000A4B2B8BF01207A
:20B790005FEA000B0EBF2D1BA1440024314807A90823ED1B2530ADB210F801295B1E01F873
:20B7B000012BF9D14FEA186001F8010B4FEA184301F8013B4FEA182201F8012B01F8018BE7
:20B7D0000E70234E109A30689DF83C104369706898478046B8F1FF3F24D00BA904910120D9
:20B7F0008DF801009DF83C308DF8023007AA01928DF800B08DF80370CDF80890CDF80CA0BC
:20B81000ADF816403168ADF81850022370680A6A8DF8143069469047804630688269706896
:20B830000FA99047B8F1000F18BFE4200AD147B14C4438460BA911F8012B401E04F8012B86
:20B85000F9D1002011B0BDE8F08FC046A48A0100043200203212002070B5ADF1380DFFF71C
:20B87000A3F93A4908682822082340F00200086001A800210CF01AF8354E3D4C3549B07890
:20B89000002301AA079004F1D4000CF00BF800213022082301A80CF011F830780025192118
:20B8B000ADF81C502C4A099001AB009504F158000CF000F82822082301A829460BF0F6FF59
:20B8D000F078264901AA2B46079004F584700BF0E9FF01A82946302208230BF0EFFF01205F
:20B8F0007278ADF81C001A2101AB099204F174001B4A00950BF0DEFF1A492A4604F1B00058
:20B9100013460BF0BFFF18480BF0B6FD2E46052384F8503004F1400181E860004FF6FF70AC
:20B93000A4F8AC00334684F8AF3023716371A371E371237263720D4A13704FF4FA76C4F858
:20B950004461C4F848610EB070BDC04600200940048B01004D6F0100796101003D0101000C
:20B970008D32010099570100A5E4000016320020700A00202DE9FC410746BE6833687D6835
:20B99000986B20F4FA609863AC6B44B13168886B40F4FA6088634FF0FF30BDE8FC81AA637D
:20B9B00029630024EC776C630CE09DF80000296B08706B6B286BAA6B401C2863581C686364
:20B9D000501EA863A86B90B93168886B40F4FA6088636A6B6878296B0128A1EB02012963F0
:20B9F00003D1EB68384698476A6B144646E005F14000694608F010FF0028D6D50BF086FF1F
:20BA1000204F8046387820B9022009F05DFE0120387040460BF076FF1B49086840F40070AB
:20BA300008603168886B40F4FA6088636878D8B9696805F1EC000BF051FF90B9AC630BF0C7
:20BA500065FF0646387818B1022009F025FE3C7030460BF057FF1027696B286BEF77401A9E
:20BA70002863686BBDE8FC8195F82D0030B1686B20B1AC6305F19C000BF0F8FE2046BDE85A
:20BA9000FC81C0461432002030100040F8B50BF035F9434E414F0446A00822D3B96901B379
:20BAB0003D460020A8618A69086906F108032040104340F0020088610A6918689043186058
:20BAD00001F1100090E80C0030681A1C9043306005F1200009F0BCFB022105F1D4000BF0F1
:20BAF00045FAB869A10815D200F110020CCA002122400B40002B08BF002A0BD00169856950
:20BB10000C40F8612C434FF48041846107F1D4000BF02CFAB86900283ED107F1140420465D
:20BB30000BF003FE051C37D0F868E96888422DD1A86806F015FC60B1012008F03BFB58BBCE
:20BB5000F86870300AF0ACFD07F1B0000BF0A2FEF8BD06F1080128690A68104308603268E2
:20BB700005F1100393E80300081C1043306000233361A86846F80C0C06F110000068002873
:20BB9000FAD020460BF020FABD61F8BD07F1D4004FF480610BF0EAF9F8BDC046700A00205A
:20BBB0000C1004402DE9F8438146D9F808703868066CD9F8045046646A6CAB6CA86B16F4C9
:20BBD000F06F0146A2EB03082AD1F00911D270095DD301B395F83C40641EA14298BF0C1CF6
:20BBF0004846214609F0DAF9A86B001BA8630DD04DE081B1484609F0D1F995F82D10A863D9
:20BC100011B9002843D101E00020A86305F19C000BF02CFE3BE04846414609F015FE36E0F9
:20BC3000F20A19D24FF00008444602E0A86B401EA86340B34846012109F0B0F9386844684D
:20BC500014F00F04C0F80480F0D0286B401E2863686B401E686316E038684468002220299C
:20BC700004F00F044260CCBF20270F1C4846394609F094F9C7F12007B845C8BFB84648468C
:20BC9000414609F0E1FDEC77484606F09BF9B0090BD3A96A49B10F46484609F0B7F9A86281
:20BCB00018B94846391D07F017FEBDE8F88370472DE9F04105463E4804780F46002DADF128
:20BCD000280D42D03B48466A002F3ED08046D6B17069C0B10123ADF8223006208DF8200020
:20BCF00029460C2200236846ADF8243003F0D8FC03A839460E2203F0D3FC766908A803C890
:20BD10001A226B46B047787B012668B9002C14BF0FA013A06988102207F0F2FF397B13A021
:20BD30000A2207F0EDFF08E0002C14BF12A017A00BF052FA19A00BF04FFA88F8026000204E
:20BD5000314606F03BF888F803600AB0BDE8F0815265737461727465643A20307800C046CA
:20BD7000537461727465643A203078004368616E6E656C3A2000C0464465766963652052FF
:20BD9000657374617274656400C046C0446576696365205374617274656400C046726571DC
:20BDB00075656E637920486F7070696E6700C04690120020A41000202DE9F8433E4C81461C
:20BDD000A07830F0010708D0042806D0032804D0052802D00BF068FAA078384E257904217D
:20BDF0000528324FDFF8C880317005F10101CDB225711CD1022D53DC3F68B9F1010F4FD0ED
:20BE10007868398904F038FC78680088000905D34146087810B108F087FE257928460BF0B3
:20BE30009AFC8320307009F06FFDBDE8F883DFF8849099F88810A94232DB032830D007F066
:20BE50007DFEA078042809D14146383991F8380020B1D1F8841009B102208847E07899F8BE
:20BE70009510421C9142C4BF401CC1B2E1703D682989686804F000FC68680088000904D3EA
:20BE90004146087808B108F04FFEFEF7F1FDA078042808D08320307008F076F8BDE8F883C5
:20BEB000E12004F021FBBDE8F883C046640E002024140020A8110020C4180020203200200A
:20BED0002DE9F0430746ADF11C0D0BF0CBFC09F06BFB4FF000090646CDF80C900BF056FB93
:20BEF00030F0010002D00398B04202D16FF0040066E078684C4658B1B0F1FF3F05D004A95A
:20BF100009F03AFB30B1804659E04FF0FF3000E0204604900BF0A2FC049D4FF001082D18F4
:20BF300002E00A463BE00493706804990BF0D6FC00282DD0684607F0F9F8D8B99DF80400E6
:20BF500005A909F0B5F888B9BB68BDF814009DF80610029A984748B1BDF814009DF806507D
:20BF7000B881029BBD73C8463B6111E0029903A809F06AFD0498641CB0F1FF3FD4D00028A3
:20BF9000D2D00BF06BFC2B1A02D004989842CAD2039F0AF0DFFD06F1080547B13A4652F826
:20BFB0000C1C0029BDD1296842F80C1C2F600AF0F5FF24B170680BF08DFC641EFAD140461E
:20BFD00007B0BDE8F08370472DE9F04F044609AF3D4D78681E46ADF1140DEB880290B7F833
:20BFF0000090A08988469246411D89B20391C918B1F5805F63DCE288217A971001F03F0123
:20C010008DF80010A1888DF801701B1802F00302C1F3051747EA821709078DF80270C0F3DE
:20C03000831200F03F0742EA11628DF803204046B9008DF804106A4699B28B4608F00EF83C
:20C05000029820B3EF885EB13A4640465146334607F002FBF01906EB0A0387B21FFA83FAFD
:20C07000029B40464A46394605F0B0FAA689E98809EB070087B2F01B09188AB23AB109EBC4
:20C090000A00134681B23A46404607F0E5FA9DF800204046594622F040028DF800200BF050
:20C0B0002BF9EA880BF10401404689B20BF004FBFF2806D00398801880B2E88001E005204E
:20C0D000687105B0BDE8F08F441A002070B53F4C0646A07EADF1200DF0B994F85C00822800
:20C0F0001AD0394B40F2016046F25C05ADF8080034491868ADF80A50426A086802A990474F
:20C11000012814BF6FF07F009DF90C0009F09BFF94F85C10226B505494F85C00822814BF72
:20C13000401C002004F1180584F85C0094F85C0005EBE00292F82C00411082F82C104008CA
:20C1500007D294F85C00401C84F85C00C0B28128ECDB94F85C0081282CDA05F14401E12025
:20C17000FDF79EF802204FF6FF738DF81800A17EADF8103031F0020018D0012919BF072077
:20C1900083210820802100224935009204AA0195FBF7D6FADB2807D0E52805D0F32803D040
:20C1B000DF2818BFE8280AD1607603E0304604F049FF04E02A203070304606F02FFE08B01C
:20C1D00070BDC0469019002048160020B03000202DE9F84F0E463A494FF000088346642706
:20C1F00044468A464D6B91F82D0086F81E80D1460AE099F800106D1C2034ADB231E099F8CB
:20C210002D00641C6D1DA4B2A04217DDE8780028F5D0287907F098FD594608220AF034F842
:20C230000028ECD1E878B077288800047060287986F80B80F077A87847463073DAF830405B
:20C25000002F39D086F81E8042F21900694607F091FB0AF015F982461A480178642745463A
:20C270008146A94228DDA07F0028C2D0E07F07F06BFD594608220AF007F80028B9D1E07A92
:20C29000022803D0E07A58B1612710E0616850460BF041FABDF800200B495143814201D9C7
:20C2B000474604E0A07F6C2740F00800A07730462146202203F0F4F93846BDE8F88FC0464D
:20C2D000A42E0020D02E0020808D5B002DE9F04707467D68D7F8089090460E460BF016FBBA
:20C2F0008246A86A002864D105F584700AF0D8F90024EC772E6250466C620BF003FB0BF0CF
:20C3100005FB2F4E3378824623B9022009F0DCF90120307050460BF0F5FA2A49086840F4F9
:20C33000807008603846414608F070FEA862C0B93846414607F0D0FAA878D0B9A96805F131
:20C35000D0000BF0CBFAE8B9AC621020E8774946284604F067FF0BF0D9FA8246307840B377
:20C3700023E0D9F80010886B40F020008863A87810B12046BDE8F087A96805F1D0000BF066
:20C39000ADFA10B1686ABDE8F0873846414607F0A3FA1020AC624946E877284604F042FFCF
:20C3B0000BF0B4FA8246307818B1022009F074F9347050460BF0A6FA4FF0FF30BDE8F087A4
:20C3D00015320020301000402DE9F043DFF8E0808946054617464FF0FF31ADF13C0D404693
:20C3F0000BF07CFA334C04EBC504666825680BF08DFA2168096800290BD42968002905DC0B
:20C41000B9F1000F09D04FF0FF3108E0B9F1000F03D00BF077FA002442E02968491C296066
:20C430000BF070FA286802283ADA1FB90DA80BF0FDF80DAF38686860B7680021302208235B
:20C4500001A80BF03BFA4FF00009069401AB307B194A09903946CDF8009005F12C000BF0CD
:20C4700029FA01A82422082349460BF02FFA012705F1640001AA8DF81C7049460BF022FAD8
:20C4900005F1480001AA39460BF01CFA706801F01FFE0A4A05F118002346042109F0BEFC8A
:20C4B00040460BF017FA20460FB0BDE8F083C046CC310020708A01007D6001006D760100BD
:20C4D0002DE9F04106AF3D793E68984604460B1CADF1180D074611D0012B15D1307973790D
:20C4F000641C3870B17904F8013B337A04F8011BB17A04F8013B7389181201E031787078E2
:20C5100004F8011B04F8010B8AB9002D0CBF42F20C0042F20D00694607F02CFA9DF80000CE
:20C53000BDF8003004F8010B181204F8010BB8F1010F34D0B8F1020F39D1002D0CBF42F21F
:20C55000020042F203000DF1020107F013FA7589CDB1681E01468B100DF1020201EB5371F7
:20C57000C910CBB2811000EB517121F00701401AC0B20121401C01FA00F0D15CFF3080F0FD
:20C59000FF000843D054E81D0DF10201C210204603F086F87089C01D04EBE00407E0002DB1
:20C5B00014BF02210121204602F0ACFB0419E41B06B0A0B2BDE8F0812DE9F04390460A6889
:20C5D000D8F800401678814600271D463846ADF1140D531C242E0B6053D112F8016F5B1CDE
:20C5F0004C2E0B600ED1AA68E41C24F00304241D54F8040C494606F05FFB2968EF600127B6
:20C61000091A2960462E1AD1E41C24F00304241D54F8040CE41C029024F00304241D54F80D
:20C63000040C002749460390AA68ADF8047001A803F084F82968EF600127091A2960532E19
:20C650001FD1E41C24F00304241D54F8040CE861C8F80040288B0090A968EA69D9F8000061
:20C670004346F7F751FED9F80040002714B10119C9F80010D8F800402968EF60091A0127C1
:20C690002960662E0AD12B8B23B9E41D24F00704083403E0E41C24F00304241D1FB9E9693B
:20C6B0000E700127EF60C8F8004005B0BDE8F0832C4870B50568B5F1FF3F08BF00250AF0D8
:20C6D000CFF801284DD107F047FF142849DB26482649002601230660254A0B60254C136054
:20C6F00020680028FCD1264A131D2349186820F00300014321480068C0080CD2106810F0DB
:20C71000030F0AD041F003001860106800F003000328FAD101E041F001011A4819600068B9
:20C7300020B1194800682846F5F720FE174818490660184D0A686FF35B4245EA0200086042
:20C7500015490868C0F30130012806D10A681348104040F400320A60086020680028FCD145
:20C7700070BDFEE71C130050840460425C600C40082204430C00684204000020B03F00505C
:20C790000040034080012843000120438C210840482003400000390104000940FFFFFCFC99
:20C7B0002DE9F041374D044668781F4616468846ADF1380D012803D0FFF74EF801206870D1
:20C7D000B8F1000F0AD0C4F804803EB1A6600BF09DF8A978022903DB0BF094F800204DE0F4
:20C7F00005EB8102491CC2F83C41C9B2A9700BF089F801251FB909A80AF04EFC09AF3868BF
:20C8100020607868E060387C2074B86865746061788A6082F86800B1A0610021A02204F198
:20C83000200004F0AAFA68460021242208230BF04DF88DF8185004F1380000216A460BF0CA
:20C8500041F868460021242208230BF01FF80E49069404F1700000226B460BF013F8684660
:20C870000021242208230BF011F80849069404F1940000226B460BF005F820460EB0BDE80A
:20C89000F081C046700A0020F9690100E17601002DE9F04F09AF3C897D6816464FF0000A60
:20C8B0000246002EADF1440DA04610933C888DF83CA05CD0304810F80690042E03DAA8EB71
:20C8D0000900C8462D18F868A4EB080407AB0827A4B2C01D10F801C97F1E03F801CBF9D1DD
:20C8F000080E264F03F8010B080C03F8010B080A03F8010B386803F8011B9DF83C101E703C
:20C910004369786898478346BBF1FF3F2AD0042E04DA03208DF80000022002E002208DF88C
:20C9300000008DF8140002959DF83C608DF8026001218DF8011038688DF8039007ABADF8D8
:20C9500016800BADADF81840026A0193109E04956946786803969047834638688269786802
:20C970000FA99047BBF1000F18BFE42000D1504611B0BDE8F08FC046A48A010004320020AB
:20C990003A4834492DE9F047012500240570DFF8C880DFF8CC900C70304901F16A06378814
:20C9B00082460220104004EA0306002E08BF002810D14FF0E04720461F401040002F08BFC7
:20C9D000002832D0424692F90000401E10700AF061FA2AE0424692F90000401E1070BFB964
:20C9F0004A8E43F2084320464646934204D191F84010090938BF281CFFF7DEF9484604703E
:20CA100096F90000F0B196F90000002817DD1DE0B7F5505F07D114481249006800F5C070B7
:20CA3000086002F06DFA0AF011FA48464246047092F9000030B192F90000002806DC0AF09B
:20CA500033FC03E020460146FBF754F88AF80040BDE8F087CC1A0020CD1A0020280D002089
:20CA7000CB1A0020401600200C010021E41A00202DE9F84F07463248DFF8C89000EB470654
:20CA9000183699F83800348890468B46B8B1D9F85010A1B12C4D05EB8705686B00F0FF0069
:20CAB00088478246D9F85010686B00F47F008847504480B218B131884018001D84B2254829
:20CAD0001230007801280CD198F808604EB11F4898F8093081190D79C05C2418641DA4B210
:20CAF00000E00025281980B209F0BCFB0646184890F80090D6B13046002122460AF023FE99
:20CB10004FF00008A41937700D4986F8018006F180007460CA5D358159460AF0DFF94846DE
:20CB3000314605F09DFE4046BDE8F88F8DF8007068461A2103F092F91A20BDE8F88FC04664
:20CB500014830100EC130020D4860100A08A010014150020321200202DE9F04F364E0025DD
:20CB7000ADF1340D07464FF0010AA846A9460C93DDF858B00B914AE017F8020FAD1CADB2C8
:20CB9000401E1BD0401E09D0401E04D0401E36D1022C34D138E0032C31D135E0072C2ED1AB
:20CBB000B9787878FB1C40EA0120A6F84400186806F14802106086F859A025E0052C1ED133
:20CBD000CDF80890B91C0A8802A80280897881700B9803A9FFF7FCFA9DF82A00A0B1029B7B
:20CBF00040F0020000F0F7008DF82A0006F1500203931068049003A805F01CFB04E008EBE4
:20CC10000400801C1FFA80F8E7196419A5B23846694608F0EDFB041CAED1022D03DC4D46B2
:20CC30006720A84600E048460C990D800DB0ABF80080BDE8F08FC046E82D00207CB5354CDE
:20CC5000054694F871000F285ED03348697E0078890959D2297E002841F00201297639D0D5
:20CC700069684A1C1078801010F0030F32D000F0030002280ED1B4F884304FF6FE70984258
:20CC900008DD56791179002001EB0621994208BF012004E004F17A00491D09F04DFFC8B9D1
:20CCB000687E696840F0010068764A78C2F38102022A2DD1491D4A7809784FF6FF7601EB2B
:20CCD00002218E4224D1297E00F0EF0041F0200129761CE0687E114E40F0030068763078EB
:20CCF000B0B994F8A7008DF80000FF238DF8033094F8B6608DF8016094F8B7508DF8025037
:20CD100068460AF09BFC7CBD687E40F0010068767CBDC046A8110020EC1300202718002000
:20CD30002DE9F04F9246ADF11C0D0493071C039114BF5FEA0100EB205FD000200446CAF81E
:20CD50000000A146CDF8149078783D7845EA00255FEAE5380CBFC5F30626C5F3C326049828
:20CD7000BF1C20B1B8F1000F39D00F2E44D0082004232349ADF800000C22ADF8023001F18E
:20CD90002400016801926846884700280CBF02980598834608B305990C2203F0EEFFDAF8BA
:20CDB000003003B95446C4F800B05C4684F8048066712679002E0CBF05F0FF05C5F30A05A0
:20CDD000E580A760039EE08809EB0001C719891C1FFA81F94E45B7DC0EE01A2000E018205B
:20CDF0000590DAF8000038B1046809F0E9FA201CFAD10020CAF80000059807B0BDE8F08F2A
:20CE10008C14002070B50546344C2878ADF1200D00284FD1208F04F148066B88ADF8000015
:20CE30003146ADF81030E2200AF016FA0DF1120031460AF0E7FB6988532009F0F3FE208F1A
:20CE500004F13E063146ADF80E004A200AF004FA01A831460AF0D6FB00268DF80D60A08FCB
:20CE7000ADF8020094F83A308DF80C30304608F073FC5220314609F0C9FE94F850000F28AB
:20CE90001CBF01206070E06828B102681AB10DF10E0069469047032008F090FA94F852004B
:20CEB000032818BF042813D104F10800102109F08DFD0DE0002060700AF07AF941F288306A
:20CED00008F04AFC0649B1F84E00401CA1F84E00216E09B12846884708B070BD4813002095
:20CEF000901200202DE9F0470D4606465FFA85FA280824BF2E4845402E494FEA8A03C85831
:20CF100085EA00023240C2F300672B4A06EA0504B043224006F4E0240243B4F5E02F01D172
:20CF3000500E14D306F4E020074310D002F4E027B7F5A02707D0B7F5803704BF22F40032C3
:20CF500042F4A02203E022F4803242F4C022DFF86C80CA5008F1D00739680122002002FA79
:20CF70000AF40C4218BF101C5FEA000906D1F00D04D34146C5F3805001F80A00300E0BD327
:20CF90000AF0C4FC290E34BF0021211C3A68A243114339600AF0B6FCB9F1000F06D0F00D93
:20CFB00004D34046C5F3805100F80A10BDE8F087006000A000100840007F077F002002408E
:20CFD0002DE9F04117460D460AF0A0FC324C8046207800266DB16D1E04D06D1E55D0681EFF
:20CFF00011D00EE0B4F8AC004FF6FF71814202D005E0A06908B9802648E0A069808C388066
:20D0100044E0842642E0386831465022054603F0B4FE022704F59E7C04F5A672A5F11001A3
:20D030005CF8040B41F8100F137A0B735068486052F80C3B7F1E18448860F1D1A069002855
:20D0500008BF02200ED0A069C068A769286297F82600A36985F82C00D869A2696862106A34
:20D07000A862032067698FB105280FDAFA6801016A5097F826204C192273FA6962603A6A97
:20D09000A2603F68401C40B2EDE7387040460AF039FC3046BDE8F081700A00202DE9BE411D
:20D0B0000546DFF8CC802978B8F86000E1292FD0B8F86200E92926D0B8F86400D9B92D4CFF
:20D0D0002869676A02903FB37F692FB3A16A1931814221D806208DF800000422ADF80220E7
:20D0F0000023ADF804309DE8030002ABB84708B90298A06210E0401C80B2A8F8640019A058
:20D110000AF0DDFA08E0401C80B2A8F8620003E0401C80B2A8F86000687830F07F071ED0D1
:20D1300000F06001402906D12F7827B9B8F85210491CA8F8521000F06001202906D128783D
:20D1500020B9B8F85800401CA8F85800602906D1287820B9B8F85E00401CA8F85E00BDE8A4
:20D17000BE81C04664617461436E663A2000C04690120020A41000202DE9FC47314CA11C20
:20D190000888401C088009F07BF90026B046354681462846694604F0F7F88246BAF1FF0FBF
:20D1B0004CD09DF80030206B23B900EB4A104068010402E000EB4A10416848460AF0ABFA28
:20D1D000864203D29DF800700646D0466D1C0A2DDFDB1E4D281D0068804794F82F106FB9EF
:20D1F000626B08EB88030026FF27491ED218D67013791771C9B284F82F100CE0216B00220D
:20D21000FF2701EB48118A77CB7FCF7794F82E10491E84F82E100C4A643BD9B2136804EB2D
:20D23000C10138310B6052684A6094F88810491E84F88810A9688847BDE8FC870AF069FAE0
:20D25000BDE8FC87A42E0020D08A01008C140020E0B501880025A1F6020159B143F2040267
:20D27000891A04D0491E57D190F8246000E00226C76901E0C67B4769002F4DD03F1F0520B3
:20D2900044F2380357F8041F0A04120C934203D0401EF7D13F1D01E0C1F30345002D3BD030
:20D2B0001F4B3046401F18D01C4A401E10D0001F0CD0801E0DD0C01E06D00F3819BF1A1C14
:20D2D0006032184A443204E0121D02E0121F00E0083A1068C0F3834003E01A461068C0F330
:20D2F00003200F2806D0A84216D921F4702141EA004110E0761F0AD0761F08D0761F06D0CC
:20D310000F3E1CBF21F4702141F4802103D121F4002141F4E0213960E0BDC046001100507C
:20D3300020130050C4100050F0B5064600210B22ADF1240D0DF119000AF005FA2E4F2F4C20
:20D350003078C01E14D0801E04D0143810D0801F01282DD801208DF8180006F18B0103A8FC
:20D370000AF0CBF9032538788DF8145068B112E000208DF8180006F18B0103A80AF0BDF978
:20D39000032538788DF8145028B9B4F88E000225ADF8020005E00DF1020004F1A8010AF056
:20D3B000ACF98DF80A50B4F88A00ADF8160017E002208DF8180006F1320103A809F0EEFE78
:20D3D0000DF1020006F1280109F0E8FE8A34208806F11C01ADF816000DF119000AF08AF975
:20D3F0000B208DF8000077788DF80170684600F045F909B0F0BDC04624140020A81100200F
:20D410002DE9F84F8A463149044601F1B400007828B920465146F8F73DF8BDE8F88F0A2590
:20D43000884642F2107B20465146F8F733F898F8B410002848D19AF80060D4F8009000292C
:20D4500037D023480168C88AC20832D280094FF0000702D3087D15282BD008F0F1FF98F8E8
:20D4700000308446002B0EBF09235B1EDBB20A2003EB830208EB0201491C0A78964207D04F
:20D49000002B0EBF09235B1EDBB2401EF0D110E0D1F8011060460AF03EF9642101FB090107
:20D4B0008B4505D942F242706426401AB0FBF6F717B90020BDE8F88F20686D1E074427604B
:20D4D000B1D10AF026F96120BDE8F88FE82D0020640E002080B50288A2F602073FB143F2A8
:20D4F0000502BF1A14BF002090F8240000E0C07B2C4AD2F88832401F0B6048D0401E3CD03C
:20D51000001F30D0801E24D0C01E18D00F380CD0D2F890024860D2F894028860D2F8BC028D
:20D5300020F0784040F080503AE050694860D06A8860506C20F0784040F0704030E0106989
:20D550004860906A8860106C20F0784040F0F04026E0D0684860506A8860D06B20F0784002
:20D5700040F0C0401CE090684860106A8860906B20F0784040F0A04012E050684860D0690F
:20D590008860506B20F0784040F0405008E01068486090698860106B20F0784040F0205084
:20D5B000C86080BDC41000502DE9FC41274A28491778002F41D02C48077837F07F073CD121
:20D5D000244C488C94F87470234E284B401C0025488407F0F00084F874000120307019782D
:20D5F000256704F16807012902D02946FAF782FA0AF07DF81E4E301D006880472A468046C6
:20D610001C4DA4F86A20286A144B84681A4802218DE806000C3000683946A0471049002803
:20D63000088005D40F4991F90000EF60401C0870B16840468847BDE8FC81888C401C888468
:20D650000020107009F008FABDE8FC811E320020C4180020280D0020CB1A00201D09010010
:20D6700094180020CD1A002020320020E41A00208C140020281600208419002070B50646EB
:20D69000304930780D5C401F1CD0083851D0401F4FD0284608F0E6FD041C0DD130780C28A3
:20D6B00008D1706830B1301D07F056F8284608F0D9FD0446002C43D02A462046314609F02B
:20D6D0000DFC37E0B07810BB327A307C51005410401901F00E01091804F0380040182430C8
:20D6F000C0B208F0BFFD041C2AD03146182209F0F5FB04F1180060607168242209F0EEFB72
:20D710006068243060617169327C0E46D6E7012816D12435E8B208F0A5FD041C10D031466F
:20D73000182209F0DBFB04F11800606071682422EBE7344624B104480078214605F090F81B
:20D7500070BDC046488A0100381A0020F8B509F0BDFE04F09BFB09F0D1FE044604F00C0044
:20D770000C284BD0E0081ED208F08CFA264E376805460120014608F0F0FF31686943884238
:20D7900011D2224C8220B0FBF7F0291A20460AF071F820460AF07EF80120F8F7AFFC2046F1
:20D7B00008F07EFF2CE0200928D2194809F03BFE0428FAD0174A610905D220B111681046EA
:20D7D00021F0010103E01046016841F001010160983210684FF0805540F003001060D5F82A
:20D7F000B8018169202088470B4CD5F8B8712068B86B804701202060206801E009F085FF21
:20D8100009F06AFEF8BDC046108B0100A00F0020004003408C2108402C2009402DE9FF410E
:20D830002E482D4F00683E78C06B80477968401AB100B0FBF1F4B868FF680025A846414639
:20D85000BC4271EB080101DAB84206D82946424684428A413CDA074600E029463846324672
:20D87000F317001BA94109F05DFB272704464FF47A7200230D46ADF802700820ADF8000017
:20D890002046F8F777FF01901548016868468847029843464FF0000100F6FC02A41A9D41E6
:20D8B0006042A94111DA0F48026829462046F8F761FF0D4604464FF000016042A94104DAB5
:20D8D000204606F029FE002000E00120064908700090BDE8FF81C046C81900204816002093
:20D8F000B0140020801800201F3200202DE9F84F2E4C012683461D4690468946C4F87C679D
:20D910000320C4F880670AAFC4F88407D4F88C0710F0030FFAD1387A58B14FF0805ADAF84F
:20D93000B001016A27208847DAF8B0010169272088470220C4F8FC063868C4F808043046E4
:20D9500009F0B7FED4F808040008F8D2D4F88C07800F28BF301C26D22868C4F83C056868E9
:20D97000C4F84005A868C4F84405E8681049C4F848053879002814BF081D081CC4F84C05CD
:20D99000C4F850850020C4F85405C4F8580509490E60C4F800B0C4F80880C1F80064C4F84F
:20D9B0002090C4F82880BDE8F88FC0460440024028000020000048422DE9F843044609F025
:20D9D000A5FF81462B48021992F8ED10491ECFB2002F82F8ED7046D1294901EB840425782F
:20D9F000618835F07F07884618D1E9090FD24FF0805000F5DC76D0F8B801816940468847E3
:20DA10003068416B404688470228F9D11EE000EB8800D0F800110020884717E04FF0805624
:20DA3000D6F8B801016A40468847D6F8B801816A40468847D6F8B801016B404688470E4929
:20DA5000012008600D4908688008FCD305F03F003F2801D0FFF7B0FF607800F03F003F2891
:20DA700001D0FFF7A9FF484609F04CFF0020BDE8F883C046940F002028200860282008400C
:20DA900014880100F8B5314D6868804706462D4CA9682068002852D160698047676A40F0DD
:20DAB0001000002F4AD00022797E0140884205D03A4657F80C7C002FF6D13FE004F124007F
:20DAD000394607F04FF8002F38D02760787E30F07F0005D194F82F00401E84F82F0004E0A8
:20DAF00094F82E00401E84F82E00A9683046884723681889D98A08F032FCA0851248007852
:20DB100008F068F8D98A090A0FD2407B012803D0022816D1052005E0187E401080F001001D
:20DB300000F00100FAF7D0F8F8BDD87E05F084FE206890F91C0009F0F5FAF8BDA968304658
:20DB50008847F8BD640E00205F1200208C140020F0B506460F4600251446ADF1240D8B200F
:20DB70000DF10E010095FCF7EFFA8A2001A9FCF7EBFA707A00282ED1387AA0B9BDF80E10FC
:20DB90004FF6FE70884205DCBDF80E10884220D101A90DE020489DF80E700488BDF80E0028
:20DBB0008DF812700CE0022807D0032811D1394604A809F0A2FD09240BE038888DF8120022
:20DBD0008DF81040211200128DF8111005248DF81300284611E002280CBF052409240128E1
:20DBF00018BF311C04D1892007A9FCF7ADFA07A9224604A809F072F9B07A04EB0D01C8739F
:20DC10006A4604A8214603F049FB002814BF281C009809B0F0BDC046321200202DE9F0410C
:20DC3000294D012001462870F9F764FF27496FF0010008702B480068C06B8047244C074639
:20DC500021786068A2688B003E1AB6FBF3F05843361A88001F4902FB03F8B1FBF0F09042A1
:20DC700001D209F021FBB91B1B486160414400F03BF81A4CA06867682168404207F050FB82
:20DC9000002F08BFA16808D0A16878688142DCBF401A78603F68002FF7D1E068884202D0A2
:20DCB000A06005F071FF02F097FB0D4C606880470646FFF7B3FDA1683046884708F0E8FE65
:20DCD00000202870BDE8F081E41A0020C81A0020C8190020FFF6C2FF2DDC0000241A002028
:20DCF0008C140020481600202DE9FE4F294D814668680091804729F00106274CDFF89CB058
:20DD1000DFF89CA0274FDFF8A480274D019024F00104B44212D02BF00100B0421CD15146E7
:20DD300091F9000010F1020F18D02868826B91F900103868904701280ED10FE0414691F9B9
:20DD5000000010F1020F09D02868826B91F9001038689047012801D009F0A6FA2868C56AE8
:20DD70001349009A38684B46A847051C01D509F09BFAB44206D02BF00100B04204BF5146C4
:20DD90000D7001E041460D700249019889688847BDE8FE8F8C1400202DDC000015F6000067
:20DDB000C91A00209019002048160020C81A0020280D00202DE9F04F0446B4F80AB0A08984
:20DDD00098460B46ADF1240DABEB00010690ABEB0000181885B228481FFA81FA8178914637
:20DDF000164642460027079101E00127521C3046411E8EB268B9002F08BF002039D0012F74
:20DE100012D10798534499B24A46434603F0DEFB2DE02946481C85B2079809F04DFC117828
:20DE30004840E3D00842E0D01348069FC188781D80B24018B0F5805F0DDD0294ADF80CA0E0
:20DE5000ADF80E30ADF810900798CDF8148002A9F9F7A2F80BE0CDF80090CDF80480079934
:20DE700020465246FEF7B0F8584608F047F90248407909B0BDE8F08F441A00202DE9F84F66
:20DE900007460E1C14BF4FF000094FF0E809002F4FD0B9F1000F4ED17868401E78603F2114
:20DEB0000170BD6D002D0CBF802000207968DFF890A00224083E491E7960DFF880B00870EC
:20DED0003889A7F85440801C388116F8080FFF282CD02A2828D1706830B35546296D88479B
:20DEF000804678689BF80020A0EB08007860716829B96D6D3A460023A84748B10BE06D6D69
:20DF1000786871688DF800206B463A46A84710B9EB20BDE8F88F3889B7F854504044388122
:20DF300008EB0500A7F85400641ECED17868386501E04FF0E8094846BDE8F88F88310020A4
:20DF5000EC130020F0B52F4C0546A07EADF13C0D022806D0012804D005281CBFE82060763F
:20DF700049D194F8600000284AD1002109A81822617609F0E8FBCDF828D009A8294600F0BC
:20DF90005BFC94F82E0094F85810814220DD266B70B10746BDF80A007189884204D13046DF
:20DFB000694607F059FE98B97F1E06F12406F1D194F82E00276B8100242201EB40117818A3
:20DFD000694608F08BFF94F82E00401C84F82E000D48007828B19DF8340010B994F8580024
:20DFF00028B909A8FFF74AFB94F8580040B194F82E10884204D12A202870284604F00EFFB5
:20E010000FB0F0BDB03000200E1200202DE9B841804607F0DFFFC01DC51098F8230000280D
:20E0300049D198F87E4007F0D5FFA04243DD264A1368E010191891F86C1004F00704214129
:20E05000CFB207E0401CC0B21918C40091F86C7088F87E4047B9691E8142F3DC1068002130
:20E0700088F87E10417029E098F97E10C0000830884226DD401A79080BD298F87E10401EB0
:20E090004FEA670701F1010188F87E10F3D1BDE8B88198F87E000D49087098F87E0088F8BB
:20E0B000810098F87E00401C88F87E000320F9F70BFEBDE8B881002088F87E00072005F033
:20E0D00067FEBDE8B881C046640E002084190020F8B5064609F01AFC2A4D0746A91991F881
:20E0F000ED00421C002881F8ED2045D1264C04EB8604267806F03F003F2801D0FFF7E8FF2E
:20E11000607800F03F003F2801D0FFF7E1FF648836F07F0018D1F0090FD24FF0805000F582
:20E13000DC75D0F8B8014169204688472868416B204688470128F9D11EE005EB8405D5F876
:20E1500000110120884717E04FF08055D5F8B801C16920468847D5F8B801416A2046884758
:20E17000D5F8B801C16A20468847084901200860074908688008FCD3384609F0C3FB002063
:20E19000F8BDC046940F00201488010028200860282008402DE9F041054608F0A5FF287E40
:20E1B000000904D2287D012808BF022700D00527DFF89C80464670688047264C04F124010C
:20E1D0000B68002B08BF0D600CD07F1E0026FFB202E07F1E1346FFB253F80C2C22B92FB146
:20E1F00043F80C5C012601E0002FF2D1D8F8081088471EB3216928468847E88AA168C008E0
:20E2100018D2D8F80400804794F82F10491C84F82F10D8F8081088470C4991F8380028B1D8
:20E230000846C06C10B18047BDE8F081FFF72AFCBDE8F08128468847BDE8F081F120687048
:20E25000284603F04FFDBDE8F081C046EC1300208C140020640E002070B5214E002086F842
:20E270005400032186F85500E82008F0E7FC5220012108F0CBFC1B4D482205F1700406F1DA
:20E290005C00214601F00CFA17486867343CF4601648C5F880001648C5F888001548E867D8
:20E2B0001548C5F8AC001548C5F890001448174CC5F8A00013481649C5F89400124847F224
:20E2D0003052A86704F1980005F0F2FD4EF660221049A06104F1BC0005F0EAFDE06170BD11
:20E2F000481300209012002015CE0000750E01001D0A0100954E0100ED5100008D0C010086
:20E31000CD1A01001DE60000C9570100A4100020F56A0100516601001A481B4901641B4966
:20E3300041641B4981641B49C1641B490165022280F8202019494165194981651949C165D8
:20E350001949016619494166194981661949C166194901671949416719490160194941606F
:20E37000194981601949C16019490161002180F83C1080F83F101749C161C162012180F818
:20E39000301070473830002091730000E1320100513F010059370100D5230100CD4E01009F
:20E3B000C1610100D5420100852E0100E9460100FD6D01000D07010019430100856A010061
:20E3D00029730100B165010011FC0000392401004B77010059730100F0B52B4D05F12C013E
:20E3F00058C9ADF11C0D02AA58C20AC94FF0805682E80A0047688468D6F8D001C168206818
:20E410008847216821488A6B10408863206840F2F271416497F83C0097F83D10C0100DEBCA
:20E4300080008068084321684863684609F012FAD6F8D001397F466805EB8101BA698B68A5
:20E45000797F206855F821101943BB7F05EB8305AB690B430199B0470D490A1F106840F086
:20E4700010001060086840F001000860A07D0027FF2802D0E07DFF2800D11FB1086840F4FD
:20E490004040086007B0F0BDA88801000DF8FFFF30100040042998B54AD108F0E9FD254C88
:20E4B00004F1400282E8030004F1140009F03DF900280EBFE068C068E06041681E4A097839
:20E4D0001160416812680978914207D087692FB16FF0FF0100224FF00073B847022007F052
:20E4F000F3F81120FFF7F4FD01206071E168087C10B12079012803D00E20FFF7E9FDE168A1
:20E5100049680E488F680FB9CF681FB10021C1610B4F07600B4A40F2FF71116000278761A3
:20E5300009494161094808F0A7FF192009F08EF998BDC046700A0020D021084000100440AD
:20E550005100070600000460020000402191000029482DE9B0410025DFF8A080294C057077
:20E57000ADF1140D88F83B50012088F83800201D006888F83D508047234924310F686FB117
:20E59000797E8A0806D341F001017976397E01F0FD01397657F80C7C002FF1D1A1688847F2
:20E5B000102008F0D1FE082008F0CEFE98F83C00E0B90920124C8DF80000B4F88A108DF82C
:20E5D0000F50E027ADF8021094F8A7308DF8017094F8B6208DF8043094F8B7108DF805209D
:20E5F00068468DF80610FFF749F801E088F83C5005B0BDE8B081C046EC130020EC170020CB
:20E61000A81100208C140020640E002070B505462B4C2878ADF1200DEB2829D040B3E9285D
:20E6300006D0E12843D14FF4FA7007F065F83EE004F156010878401C087094F8520003280F
:20E6500018BF042803D14FF4FA7007F055F894F85600032809D094F85200022827D104F107
:20E670000800102108F0B2F921E007F013FC1EE094F85200022817D104AE6946304606F0EC
:20E690008BF85220002108F0C1FAE06820B1026812B1304669469047042006F08FFE04F1C3
:20E6B0000800102108F092F9002084F8560005482A30016809B12846884708B070BDC046AA
:20E6D000481300209E13002010B5401EADF1380D28D0401E09D0801E4FD0401E43D0401E1D
:20E6F0003FD0401E3BD0002048E001A800F004FD04460CA942F2090005F03CF99DF8300085
:20E71000002808BF002203D0022007F05BF9024601209DF83010009001AB204605F07BFC4C
:20E730000A3028E001A800F0E7FC04460CA942F2080005F01FF99DF83000002808BF0022ED
:20E7500003D0012007F03EF9024600209DF83010009001AB204605F05EFC001D0BE0202011
:20E770000CE002200AE042F2130004A905F002F904A808F0FFFC80B200E004200EB010BD4D
:20E7900070B52A4D0C460646A00833D2A00F48D306F034F9234808F06FFE2648401C007883
:20E7B000012803D006F1380009F094F81E4800240460022006F070FF1120FFF7FDF8307C5C
:20E7D00010B90E20FFF7F8F81949AC710878EC7128B10C7005F1D400042108F0C7FBB5F944
:20E7F0002400B5F92610884214BF0220072001F001FF70BD05F12006304608F096FFFCF7EB
:20E81000EDFD304608F091FF30B924F00204A00F07D34FF0005100E0022105F1D40008F01F
:20E83000A5FB70BDA5E4000000000460700A002017320020700A0020F8B505460E46052000
:20E85000287096F849006968E870F06B4861686806F1280108F0A2FCB6F8420069684881FC
:20E8700096F84600696848746868002404761F4869680078C873686806F11C01193008F0A9
:20E8900039FF307C69688873706810F8011B6A68918110F8013B6A68918941EA0321918147
:20E8B00007786A68F91117F007071174214607EB470218BF012189184018401C10F8011B3F
:20E8D000297201F00702E860491001F0380101EB420140187268318968618B18834239BF84
:20E8F0002C72211C801A091A2974F8BD5E1200202DE9F84F274C834620888A460A254FF00F
:20E91000FF09002604F138084746401C208038465946082207F0B8FC30B16D1E07F1080796
:20E9300006F10106F3D100E0B146B9F1FF0F05D12079401C2071FF20BDE8F88F4846694692
:20E9500002F022FD0646FF2EF5D09DF80000012806D0606B06EB8601401880F804A004E029
:20E97000206B00EB461080F81FA00B490A6808EBC900026049684160084D6868804794F8D6
:20E990008810491E84F88810A96888473046BDE8F88FC046A42E0020D08A01008C140020BF
:20E9B0002DE9FE4FDFF888804FF0010B0446DFF8849088F800B099F80000012803D058462A
:20E9D0000021F9F797F8204606F090F81F4F7868804700241A4D02901749286A174A866830
:20E9F0004C8302238DE81800164B106818318A462246B047B968A88000280AD4124A92F9FF
:20EA10000000401C10700298C5F80CA088475C460BE0404604700298884748460078012819
:20EA300003D020460146F9F765F82046BDE8FE8FCC1A0020E41A0020280D0020901900201F
:20EA500028160020F9370100CD1A00208C14002010F47C1F70B51CD110F00F0F1CD001464E
:20EA70000024012202EA010091435200401E0BD0401E07D0801E03D0001F07D1093404E035
:20EA9000241D02E0E41D00E0641DA4B20029E9D133E010F00F0F01D0002070BD06460224E7
:20EAB0004FF4803505EA0600AE436D00B0F5803018D0B0F5803013D0B0F500300ED0B0F52E
:20EAD000802009D0B0F5002004D0B0F580100FD1072008E0062006E0052004E0042002E0D5
:20EAF000022000E00120FFF7EFFD2418A41CA4B2002ED7D1022CD8BF0024204670BD7047A6
:20EB100003B42DE9F04F92461E4609AFBAF5806FADF1040DA8BF052041DA97F80090B9F128
:20EB3000400FA8BF09203ADAB7F80280B8F5806FA8BF072033DABF88B7F5806FA8BF0820F9
:20EB50002DDA194C2079032808BF032027D04FF0000B09F03F01C8F30900C7F3090584F809
:20EB700005B040EA013045EA0035E188A0782A4602F0F2FC014600290BDCA6F80CA0A6F801
:20EB90000AB03560B780A6F8068086F808900A2005E0A07889B2324602F0AEFE607901B0A3
:20EBB000BDE8F04F02B07047441A00202DE9F0470020DFF89080224E234D88F83D0096F8FB
:20EBD000719095F84000401CC0B2042885F8400030D0202005F06CFF96F8B3100F2917D090
:20EBF00098F83E7096F87100B84211DD194C8946606886F87170804782461448144950F8F5
:20EC100027008860C86004F0BFFFA1685046884795F8401096F8713038F819404FF47072D3
:20EC300005F11000491C9A4001FB142107F096F9BDE8F08706F05AFBFFF78AFCBDE8F087C9
:20EC5000A8110020EC1700201C310020E8880100241A00208C14002090B50446002140229A
:20EC7000ADF1440D684602F088F8A0788DF80000E0788DF801009DF8000000BB616811B11F
:20EC900001A805F0C8FB217A01F007028DF82820E0689DF82870C1F302118DF8301027B1C8
:20ECB0009DF828100B9000EB41009DF8307007B10D90207C8DF8380067690F9719E0616895
:20ECD00011B101A805F0A7FB677A8DF82970A37A8DF82A30207A8DF82800E27A8DF82B20B4
:20ECF000217B8DF82C10677B8DF82D70E389ADF82E300348006801696846884711B090BD8C
:20ED1000181A0020F0B5012904460546ADF1140D04D0022941D142F2030001E042F202000F
:20ED3000694604F027FE04B16D1C07F053F9C01DC010C0B2002830D000230646ADF1010C19
:20ED50001F4618461CF801EF00224EFA02F101F00101884211D028B97F1CBFB25CB102EBFA
:20ED7000C30103E03CB102EBC301491E05F8011B091205F8011B80F00100521C082AE4DBBA
:20ED9000761E03F10103DDD130B12CB1D800401E05F8010B001228700FB9002005E004B100
:20EDB0002770012000EB870080B205B0F0BDF0B50446ADF12C0D08F0BFF9002818BFFC20F4
:20EDD00048D168462146112200F06AFCE67CA07C8DF81360257D8DF81200677C8DF81450F1
:20EDF000637D8DF81170A67D8DF81530002006B1012094F82450E28C8DF81600267E8DF806
:20EE1000245094F82530ADF826208DF81860E07D8DF825301A258DF8170057B9812007F0EB
:20EE3000B1F804460A94A4B1FF21812208F08BFC09E09DF81510880000EB411080B207F00A
:20EE5000A1F804460A9424B10720694603F056F9002528460BB0F0BD2DE9F843254C8046B1
:20EE70006068804781466946722006F087FF3225FF27002600994046091D07F05DFE01280C
:20EE900008D000986D1E06F1010600F118000090F0D100E03746A16848468847FF2F18BF47
:20EEB000381C22D1144DD4F804900A270026383512492846082207F0E7F930B17F1E05F138
:20EED000080506F10106F3D10DE040460168296040686860C847064A92F88810491C82F81E
:20EEF0008810A16888476436F0B2BDE8F883C046A42E00208C140020A42E0020D08A010031
:20EF1000F8B5214C236813B908F0CEF92368234808380068044608F0F1F8D860204607F053
:20EF30008DFD1F4D18826868804706461748A9680278832A24D1164CE21D17783FB9852233
:20EF5000027030468847002001F0CEFAF8BD86210170082007F034FB26340E4F0E49114B8C
:20EF7000208840F64852B962401C1978208007F12000B2FBF1F101F2A32107F097FDA96867
:20EF900030468847F8BDC046640E002020320020C418002094180020E53B010048160020F6
:20EFB0008C140020C8190020F0B52348214D4FF08056A861D6F8D801204C036801210A46F4
:20EFD000ADF13C0D20469847D6F8D80142680121204690471A48012606601A48F9F7D8FA32
:20EFF00005F01AFB05F11C07384607F0ABFE05F134044FF4E13039462060002005F02CFB03
:20F0100011493C22082308600021684608F01AFCA4344FF46170002307940C4908906A4671
:20F03000069605F1880008F009FC08F003FC0FB0F0BDC04608020020F97601000040034023
:20F0500004011CE228890100680600207D28000038B504F073FD02F07BFE204D05F1380061
:20F07000007820B11F4808380168012088471E48007810B91D48007808B108F015F91C4C8C
:20F09000606880471B4AA1681378022B1CD1144CA31C1B78042B1CBF832313708847A178F1
:20F0B00031F0010008D0042906D0052907D10020207108F050FB01E0FBF7DAFCA17804295A
:20F0D00003D007F0FDFA00E0884795F8380020B1E86C10B1102008F037F938BDEC13002099
:20F0F000C4180020401600201C3200201E3200208C1400202032002070B50446E820ADF169
:20F11000280D09A904F068FE9DF82400694607F006FB00280CBF00981E480DF12501606069
:20F13000E82004F059FE9DF8250004A907F0F7FA58B90599C8200322B1FBF0F0401EB0FBCC
:20F15000F2F15143401AC0B200E00020207206F041FF00216081656821700F4B61700A46B9
:20F1700008925968A9420CD1197A267AB14208D15989814205D1187820705E7866701046C0
:20F1900006E008990C33491C06290891E9D901200AB070BD38C40D00D41500202DE9F04743
:20F1B000254C01258246984691460E46C4F87C570320C4F8805708AFC4F88407D4F88C0735
:20F1D00010F0030FFAD1387858B14FF08057D7F8B001016A27208847D7F8B0010169272041
:20F1F00088470220C4F8FC06C4F80894284608F060FAD4F808040008F8D2D4F88C07800FA0
:20F2100028BF281C15D2B8F1010F14BF08200C20C4F84C051021C4F850150020C4F8540558
:20F23000064A1560C4F800A0A160C2F800542662A162BDE8F087C0460440024000004842D1
:20F250002DE9F041DFF8948006460C4636F07F0015D1002E3ED1224D243D686880471E4938
:20F27000096831F81620144321F81640A968884741461431086807F033F9BDE8F08104206F
:20F2900006F0F0FF071C25D04FF6FF7038807C8008F076F941468C78A7F10C05FF2802D065
:20F2B000C96A40184478FF2C06D1384607F0C2FF07F0ACFABDE8F081304607F005FC014657
:20F2D0003A46FF20A872204605F026FF10B1384607F0B0FFBDE8F081242D002064180020DD
:20F2F000B014002025483EB50078002843D042F20100694604F03EFB42F2050002A904F01E
:20F3100039FB1D4D95F8540010B39DF8080000249DF80810009B2864642285F85440581AFD
:20F3300002FB00F1E96705F1780003F0D5FE01A805F0B0FA124801992E300078B1FBF0F2AB
:20F35000451E4243891A01918D4214D9204610E09DF8081064204843E86705F1780003F002
:20F37000BBFE288F401C288700242C64012085F8540004F00DFD3EBDE82D002035120020C7
:20F39000302F00202DE9F041224C064604F1580005780F46002D04BF0020011C1CD0204D38
:20F3B0001D49281D0B780068D3B91C480568E06C07F01CFF228FB0FBF5F1B0FBF5F3891876
:20F3D00089B203FB05F2236C3980801AC018306085421CD8401B491C30603980BDE8F081C9
:20F3F00080475FFA80F804F1780007F0EBFF226C4FF47A73410001EBC001B1FBF3F0238F2A
:20F410003060A9683B808018306040468847BDE8F081C046E82D002035120020382F0020C4
:20F430008C1400202DE9F043254C0746243C606AADF1240D00283ED0002F3CD0387A0028B1
:20F4500039D004F01DFF5FEA000834D0062000250323A1468DF808002E46ADF80A30B5F54C
:20F47000FA7F28DAD9F82400ADF80C5004AB02AA0469009392E803000A230022A047B0B994
:20F49000387A9DF81810814210D1022804D1BDF810103A88914207D0032807D104A93846DB
:20F4B000082206F0F1FE08B9284606E0761CB04505F10105D3DC4FF0FF3009B0BDE8F083A7
:20F4D000C8100020F0B520480127F84201D004F0A7FB204D204F214EBD4206D203CD0478E0
:20F4F000A4003459401CA047F6E71D48002800D08047164D164FBD4202D210CDA047FAE747
:20F51000F0BD03251BE0416808300A1C2A400BD11A1C2A40AB4305D0046804300C6004311A
:20F53000043BF9D1131C05D0047801300C700131013BF9D1021C2A4001D0A843043003686A
:20F55000002BE0D17047C046FFFFFFFF0000000000000000400E0000A00E0000000E0000FC
:20F5700055C5011070B504466068254E4078ADF1480DC00921D3B4F842003546B63DB5F835
:20F590008A10884219D11D480078A0B995F8940098B104F1280006F0A5FC70B901200090DF
:20F5B0001C340194B5F88A3005F17A0203210620F8F7C6F81FE007F033FA0BA80021182255
:20F5D00001F0DBFB02A821460C900BA8FFF734F92C208DF82C000BA803F020FC3546503D0A
:20F5F000287810B19DF83C0028B105208DF82C000BA8FEF743F812B070BDC046ED13002022
:20F610005E120020F8B5234D012001462870F8F771FA6FF00100204C1D4927690870381C45
:20F6300028D0A1684268914203DA07F03DFE27693846C8B105F07AFC7968884224BF27691D
:20F65000381C11D200F0C8FE14E026697068002802D507F029FE2669304604F015F9B16815
:20F67000307B88472769384620B105F05FFC79688842EAD2094C606880470646FEF7CEF87F
:20F69000A1683046884707F003FA00202870F8BDC91A0020E41A0020241A00208C1400206C
:20F6B000002A4AD05FEA000C8B071CD1830722D1102A08D370B4103A78C978C0103AFBD292
:20F6D00070BC103238D0042A2CD3082A05D30C2A24BF08C908C008C908C008C908C09207F0
:20F6F0002AD0920F22E00B780370491C401C521E22D08B07F7D1C30714D18307D8D0121FD8
:20F7100012D308C903801B0C4380001D121FF8D20AE008C903701B0A43701B0A83701B0A5B
:20F73000C370001D121FF4D2121D05D00B780370491C401C521EF9D1604670472DE9F843CF
:20F75000002A894607464CBF47F6FF75151C002F08BF002032D03888002808BF002403D0A8
:20F770002A4600F0E5FA0446281B26DD388828B1291B484612A204F00BFE0419B868E0B1C0
:20F79000D7F804802E1BB8F1000F0DD0404607F0F1FC401DB04207DC291B484609A2434686
:20F7B00004F0F6FD04192E1B122E06DBBB68291B484606A204F0ECFD04192046BDE8F883AE
:20F7D0003A2000C0222573222C2000C06C696E652025643A200070471CB51F4C04F178000C
:20F7F00006F0A4FA04F15C0006F0A0FA04F1940006F09CFA0021882204F1340007F0A3FFE2
:20F8100007F018FC06F0E6FB84F85A00134984F85B001348086001200DF1010184F8B300DA
:20F8300042F2040004F0A6F842F20500694604F0A1F80C489DF80110A066642041432166EA
:20F850000949C4F884109DF800104843E0670748C4F8A0001CBDC046E82D00203816002052
:20F87000C954010039390100F5F200009F760100D0B5244C04F124010F68002F3FD0002204
:20F8900015280AD13B7D0126022B08D0032B06D0052B04D0042B02D000E03B7D00269842BB
:20F8B00000D016B17B7E5B0905D23A4657F80C7C002FE5D123E00846394605F053F9F88A9E
:20F8D0002760000A03D397F91C0007F02BFC387D022818BF052802D1012006F071FE206823
:20F8F000407E30F07F0005D194F82F00401E84F82F0004E094F82E00401E84F82E003846DD
:20F91000D0BDC046640E0020F0B50546224CAF686068ADF12C0D5FBB0C2000F029FE071C1E
:20F930001DD0684600212422082307F0AFFF002306976A466968ADF810301848059307F0D0
:20F9500075FF386070B908200C26ADF82400616AADF8266009A88847384606F05FF86FF09F
:20F97000030017E0E86878602869B860AF6009E080470646386806F093FE2869B860A168C8
:20F99000304688473868696807F074FF386807F081FF00200BB0F0BD8C14002095740100CE
:20F9B0002DE9F0418046204800680E464169272088471E4D0124C5F87C470327C5F8807758
:20F9D0001B480460C5F88477D5F8040420F00300C5F80404D5F8040440F00100C5F8040420
:20F9F00004FA06F6C5F8FC6312480460C5F800801020A860204607F05CFED5F88C0740084F
:20FA1000F8D3D5F88C0710F0404F0AD1C5F884770020C5F8FC06D5F80004864218BF201CFE
:20FA300000D10020BDE8F081B00100100440024000E04842000048422DE9F843234D8846E5
:20FA500006464FF0FF3105F12400814607F046FF00200CE0FF2909D02A688A4204D905EB86
:20FA70008101D1F894700FB1002627E0401CB8F1000F03D018F82010FE29EBD10024346078
:20FA900074600127B46011E0FF280ED005EB80000B787268C0F8946007FA03F010437060C0
:20FAB0000A680949304605F0B9FB641CB8F1000F04D008EB84010878FE28E5D1484607F0EE
:20FAD00009FF3046BDE8F883007FC7674C2B0020B0B5456884682349607DA27DADF1180D0B
:20FAF00040F000400090207D0027FF2A41EA000001904FF0020002D0E27DFF2A00D13FB1F1
:20FB1000E37DA07D1943039140F0004002900420FE214DF8201005F158006946FFF78CFF30
:20FB30006866002808BF381C1AD0617D0F2205F0F9FF686E217D102205F0F4FFA17D384694
:20FB5000FF2902D0E27DFF2A00D140B1686E112205F0E8FF686EE17D122205F0E3FF01200C
:20FB700006B0B0BD0000C0A098B5244C0746A8B1401E0BD0401E2CD1204690F8402042F07B
:20FB9000080202F0EF0280F8402022E094F84020204602F0E70242F01002F4E7214601F1E9
:20FBB0007402107891F83C3000F0F000107003F0F000002281F83C0091F840308A6343F00F
:20FBD000080000F0EF0081F84000F420413104F003F9002F08BF44F620600CD007F021FD5E
:20FBF0004FF4FA670A2244F6206390FBF2F15143401A07FB0030A06498BDC046280D002026
:20FC100038B5054695F83000032839D195F83A00032835D105F128044A202146F9F740FB94
:20FC30008A202146F7F77AFE6C686178207800EB0120ADF8000069465020F9F731FBA41C4C
:20FC50006178207800EB0120ADF8000069464B20F9F726FB8B206946F7F760FEA41CE120E0
:20FC70002146F9F71DFB641C6178207800EB0120ADF8000069465320F9F712FB002000E044
:20FC9000E82004492A24087028462C7003F0C6F838BDC046C93000202DE9F8432020EFF3F7
:20FCB000118780F31188214CA068012107F0BAFD4FF001094FF0000865692168A4F81C901C
:20FCD0006A1A2168A4F81E80461B401A904227D387F3118840464519361A4846294607F00B
:20FCF0009DFDB042F7D92021EFF3118781F31188E18B012903D14046294607F08FFDB0F14D
:20FD1000FF3F06D0A169801B814238BF081C411901E0A069291807F07DFDA4F82090256075
:20FD3000A4F81C8087F31188BDE8F883780100207FB503461F480D4601881F4800881446A6
:20FD500014A6984205DB32462146284604F020FB1DE0994206DB184606F0C2FC0028F2D00E
:20FD70004268F1E715480088002808BF0CA2EBD00095002C48BF47F6FF74114E0020114963
:20FD900001946A46346802901846A047029800907FBDC0467B6D6F64756C652325647D0005
:20FDB0007B6D6F64756C652D726F70653A25787D00C046C06E8A01002C8B01008E140000E2
:20FDD000248B0100495901000FB42DE9F04106AF8046ADF1300D07F0D9FB3E1D002526F0FF
:20FDF0000306361D0A961420ADF82400FF24079508268DF826407868ADF80060164F0B903D
:20FE10001A203968ADF802006846884708B99DF80440ADF80860ADF80A600320ADF80E80C7
:20FE30000AAB8DF81000243F8DF80C40796A059302A8884706A8069504F0B4FF012804D053
:20FE500018B9069808B106F0CBFA0A9800680CB0BDE8F04104B07047B014002090B50C462D
:20FE7000214A0178575CADF11C0D0B2F8DF8007035D0002F36D00C2F04D0112F29D107F06B
:20FE9000D9F926E01A2C22D090F899100190C7688DF80210038A0297C28AADF80C3051090D
:20FEB00005D21249827E98310978891A00E000218DF80E10877F8DF8107090F91F308DF807
:20FED0001130826A0592417F8DF80F1001E0002001908DF801406846FDF7D0FB02E044708F
:20FEF000FDF722FA07B090BD20830100A81100202DE9F04107467868BE68044600F5847094
:20FF100006F0CEFB30681C4980690968C0F3C00008BB07F0FBFC194D8046287820B10220D8
:20FF300005F0BAFB00202870404607F0EBFC3168134D886B20F020008863286820F4807050
:20FF50002860606A216A091A21622369626A38469847BDE8F0814FF4FA70B0FBF1F10129DF
:20FF700098BF012104F58474204607F083FC204607F090FCBDE8F081108B01001532002029
:20FF9000301000407CB515460E46044600E004192046694605F02CFA00282ED014F8021F27
:20FFB0008E42F4D1491E04F1010420D0491E12D0491E08D0491E18BF622029D102281CD1F2
:20FFD0002078287023E0032817D114F8010B2870207868701BE007280FD161782078A41C70
:10FFF00040EA0120288020682E1D30600FE005288F
:020000040001F9
:2000000003D120780628287001DD67207CBD2D1D0020641C2860A678AE70208828800020F2
:200020007CBD70472DE9F04106467568B46807F075FCA96A39B921688969090903D207F07E
:2000400069FCBDE8F0810027AF6207F063FCA17D3846FF2902D0E17DFF2900D118B1284673
:20006000214601F0E7F82168886B20F0200088630D49086820F48070086007F04FFC0B4CE7
:200080008046207818B1022005F00EFB2770404607F040FC686A296A091A29622B696A6A4E
:2000A00030469847BDE8F081301000401532002038B50C4644220546002100F066FE04F194
:2000C0002801284606F06AFE04F1320105F10A0006F064FEE06B6861B4F840002883B4F854
:2000E00042006883B4F84400A88394F84600A87794F84700E87794F9480085F8200094F897
:20010000490085F82100B4F850006884E06C6862A07B85F8280094F8520085F82900606DE9
:200120000B2204F11C01E86205F13000FFF7C0FA2089A5F840006068E86338BDF8B507F02E
:20014000EDFB204C0746D4F8A80010F4602F2CD0D4F8A800400CC6B2700807D2B00803D2E5
:20016000F00828BF022602E0012600E00026751D68B202F037FFD4F8A83006F111010120C7
:20018000884023EA00013846C4F8A81007F0C2FBB00004F190010A18D7684FB108580022CA
:2001A0004FF000632946B84702E0384607F0B2FBD4F8A80020B104F58470002106F0DEFE06
:2001C000F8BDC046700A002070B51E4DAC68064606F078FD4FF47A71001B4843030C05F097
:2001E000E9FD2969401A48BF404240F6B8319B19994210D306280EDAE9688C420BD828686B
:2002000048B1114A091B51438A0C02EB1141884288BF011C08E00D49486840080ED2086849
:200220007D2100F0FF004143C82905D3B1F57A6F88BF4FF47A6103E0C82101E04FF4FA61A5
:20024000084670BDE831002040420F00AC3F005003B42DE9F0411F4DA8684FF0FF3106AF80
:2002600098461446ADF1180D07F040FB396804A80160B988818004A803C822466B46FEF7DC
:2002800047FC0026071C0FD1BDF80C0084421CBFADF80C40BDF80A6008D12246684631461A
:2002A0004346FDF78FFD07460A2F09D16846414603F0BEFD07461EB1304605F027FF6F795D
:2002C000A86807F00FFB384606B0BDE8F04102B07047C046441A00202DE9F8431F4C002634
:2002E0004FF001084FF002093746A51E15F8020F03280FD0022824D168786368022820D020
:20030000304607F08CF90146384607F017F985F8019011E0304607F082F901466368687846
:20032000012805D0384607F009F985F8018003E0404607F003F96F700246C9B2184604F0FA
:2003400071FD761C022ED1DB05F098FD18B104F1200007F0F4F9BDE8F883C046A817002070
:200360007CB5042005F0BAFB022818D0032816D019480068C0F38150032814BF41F2883223
:200380004FF47A721649174C096854342046B2FBF1F107F077FA204607F084FA7CBD4FF0C3
:2003A0008056D6F8A4010D4D446800214FF040521C23032000902846A047D6F8A401002121
:2003C0004FF4007209230126446800962846A047022005F069F97CBDB43F005000A00C409D
:2003E000108B0100940F0020F8B51E4C002528462268A168256190420CD05268914209DDBA
:2004000004F09CFD0146206842689142C8BF41602061A168676837B118B142687B689A4268
:2004200001DD38462061C8B14068814216DD0E4E044606F108000068A04201D806F03CFF0F
:200440000A4D686880470746F460204601F0AEF9FDF7ECF9A96838468847F8BD05F0F8FE38
:200460002561F8BD241A0020C81900208C1400202DE9F8431C481F4D077868688047814624
:200480001A4883680026344680469C4212D013F8020C874208D134B163B138464FF4004133
:2004A000FEF7D6FE13E01C4604B91E4653F80C3C002BECD15FB9686880470D49096831F8E3
:2004C00017206FF3DF3221F81720A96888472CB108F108002146324604F04CFBA9684846AB
:2004E00088472046BDE8F8831415002064180020242D00208C1400202DE9F041804600275D
:200500001A481D4D07701A481A4E077096F83800D8B1F36F2C68C3B1207D352809D1606802
:20052000218900F0B1F860680088000901D304F003FBF16F404688471048007801280BD0D0
:2005400038460146F7F7DEFA06E003F0FFFA01F007FC4046F8F772FF286810B1007D352839
:2005600001D006F07BFCBDE8F081C0461832002020320020EC130020640E0020E41A002076
:20058000F8B5001D84B214F0030002D0241A241DA4B206F0E7FA1A4A102C01461769D1603E
:2005A000C8BF5769388800221646C30BDD0319D126B984420ADD3A46012617E01388C3187E
:2005C0009BB29C42138011DC174618469FB1001B80B20428B4BF3C88385344F400443C80F2
:2005E0003F1D08E080F40040002680B2C71938880028DAD10027084606F0D8FC3846F8BDC6
:200600008C140020F8B5054607F088F91D4C064604F5B8710878A84304F59E750870286854
:20062000002808BF002706D02868943007F099F8002700B10127686838B1943007F091F8F5
:200640000025384318BF01252F4694F87001A8B9012F13D0D4F8640198B1406988B107466E
:20066000304607F057F9D4F8640100214FF400030A46B8470020C4F86401F8BD304607F073
:2006800049F9F8BD700A00200829C8B50BDA00293BD00278491E92FAA2F24FEA226200F84C
:2006A000012BF6D1C8BD464206F00306891B37188AB2361802F00301864209D9361A037853
:2006C000761E93FAA3F34FEA236300F8013BF6D122F00302D71987420AD93A1AD21C96100E
:2006E0000268761E92FAA2F212BA40F8042BF7D1CF19874209D93F1A01787F1E91FAA1F1C2
:200700004FEA216100F8011BF6D1C8BDF8B50546012004F0D5F91D4C04F1140003F0BCF8CA
:2007200004F1240003F0B8F869684A78087800EB0220ADF800008F7804F114066FB9532087
:200740006946F8F7B5FD05F128014A20F8F7B0FD05F128018A20F7F7E9F806F1200005F17F
:200760001C010B2206F0C2FBBDF80010384604F0ABFD94F83F00800803D36878002106F07D
:2007800031FB002084F83F00F8BDC046383000201C491B4898B5FF220F7890F83B301A49FC
:2007A00080F83820012B15D091F8710091F89010884224D015480024047006F0A0FF01F0FC
:2007C0009FFE13480078012819D020460146F7F799F998BD002380F83B3087B18DF803202F
:2007E00091F8A7008DF8000091F8B6708DF8017091F8B7408DF80240684606F027FF98BD39
:20080000EC170020930E0020A81100201D320020E41A002070B50025ADF1200D07A8ADF825
:200820001C5006F029FD1B4CBDF81C10208F884227D194F85300032811D004280DD0022859
:2008400010D104AE6946304603F0AEFFE06820B1026812B1304669469047042000E00320D7
:2008600004F0B4FDA06D04F04FFF5220294606F0D5F94FF47A7004F05FFF284604F074FF8B
:2008800005E0032006F09CFC052004F09FFD08B070BDC046481300202DE9B84107F03EF86B
:2008A0001C4C1B4D804604F1E000007848B92C46A168022088470746102003F04FFD0FB36A
:2008C0001DE001F023FD70B9134800683221B1FBF0F101B901213034204606F0D3FF20466A
:2008E00006F0E0FF0EE0002084F8E0002C46A168022088470746102003F030FD17B1A168DF
:2009000003208847404607F005F8BDE8B881C046808A0100940F0020108B0100F8B51B4E07
:200920000024012004EA0307194D3070002F4FF0020000EA020008BF00280DD14FF0E040EC
:2009400004EA02011840002808BF002904D11249888D401C888503E095F90000401E287021
:2009600006F082F806F07AFA0A48047095F9000030B195F90000002806DC06F09DFC03E05E
:2009800020460146F7F7BEF83470F8BDE41A0020CD1A0020CB1A0020C41800201D491E48BB
:2009A0002DE9F041352751F8048B51F804EB51F804CB51F8046B51F8045B40F8048B51F8FC
:2009C000044B40F804EB51F8043B40F804CB51F8042B40F8046B40F8045B40F8044B40F89D
:2009E000043B7F1E40F8042BDDD151F8045B51F8044B40F8045B51F8043B40F8044B51F8D7
:200A0000042B40F8043B40F8042B09680160BDE8F081C046C802000000C0002138B50546F8
:200A20001B491D4C2878E0B96878012815D0022809D0032826D108460021817040210830A4
:200A400005F0CCFF1EE004F13A000078FF280CBF0120022006F0B4FB14E004F10800202125
:200A6000EEE76A78032A08BFEA2804D0012A09D141F2883000E0074891F8542081F85520DB
:200A800004F072FE7434216809B12846884738BD48130020E09304004813002070B51B4CDC
:200AA00005461022ADF1200D04F171016846FEF7FFFD0026049509208DF8146004F10D0104
:200AC0008DF8160001258DF815500A680DF1170002604A684260097A01720D496A461820FA
:200AE000FFF77AF90B4918208922631DFFF774F97120314606F0D8FBD520214606F0D4FB81
:200B00005D20294606F08AF808B070BD4C86010001A800002D7900002DE9F0431C4E04466D
:200B200000271D468846A2EB0409ADF1140DC6F8B071012006F0C5FD3068C00FF9D3306A7F
:200B40000090706A0190B06A0290F06A039044B128462346694611F8012B5B1E00F8012BB4
:200B6000F9D10320C6F838026CB108EB09016D1E491E11F8010F15F8012F904218BF042061
:200B800002D1641EF5D1384605B0BDE8F083C046504502402DE9FC410021054606F094FDCC
:200BA000B72806D140F6FF712846CA1E05F0D0FC40BB154C626805F0AFFEDFF8508001282A
:200BC0001CD190470646684604F016FB280305F06BFE0746009805F075FEA168304688472E
:200BE00037B928460021B72206F08EFBBDE8FC810221404641710171BDE8FC8140460B215B
:200C0000401D0170BDE8FC818C140020441A002003B42DE9F0431C4DA8684FF0FF3107AF08
:200C20001C469146ADF11C0D06F060FE396804A80160B988818004A803C822466B46FDF7EC
:200C400067FFA846061C14D1BDF80C30BDF80A20D01A484481B298F802006518AA4204DAE7
:200C6000A342B4BF0526062603E0BB68224605F0A0FFD8F8080006F035FE304607B0BDE8F0
:200C8000F04302B07047C046441A00202DE918410446DFF870802078E02828D140464278DB
:200CA0008178012A0AD049B990F85220012A05D190F8540001281AD001200CE0104BB3F837
:200CC0006620521CA3F8662041B9491CC9B2817000234370022006F073FA08E0002004F0DD
:200CE00013FD032006F06CFA052004F06FFB40467C30016809B120468847BDE81881C04614
:200D00009012002048130020F8B500680E4617464FF0FF310446483006F0E8FD4FF0FF3551
:200D2000092E08D0217A0120B040084211D108433546207210E0227A0721012303FA01F0AE
:200D4000104202D0491EF9D503E0227A0D4610432072B5F1FF3F0ED06FB129463846FEF7BF
:200D600027FE40B1217A0120A8404FF0FF3580F0FF000840207204F1480006F0B3FD2846AC
:200D8000F8BD002213460A46194671B510F0030F0BD0002A82BF00F8011BB2F1010210F03C
:200DA000030FF6D1002A08BF71BD11F0FF0141EA0121042A18D341EA0141082A0FD30E46FF
:200DC000102A08D30C460D46B2F10F0312F00F0272C0103BFCD812F0080F18BF42C012F04C
:200DE000040F18BF40F8041B12F0020F18BF20F8021B12F0010F18BF017071BD03B42DE93E
:200E0000F041DFF86C80D8F808004FF0FF3106AF1C461546ADF1180D06F068FD396804A8BA
:200E20000160B988818004A803C822466B46FDF76FFE061C12D1BDF80A00BDF80C10411A2E
:200E4000691889B261188842B8BF062606DBBB68294622466846FCF7B5FF0646D8F808009C
:200E600006F040FD304606B0BDE8F04102B07047441A002038B505461B4C287868BB60781C
:200E800001282AD0281DFEF7D5FAB0F1FF3F24D1298AC81321D001F00F010F291DD1204646
:200EA000018F4FF6FF728A4204BFE9890187A97C80F83A10AB888387298A01F00F020F2A51
:200EC00005D080F85020C1F3031180F8511090F850100F2904BF012141706C34216809B11B
:200EE0002846884738BDC0464813002070B51C4C06460E220D4604F12C00FEF7D9FB687B16
:200F000020B9022020776B88A38208E003202B1D20771A6804F114010A6058684860606A15
:200F200004F00AFC30462946FAF7CAFE207801280CD0687B50B9288869882A1D002301F094
:200F400053FD011C02D002A006F0C1FB70BDC04641757468204572726F723A20307800C04D
:200F60009012002038B51B4D95F871000F2824D0194C3B3C94F83810FF291ED094F83A00A5
:200F800068B102290BD103F0D9FF216B0F4C95F86820401A2178083101FB12010BE003F051
:200FA000CDFF616B0A4B95F89020081A1988401A34F81210411A002901D5002038BD4FF6E8
:200FC000FF708842C8BF88B238BDC04685190020900E0020A8110020271800201649B0B5A4
:200FE00005461B4C0F7820780FBB144A8100B2FBF1F1A94202D206F05FF920786168104F1B
:20100000800005FB00143868C06B8047211AA1F54871090806D30B4A011B891A090828BF2A
:2010200000F5487408482146FCF766FEB0BD074901200870B0BDC046E51A0020FFF6C2FF53
:201040004816002000093D002DDC00001F320020C81900201C4938B591F85C3001EBE30417
:20106000657F012203F0070302FA03F383F0FF032B4063778B7E01F11800032B18D091F80E
:201080006030012B10D0022B08D0B1F856108A409102A1EB821101F570710EE0B1F8562040
:2010A0009101A1EB820108E0B1F856108A4001E004490A789102A1EB82111C3005F0FEFC31
:2010C00038BDC04641120020B03000202DE9FC411B4E074670688047184D804605F12000B9
:2010E0000068154C436C04F10C00006802216A4698479DF8000028B90D48007890B906F0DB
:20110000DBF80FE00B492A6A91F83D00936900F0F00040F0010081F83D00E0683A464FF095
:20112000FF319847B16840468847BDE8FC81C046E51A0020280D002084190020281600207B
:201140008C1400202DE9F84380461948077817B9184D287810B90120BDE8F883164E243E33
:2011600070688047814668880124B8F1000F0ED1214603464FF6FF72B9404A40104068803C
:201180007BB170B9002004F0AFFF044609E018B9204604F0A9FF68882146B940084380B265
:2011A0006880B168484688472046BDE8F883C046141500206C0A0020B014002000B50021AC
:2011C0002022ADF1240D6846FFF7DFFD1848018FADF8181090F83A108DF80B10808FADF89B
:2011E0000E0002218DF8161009208DF80C0001218DF81F1003208DF80D0000208DF8080021
:201200008DF81B006A468DF81A0007498DF81D001820FEF7E1FD0549B1F84C00401CA1F8AA
:201220004C0009B000BDC046F7750100901200204813002038B50C4621680546886B20F026
:2012400020008863686E217D012202F015FE686E217D012203F0E6FD686E217D002204F0F0
:2012600069FC686EA17D002204F064FCA878012806D005F1D0004FF0FF3106F037FB03E040
:20128000216888690009FCD2686E217D102204F051FCA17D0020FF2902D0E27DFF2A00D185
:2012A00018B1686E112204F045FC38BD2DE9F84F834689467120114604F068FD17468120FE
:2012C0006946F8F749FF4FF0F308002507E0B8F1000F23D038686D1CEDB22C3038609DF8E6
:2012E0000000A8421ADD3868066890F804A0002402E0641C0A36E4B2A245E8DD737A002BB3
:201300000CBF052009208145F3D14A463046594605F07EF90128ECD14FF000084046BDE8C1
:20132000F88F70471A487CB5007880B342F2050001A902F027FB42F20100694602F022FB47
:20134000144C9DF80400216C88420BD80098884203D806F0E6F901250DE00022012584F871
:20136000542004E001259DF8040084F85450401A64214143E16704F1340606F1440004F02D
:20138000DDFC06F1440001F0AFFE84F858507CBD35120020E82D0020F8B50B461A4991F8B8
:2013A0002D704D6B4C796430C2B25FB100206D1F6D1DEE7816B12E79B24207D07F1E00F198
:2013C0000100F5D1641CE0B2487104E0FF281CBF0021197016D10120187091F82C700C6BBF
:2013E0004B795FB10020203C2034A67F16B1E57FAA4207D07F1E00F10100F5D15B1CD8B2E0
:201400004871FF20F8BDC046A42E002038B5054601201A4C68712879B0B905F0A3FB217879
:20142000002904BF6FF00704051C15D0491EC9B2217039B905F0BAFD606804F09DFA0020CC
:20144000687118E0054613E005F08CFB05462078FF2805D16FF00604284605F0A7FD0BE0C6
:20146000401CC0B20128207002D1606804F09BFA284605F09BFD0024204638BD581A0020B5
:2014800070B50646B079F4680628A4F10C042CDA3079062829DA05F065FB154DB279910030
:2014A0000C3501EBC20169184968E1B105F07EFD30792071B0796071307AA071B179880067
:2014C00000EBC1002818F1684068083004F0C4FAB179880000EBC1002D186868406806F024
:2014E00001FA002070BD05F061FD6FF0020070BDC014002003B4B0B504AF3878ADF1180D8D
:20150000002808BF092027D0164D2C46A0684FF0FF3106F0EBF904A83968BD88016004ABF4
:20152000858093E8030000226B46FDF7F1FA2546071C0DD1BDF80A0004F0E8FDA878E988E1
:20154000009A00F011F86C790028D4BF271C0227A86806F0C7F9384606B0BDE8B04002B0AB
:201560007047C046441A0020F0B516460C4607460025ADF1140D0AE0241AA4B205E0641EC7
:201580003846A1B202F0DAFD04466D1CADB2092C1DD3641F38466A46A4B2214600F0B4F94F
:2015A0000098B04207D19DF8091031F07F0004D0C80902D20CE09DF809108808DFD2BDF872
:2015C0000C008442D8DC04490520487108716C4220B205B0F0BDC046441A00202DE9FC4722
:2015E000194C6779984691460D46034657BB174E301D026805F090F901281CBF0B206071A9
:2016000020D105EB033590478246684603F0F4FD4A464046294605F039F9009805F052F9FC
:20162000B168504688476F1E4846411E1FFA81F940B117F8010F18F8011B8842F4D0022033
:2016400060712071BDE8FC87441A00208C140020F8B50C461A4991F8AF00C2080AD391F8F8
:20166000AE20A24206D100F0FB0081F8AF00002781F8AE7006F052F90746204601F0B2FC7D
:201680000D48210201F47F41084304F0A7FB0B4905460868012604F10C0306FA03F290433A
:2016A0000860384606F036F905F0FF05012D0CBF301C8320F8BDC04601000804081004401A
:2016C000700A0020F8B51B4D0129044611D005F17400064605F020FE012802D1304606F0D5
:2016E00030F82CB305F0A4FC074605F0A1FC6A6910E005F15000064605F00EFE012802D11D
:20170000304606F01EF89CB105F092FC074605F08FFC2A6900EB0720611090FBF1F34B4397
:20172000C01A0918104605F099FF304606F007F8F8BDC046A410002038B544688568606E7D
:2017400005F004F8296817488A6B1040886316480068C168286888476868FCF735F904F144
:20176000800006F05BF804F19C0006F053F8A07818B904F1D00006F049F8607818B904F14B
:20178000EC0006F043F804F5847006F03BF806F0C5F80021217006F0BDF804F16C0004F0B1
:2017A000E7FE38BD0DF8FFFFD0010010154998B50F7817BB144A1178144F52688B0089004F
:2017C00000FB0324B7FBF1F1814201D205F074FD11480068C06B8047211AA1F54871090809
:2017E00006D30B4A011B891A090828BF00F548740A482146FCF780FA98BD064901200870F0
:2018000098BDC046E51A0020C8190020FFF6C2FF00093D001F3200204816002015F6000057
:2018200038B517481749007818B90846007828B906E00846007830F07F0001D005F03CFDC2
:20184000114D68688047114C0C3C2178A278914207D10F4AA9681278D20803D288470120FD
:2018600038BDA968884705F04AFFA078FDF7A0F8012804BFA078207005F0F0FA38BDC04643
:2018800024140020203200208C140020901900201D3200202DE9F8438146EFF311882020B3
:2018A00080F31188174D154C134F012605F11C000660A4F114000660F86A016A1420884777
:2018C000D9F81000810C14BF000C04202060386802682321002090470948066054F8180CAB
:2018E00020F4C02040F4803044F8180C2E6088F31188BDE8F883C0468401001018200940D2
:2019000080022443000024433EB514460D4605226B4605F04EF99DF803109DF804009DF8ED
:201920000430658101F00F01801040EA81109DF80150A0819DF803109DF8020003F0030302
:201940000A11800642EA90529DF8020063728111A28041EA85019DF800009DF80050E1802C
:2019600000F03F0041EA003105F0C005207242EA013222602B4363723EBD30B504460D46EF
:2019800042F20900ADF12C0D09A901F0FBFF9DF8240008B342F20B000DF10E0101F0F2FFF4
:2019A00000230094BDF80E00029300040190684602F05AFD044604A942F2030001F0E2FF8C
:2019C00004F010FB024604A9B4FBF5F06843241AE0B202F053F906E042F20D0003A901F002
:2019E000D1FF9DF80C000BB030BDFEE72DE9F843194D064628780C469846012805D0687A36
:201A0000012818BF6FF0010023D162600A20208001F0BCFA071C1BD4A77005F07FFF8146DC
:201A2000204604F0DBF90446484605F073FF04F0FF04012C05D0384601F0D4FA6FF001079C
:201A400006E005EB8705903545F8088C45F8146C3846BDE8F883C046700A0020F8B506469A
:201A600005F05CFF184C0125074606F19400E57004F01EFE2078012811D094F8700170B18F
:201A8000B4F92400B4F92610884208D1384605F041FF0720FEF7B6FD05F040FF0746B4F93F
:201AA0002600B4F92410884218BF86F8BA5007D106F1700004F0FCFD284602F083FBE57196
:201AC000384605F027FFF8BD700A0020F0B50546194C2878ADF11C0DE9281CD028BB00265C
:201AE00094F8520084F8566002281ED104AF6946384602F059FE5220314605F08FF82046C9
:201B0000C06820B1026812B1384669469047042003F05CFC09E094F85600401C84F8560033
:201B2000C0B2032801D104F0BDF98C34216809B12846884707B0F0BD481300202DE9F04126
:201B400007461748174CC01F06786068804780461549A268087886281CD1104D05F12A02C2
:201B60001088401C10808720087005F0FFFCA16840468847082004F059FBA879B04207D119
:201B800027B90020FEF7B8FCBDE8F0811B20F9E7E920F7E740469047BDE8F081C418002015
:201BA000943100208C140020203200202DE9F8430024002B16460F468046254606D5002F82
:201BC000C3F1000302D57F42761E2D2599463846494602F009FE0CA0405CB7FBF9F7002FD2
:201BE00004F1010408F8010DF1D1A64205DD3021301B401E08F8011DFBD10DB108F8015D51
:201C00004046BDE8F883C0463031323334353637383961626364656600007047B0B5ADF1FC
:201C2000400D05F073FE044600213C220823684605F010FE114841680691816800680490CE
:201C40000F480068002205900E480891694605F0D5FD071C01D105F046FD04F083FF0546BB
:201C6000384602F049FA08B905F03DFD284605F09DF9204605F046FE10B0B0BD80850100F6
:201C80008C140020E972010030B5401E4FF00004ADF12C0D0AD0401E04D0401E20D1F6F783
:201CA000DDFF1DE000F02EF9044619E001A821462422082305F0F2FD06940D4DADF814409F
:201CC00009490794012201AB05F1780005F0E2FD064A23462C2105F19C00009305F0F2FDF7
:201CE00020460BB030BDC046FD2A010055460000940F002080B501460A7D012A05D0152A08
:201D000003D0252A18BF352A02D1087E00091DD3087EC30916D2012A18BF152A01D10009C3
:201D200009D24F781B2F04D00B4807B10E30805C02E0232000E0312008700848007800F038
:201D400097FD80BD48780021884780BD4A7808461146FEF78BF880BDEB86010014150020EE
:201D60009EB51849A1F12404606880472146124CE288A38893421CD0104B1F78CFB9104B76
:201D800089681F7837F07F0714D1A28088471027A088ADF8007001A9ADF8040009880DF1E2
:201DA0000203198008480068426AE068694690479EBD896888479EBD841900201E320020B0
:201DC00020320020B01400204816002038B5042903462BDA05F023FC0546084605F0AEFB7C
:201DE000134C5B0002460229195503EB040012BF0329002141706068E9B203F013F804F032
:201E00003DF850B904F12000044605F085FA01280CD1204605F095FC38BD04F1200004466B
:201E200005F07AFA10B9204605F089FC38BDC046A81700202DE9F843174C04F12401086878
:201E40008846074628B300261D25387D35281BD140463946324602F08DFE787E30F07F0097
:201E600005D194F82F00401E84F82F0004E094F82E00401E84F82E007D7057F80C9C3846C0
:201E8000FFF738FF4F4602E03E4657F80C7C002FDBD1BDE8F883C046640E0020164880B51D
:201EA00007683FB315498B6803EA5300C00E21D2134A106880081DD2486880081AD2106887
:201EC000096810F0050F4FEA114101F0F00101F5E0710AD1B9420DD2190F38BF40F00100C4
:201EE000D90E38BF40F0040003E0B94202D920F00500106080BDC04628500940AC3F005053
:201F00000000094098B5154C94F8E100002710B91348007860B105F001FD94F8E3100029EE
:201F200006BF012184F8E310012705F0F3FC0FB1002098BD022003F0CFFB0E20FCF7D0F842
:201F40000849086840B9084A402010600127CF61002084F8E20098BD012098BD940F002041
:201F60008E8A010004800C402C500C402DE9F04180461748243007680E46ADF1300DBFB1E2
:201F80003869A8B1B8F1000F12D08EB106208DF828000125ADF82A500022ADF82C2002AC95
:201FA00000943C690AAB93E803001A23A04708B100200AE002A940460C22FDF779FB05A959
:201FC00030460E22FDF774FB28460CB0BDE8F081A4100020F8B50646B06801687568886B9A
:201FE00020F4FA6088631349086820F40070086005F094FC104C0746207820B1022003F024
:2020000053FB00202070384605F084FC05F086FCA96B11B905F07EFCF8BD0021A96305F034
:2020200079FC686B296BEB68091A29636A6B30469847F8BD3010004014320020F8B5844686
:2020400040F6FF741CF8013B002210E0481B401E10F8015B7F1E01F8015BF9D103E01CF89D
:20206000010B01F8010B521C5B08082AEADA5808F5D21CF8010B1CF8015B05F00F07FF1CAB
:20208000C5F30315122F45EA001508D11CF8016B300A24BF1CF8010B60F3DF16F719AC420F
:2020A000D4D1F8BDB0B5184C05460F46101C28D00DE03868606197F82700394640F0040082
:2020C00087F8270004F1200003F0CAF86769D7B1F8688542EDD014E0386888B13868C068BF
:2020E00085420DD139680868386091F8270040F0040081F8270004F1200003F0B1F800E07D
:202100003F68002FE8D1B0BD700A00202DE9F843DFF85880044608EB440000F11805008B0F
:20212000894604F0A7F8074611480678AFB12A883846002105F00FFB00253C7041467D7024
:202140000A5D381D494604F0D1FE3046394600F08FFB40B92846BDE8F8838DF80040684608
:202160001A21FDF783FE1A20BDE8F883148301001415002010B5164A144C92F83D0094F89C
:20218000401048B91348006860B9012082F83D00202005F0D9F805E0481CC0B2042884F8D1
:2021A00040000DD00C4971310A784FF4707304F1200003FA02F101F2636104F07FFC10BD6B
:2021C000202002F07DFCFCF7CBF910BD1C310020EC170020640E0020A811002010B50446C6
:2021E00000212822ADF1280D6846FEF7CEFD134911226846FDF75CFA05208DF812008DF86B
:20220000114000218DF8151001208DF816100B228DF81700FF208DF8180009208DF8130090
:2022200003208DF814000DF11900FEF7AEFD044918206A46FDF7D0FD0AB010BD63860100C4
:20224000BFED0000C8B50146164AC87AB8B992F82D70506B2FB3401F401DC6781EB1CA7F25
:2022600003799A4202D07F1EF6D1C8BD8A7FC270CA880280CA7F0271097B8170C8BD92F8FC
:202280002C70106B6FB120382030867F3EB1CA7FC37F9A4203D12022FDF70AFAC8BD7F1ED4
:2022A000F2D1C8BDA42E0020F8B5044605F0E2FA01F022FF071C17D004F054FC0546A18848
:2022C00011480022183030F80C6F46B901804760A168816022737868206100240EE08E42AF
:2022E00005D1284604F062FE6FF0020409E0521C062AE8D305F0F7F96FF00304284604F0F2
:2023000055FE2046F8BDC046A814002038B5012003F0E4FB012820D0114DD5F82401C468F8
:202320001048342101220023A047002808BF002014D0286803F08EFD04F0C4FC0B4A0A4D62
:2023400093681168D060C01AA1EB910105FB00F3180C884228BF011C1160012038BDC0466F
:202360008000001000A00C4040420F00E831002098B50446207B00F00F00022824D100F0D7
:2023800007FFA168081A8108114800F10C021768002F14BFFB6840F6C41303F57A728A428A
:2023A00012D20A4A12686FF050448C420CD3C91AB1FBF2F3012B8CBFB1FBF2F10121B0304F
:2023C00005F060FA012098BD002098BD108B0100700A002010B50446012002F071FB208956
:2023E00000280CBFEB2000201249607091F83F00C20824BF20F0040081F83F00820809D2EE
:20240000400813D32B202070EB236370204600F00DFD0BE091F83F0000F0FD0081F83F001A
:20242000217C6078C1F3001104F0DCFC204604F083FF10BD3830002030B5174C054605F1DC
:202440002801ADF1140D04F17A0003F00DFC08B3EF2309208DF801306B688DF800005A7853
:202460001978181D01EB0221ADF802102A890178082A8DF8041014BF94F8B600C07805F196
:202480001C018DF805000DF1070005F03BF96846FBF7FCF805B030BDA811002010B5044649
:2024A0000320ADF1180D04F128018DF8020000208DF8030001A805F028F96068007804F1F5
:2024C0001C018DF80C000DF10D0005F01BF904F1280003F00FFD58B14FF6FF74532069463B
:2024E000ADF80040F6F7E4FE044920460A3108800DF10200FBF7CAF806B010BD2212002027
:2025000070B5164D286808B105F024F8144C606880470C3DE9690A68002616710968E96175
:20252000A16888470A4A0B49107810B90846007860B1167008460670FCF792FD0648007861
:20254000012803D030460146F5F7DCFA70BDC0461C3200201E320020E41A002094310020EC
:202560008C140020F8B50025114C1348A5604FF4700665600068E660C06B80470D49C0F1E7
:20258000FF3008600D48C76865700FB90C49C1600C480570012001F0C7FF08B104F08CFE35
:2025A000304601F0F9FAE068FFF700F9F8BDC046C819002008300440481600206418002038
:2025C000112C01001F32002070B5164604460D1C08BF052426D034F07F0001D004F01EF9F3
:2025E000002C18BF032407D155F80C0C18B915F8020CFF2804D00524284604F023FE11E0F0
:20260000012E094805F8024C03D0294602F0AAFE02E0294604F00CF820464FF40041FCF7ED
:2026200017FE0024204670BD6C18002030B50446606800252062ADF1140DA5657820A4F88F
:202640004C0094F82C0025650F2807D004F12C0120460122F7F778F808B116E0284694F82C
:202660003C10FF2901D1A16D21B104F13C012046FBF70CFC48B92B4601208DF80C3003212A
:2026800001AA00902046F1F7F5FA05B030BD7047F8B5044605F0EEF801F02EFD071C04D183
:2026A00005F021F86FF003041DE004F05BFA05460E480022183030F80C6F56B94FF6F871F5
:2026C000018047600026866022717868A060344606E0521C062AEED305F005F86FF003043C
:2026E000284604F063FC2046F8BDC046A81400202DE9FC41144C154F06468846700809D397
:2027000020684568002101220B461FFA88F000903846A847B00809D3206845680021022253
:2027200001231FFA88F000903846A847F00809D320681FFA88F600210C220223446800963E
:202740003846A047BDE8FC81A401001000A00C400246F8B5084611464C68203821D0401E5C
:202760001CD0401E18BF6FF001001ED18D6805F0D5F80E4E07463068016928688847B0F187
:20278000FF3FF8D10025A564606C401EE06425653846A56305F0BEF82846F8BD0021084649
:2027A00001E00121002084F82D10F8BDD001001038B5154C04F1180005461C3001F06CF860
:2027C00003F010FD042003F031FDA07E032801D1607EA0B105F14501E120F6F769FD05F1E4
:2027E0004601E720F6F764FD084894F85F100078884204D005F14701E820F6F759FD2846E5
:20280000FAF744FF38BDC046B03000205F12002038B50120124C114D94F8711085F83D0067
:202820000F2917D00F490870202004F08DFD94F871200E490C4835F81220886201F12000C8
:2028400091F84010491C5143490001F2A32103F08DFB38BD02F052FD38BDC046EC170020D7
:20286000A8110020EC130020BDEB00001C31002070B502460D4632F07F0004D1104600229D
:20288000FFF7A2FE70BD04F083FE104908398C78A5F10C06FF2802D0C96A40184478FF2C4F
:2028A00002D103F0BBFF0DE0104604F015F901462A46FF20B072204602F036FC20B1284692
:2028C00004F0C0FC012070BD002070BD6C1800201CB5002922D04C08002948BF49424210BC
:2028E0005440002848BF404200230A1C904201D95200FBE790425B41904200D3801A9142EA
:2029000001D25208F6E7191C002C48BF4042640048BF4942021C081C111C1CBD0123DB077F
:2029200010B1A8BFDB431846FDF77BFB1CBDFEE738B5144DFF2822D0B63D95F8B4100129F6
:2029400015D1032844F6206416D00F48006890F8690088B104F06DFE0A224FF4FA6390FB23
:20296000F2F15143401A58432418A4B204E0032814BF4FF4FA540024A5F8B64038BD00201A
:20298000288038BD9E2E0020640E0020B0B5044604F004FE30F0010008BF6FF004041ED03A
:2029A00004F068FF054604F0DDF801460D480622343030F80C7F6FB1A388BB4208D1406804
:2029C00000680022854208BF0122A260002403E0521EEED14FF0FF34084604F0E7FA204689
:2029E000B0BDC0468C14002000B5ADF1240DADF80000ADF80210116801A801605168002266
:202A000041600E490693887D8DF80C200D318DF80D000B680DF10E0003604B684360097AE4
:202A2000017218208DF81C2005498DF81D206A46FDF7D2F9C0B209B000BDC0464C860100EA
:202A4000FD59000098B5154B1B1D18680004070C21D003F0AFF9104991F90720824205DD68
:202A600010F1800FB8BF6FF07F00C8718C88BC4210D80A68D3F8D40F801A801C1F2888BF5A
:202A80001F203F1B4008C7404FF6FF70E719B84238BF071C8F8098BD0C320020301009403B
:202AA00003B4F0B5144CA0684FF0FF3105AF1D461646ADF11C0D04F019FF396804A80160EF
:202AC000B988818004A803C8B2B26B46FCF720F807460A2F02D007B9012704E068462946DC
:202AE00001F0A6F90746A06804F0FCFE384607B0BDE8F04002B07047441A002008B51348FA
:202B0000134A14490078801E0A2807D8DFE800F01814100614100614100609C004F0C6FE06
:202B200011E010688008FCD250688008FCD20AE008688008FCD306E008688008FCD202E089
:202B400010688008FCD3F6F789F808BD7810002034600C4038600C40084610B500F00051B3
:202B600000F0040008431CD0012002F0B7FF104C012811D00B4801683220B0FBF1F2012A34
:202B80008CBFB0FBF1F101218834204604F07AFE204604F087FE10BD034804F075FC034806
:202BA000046010BD108B01006D35000000100440980A0020F8B5134C134940F27C622046B2
:202BC000FCF776FD002102220B46181932278D3000F8031F41707F1E8170F9D1521E03F12B
:202BE0009603F2D1094E04F5E275322728463146182204F07BF918357F1EF7D10220A0700E
:202C0000F8BDC046A021002050790100147B010070B5134C6068804712490025064648781F
:202C20004D70A168820808D2C00816D33046884728460146F4F766FF70BD304688470A48AB
:202C40000078012803D001202946F4F75BFF606880470646FAF7EAFDA1683046884770BDFD
:202C60008C140020C8190020E41A00201549096821280ADC212819D00C380FD00D380FD0FE
:202C8000001F0FD0C01E0FD01AE0253810D0001F10D0401E10D0401E10D011E008687047AF
:202CA0004868704788687047C8687047086970474869704788697047C8697047086A7047D6
:202CC00000207047F0010020F8B50646B08815460F46FDF735F80446002D02D4281B0A2848
:202CE00006DB3368291B38460BA201F059FB0419B08978B1002D06D4B06804F043FA291B91
:202D0000401D884206DCB368291B384603A201F047FB04192046F8BD257000C02827257381
:202D200027290000F8B50746C81D01F00705C610002F4FF0010000FA05F0A0F1010C14BFC2
:202D40000029002019D00020BEB17F1E33460246941B17F8011FB4F1FF3F08D10DB10CEA06
:202D6000010104E001F1FF04401C2140C0B20029F8D15B1E02F10102EAD1F8BD38B50C4639
:202D800020B141680122A240114201D1022038BD914341600E480025231800EB8401C1F824
:202DA000945003F140010978FF291ABF406850F8211044F020410548FAF79CF820464FF04B
:202DC000FF3103F08DFD284638BDC046007FC7674C2B002010B5144CE2685168496839B1D6
:202DE00010B102F091FEE268506840688047E2685268916809B9D06880B1094B18680028FC
:202E0000FCD00020186019B108468047E0684268D06800B18047034802F0E0FF10BDC046DE
:202E20001C10044001000706700A0020144BB0B5997B03EB81010A69017801F07F014D0088
:202E40000170AC185219527803EB82052F6907B19A732278141103EB84031F6C2FB90C295A
:202E60000CDA1821FDF702F8B0BD02F00F0257F8221011B904F020FAB0BD8847B0BDC046CD
:202E80001415002038B50546012001F019FE124C2046143000F000FD288900280CBFEB20E4
:202EA0000020687094F83F00C10824BF00F0FB0084F83F0080080BD394F83F0000F0FD00DF
:202EC00084F83F00297C6878C1F3001103F08AFF284604F031FA38BD383000202DE9F04120
:202EE0000120114E114D307028781F469046022801D004F0E1F90024022104EA070001EA89
:202F00000801002808BF002902D104F0D5F907E0074991F90000401E08702C7003F0B6FF20
:202F20003470BDE8F081C046E41A0020E51A0020CD1A00202DE9F041054612480E4600212C
:202F400000782960012802D00120F4F7DBFD0E4C606880473768804630463FB16A6879682A
:202F6000914203DC38463F68002FF8D1056030682F60854201D1FDF737FAA16840468847DA
:202F8000BDE8F081E41A00208C140020134A38B5B2F8AC504FF6FF71A9421BD0002401207D
:202FA00000FA04F32B4212D05940B2F8AC300C4D1940A2F8AC10291D0A6804F10C03984016
:202FC00010430860022003F0D1FC204638BD641C0F2CE5DB6FF0010038BDC046700A002089
:202FE0000810044038B5044604F098FC05461148D43890F8AF10C90803D390F8AE10A142EF
:2030000014D0B0F8AC30012101FA04F21A430A4BA0F8AC20181D026804F10C0399408A43D6
:203020000260006810B9022001F0CCF8284604F071FC38BD440B00200810044038B5044660
:2030400042F209000DF1020100F09CFC9DF8020050B19DF8020002281AD1A08894F827107B
:20306000FEF78BFC054606E042F20D00694600F089FC9DF80050284600F0E6FB0020A4F85E
:203080007C5094F82130607013B1102004F064F938BD38B5046845682068002808BF4FF0C1
:2030A000FF301FD004F03AFC2168002954BF491E0021216004F02EFC206890B904F12C00EA
:2030C00004F0ACFB04F1480004F0A0FB04F1640004F09CFB6868FAF777FC04F1180003F071
:2030E00047FA002038BDFEE72DE9B841124C0546201D00688047804603F0BAF96F7E002FE9
:2031000008BF6B6807D069682A69AF68091A5218B9180B466960E968286105F11402184607
:2031200002F01CF8012768686F76A168A86040468847BDE8B881C0468C140020D0B50446D3
:2031400004F098FB02F038FA061C08BF6FF004001DD003F007FDB168002908BF002709D08B
:2031600051F80C2C0023B2600F4641F80C3CFF2601F8026C03F01AFFA7603FB117F8080C11
:20318000207117F8070CA0710020D0BD0220D0BD10B504F0C3FB104C217829B10F490C68FD
:2031A00004F0B8FB204610BD04F0B4FB03F068FF0B4A002303F0BEFEA26B002314001B189A
:2031C0004FF07A024FF0905044EB0104C11842EB04021046001C10BD700A00200430044084
:2031E00000093D00B0B5134C6068628800B325880021AA42C8BF01210B46AA42C6BFA91A78
:2032000001F58061A91A8FB28FB1012B03D0A1183A46083109E0A118C2F58062083104F0BA
:20322000F4F9606804F108012A4604F0EEF96580B0BDC04664060020012838B51ED1012088
:2032400002F04CFC01281BD003F054FD0E4D0D4C012105F1E000017020683222B2FBF0F452
:2032600004B90C463035284603F022FA2846214604F008FB284604F015FB01E001F0A2FFAC
:20328000002038BD108B0100940F002038B51248104C0168114D0C40E1430160A10907D3FB
:2032A0004068800904D328464FF4005103F066FE14F4602F0DD02846D43800F1A8010A68B3
:2032C00004F4602400F5847014430C60002103F055FE38BD20000E0008100440440B002071
:2032E000134910B5044691F83F00ADF1180D40F0020081F83F00012003F06AF9607890B956
:20330000211D02A803F062FC03F060FD01460120009004F110030193E38902AA0520F4F768
:2033200017FA607010B1002103F05CFD06B010BD383000201FB5014604208DF800004878EF
:203340008DF80100B1F896000DF10203ADF80C008C31184603F03AFC02F0CCFD60B14FF69F
:20336000FF7453200DF10E01ADF80E40F5F7A0FF044920460A3108806846FAF787F90090B7
:203380001FBDC04622120020C8B5071C01D103F093FF79684878C6111FD03B89F964002058
:2033A0004A78C2F3C3020F2A09D00A781018801C80B25218834202F10201F1DC01E0801CD8
:2033C00080B2834206DB79683E8941187960311A398100E00020A7F85000C8BD10B50446B3
:2033E00000211C22ADF1200D6846FDF7CEFC60788DF80000A0788DF80100E0788DF802005D
:2034000020791122611D8DF8030001A8FCF750F9A07D8DF8150008B1A06906900348006833
:2034200081696846884708B010BDC046181A0020F8B504460D46084611220021FDF7A5FCC7
:2034400094F800C0BCF1000F1AD0641C00214FF0010EE078A37843EA0023207809E0C61071
:20346000AF5D00F00702401C0EFA02F2C0B23A43AA558342F3DA491C241DC9B28C45E8DCB9
:20348000F8BD80B502465378107840EA0320C7130F7007BFC0F3062300F0FF00C0F3C323D7
:2034A000C0F30A004B70802848800DDA02280BDB012B0CD0022B0AD0042B08D0052B06D011
:2034C000062B04D0072B02D00022104600E0921C4A6080BDDCB5044604F0CCF902F06CF80C
:2034E000064604F05BF830F0010014BF002E6FF0040017D0606858B1B0F1FF3F05D0694699
:2035000002F042F830B107460BE04FF0FF3000E0002000907068009904F0E8F9002700B942
:2035200001273846DCBD704770B5114C2068E8B1104D686880470646216894F82F00022844
:2035400006DBA96830468847F120F5F777FF70BD04F1240003F06CF8002394F82F00A96835
:203560002360401C84F82F003046884770BDC046640E00208C14002038B5044642F2080084
:203580000DF1020100F0FEF99DF8020040B19DF80200022817D1204601F046FB054606E049
:2035A00042F20C00694600F0EDF99DF8005094F8200030B9284600F047F9A4F87C500020A6
:2035C00000E00120207038BDF8B5114C60680D468047104A8446A16892F82C70106B9FB15B
:2035E000002420382030867F56B1C27F954207D100228277FF22C277604688472046F8BDFE
:203600007F1E04F10104EDD160468847FF20F8BD8C140020A42E0020F0B5124D00260C46DE
:203620000746ADF1140DC5F8B061012004F049F82868C00FF9D3286A0090686A0190A86A98
:203640000290E86A03903FB13846694611F8012B401E04F8012BF9D1032005B0C5F8380282
:203660003046F0BD504502402DE9FE431F1C14460D4680461BD0DFF83C90082FACBF0826ED
:203680003E1C09F10200007829466B46324603F090FA404621466B463246FDF79FFFBF1BC5
:2036A000BFB230197319002F84B29DB2E5D1BDE8FE83C046441A002003B4B0B5114C04F142
:2036C000080000684FF0FF3104AFADF1180D04F00DF9396804A80160B988818004A803C834
:2036E00000226B46FBF714FA00280CBFBDF80C500025A06804F0F6F8284606B0BDE8B0402B
:2037000002B07047441A00201048114908B54FF42372FBF7CDFF4FF00451002081F89003FD
:20372000012081F87903022081F87503032081F87703042081F8AE03052081F8AB0306208A
:2037400081F881030348C1F8C00308BD1C0400213C000000BD05002110B50446012001F05F
:20376000AFF92078212804BFEB2060700D4991F83F00C20824BF20F0040081F83F00800803
:2037800005D22B2020702046FFF750FB10BD91F83F0000F0FD0081F83F006078002103F0AA
:2037A00021FB10BD3830002070B5114D95F87100B5F896400F2810D00E483430066801F064
:2037C000BDFB2018864208D895F871104FF4707088402418A41B04F57074044D284600F0D1
:2037E0005BF82146284603F069F970BD4C300020A8110020EC170020114898B5012101704E
:20380000022111400F4A4FF0E0471F40002F08BF002903D092F90010491E1170044692F9CC
:20382000000030B192F90000002806DC03F044FD03E000200146F4F765F90020207098BD46
:20384000E41A0020CD1A0020B0B50546802D01DD03F032FD0D4C606880470D4B0D490A4AFC
:203860001F780A390D701FB91778A1682FB907E01778A16837F07F0702D088470120B0BD3E
:203880008847FDF7CDFFB0BD203200208C140020241400209019002070B505460F4800789A
:2038A000012803D001200021F4F72CF90C4C201D006880470B49064628460B4602F082FF24
:2038C00018B9191D284602F07DFF1869A84201D1FCF78AFDA1683046884770BDE41A0020B5
:2038E0008C140020241A002070B540680C46054600F5847002F0DCFE0D482A7F0168687F3D
:203900008018AA69C01D80B244430A4805F584766043B0FBF2F008186330B0FBF1F1491C4B
:20392000304603F0AFFF304603F0BCFF70BDC046108B010040420F000F4838B50078C8B1B7
:203940000E4D0F4C95F82E106420503C4843206604F15C00FFF7C8FBE08EE26B95F82E1035
:20396000401C80B28918E08600B900210020E16300F016FA38BDC04635120020302F002093
:20398000382E0020F8B50E4602F039FF05464FF6FF70A84208BF682013D00B4C6068804775
:2039A00008490A4B0746680000EBC50008180278991842783046FBF77BFEA16838468847C0
:2039C0000020F8BD548001008C140020302F0020B0B5054603F04EFF044603F0DFFD30F0D5
:2039E000010008BF6FF0040414D003F0BBF80A4A002132F80C7F4FB153681B689C4204BF05
:203A00002971002404D0491C0629F2D36FF0040403F0CCFA2046B0BDC014002070B5114C52
:203A20000546E01C0078FE28AEBF0126401CC6B203219622284603F067FC022101222846E5
:203A400003F062FC01212846324603F05DFC0021A522284603F058FC607908B9A570E6701F
:203A600070BDC046441A00201149D0B524310F68ADF1180DCFB17E69BEB1B0B106218DF844
:203A800010100226ADF812600024ADF814404388ADF8003042680192816802917C6904AEBA
:203AA00096E803000C226B46A04706B0D0BDC046A4100020104938B54A39C9690C69257994
:203AC000002101E0491CC9B28D42D8BF4FF6FF7010DD23680A4602EB82029B1893F9002052
:203AE0009042EFD105490839C87803EB4003B3F80100C88038BDC046721600208C190020D8
:203B000038B5EB2003F06FF80D48002505700B480078862802D1284600F064F8094C606841
:203B2000804709490C39CA6913681D711268CA61A168884702F0FAFF38BDC0462032002016
:203B40001E3200208C1400209431002038B50D4C6068804705460C48007870B90B48007870
:203B600030F07F0009D10A48007830B90948007830F07F0001D103F0C2FDA16828468847E7
:203B800038BDC0468C1400201D3200201C3200201E32002020320020F8B506460F480068F3
:203BA0000D4CC06B80476168401A21788900B0FBF1F0B04201D303F07FFB094D243D68682F
:203BC00080470746A6603046FDF708FAF9F72EFEA96838468847F8BDC819002048160020B1
:203BE000B014002038B50F49104C088D401C08856068804705460C480178862903D0A16890
:203C00002846884738BD8721017003F0AFFCA16828468847082002F009FBE920FCF76CFCF3
:203C200038BDC046C4180020203200208C140020F8B506460F4D104F7388002417E0A000F1
:203C400000EBC400321851689068D26852B9AF420BD00A7855F822200346491C084619463D
:203C6000904701E0FBF724FD7388641CA4B2A342E5DCF8BD000E00000C0E0000F8B503462F
:203C800000208C460446074613E01CF8015B082685F0010101F001014018C0B2411E99429C
:203CA00006D0641C761E4FEA6505E4B2F0D100E00127A24203DC27B903F033FD01E0002F42
:203CC000E3D02046F8BD3EB5054615F8060C03281DD12B6818690090586901909869029017
:203CE0006C6859689A681868DB68A0472968086015F8080C01F098FD0446012002F0BAFAD2
:203D0000011C04D0422008702046FEF7B1FD3EBD2DE9F04117468846064603F033FA0D4C9D
:203D20000546002128222046FDF72FF831462A462046FBF7BDFC40463A46291900F0E4F840
:203D4000204602F05DFF02A002F05AFFBDE8F0810D0A00C06031002038B50446642C13DA70
:203D60000D4D6868804702466946722002F00EF80099E00000EB04104018A968009010460A
:203D800088470098001D38BD0448643CE1B2383000EBC10038BDC0468C140020A42E00206A
:203DA00070B50F4C05462179E079814217DD6179A94214DDA3680B4E23B1294632469847DA
:203DC000E0796179A07101FB0050216800EB800009180878E071D1F801103046884770BD21
:203DE000781600201C2E0020F8B502F0CDFC0D4607463A2F08BFF42012D00B4C6068804797
:203E00000646BA0007480949835C801842784E39C918284603F06AF8A16830468847002031
:203E2000F8BDC0462C8201008C1400205A120020FEB505460F4CA889E2880F46411D8EB2E5
:203E4000A178B218B2F5805F0BDD08460021F3F7ABF8864203DD607900B90520FEBDA889CA
:203E6000A17800900022284601971346F8F7B4F86079FEBD441A002038B50D460E4914467A
:203E800060390A68AA4205D901EB8501D1F89410884201D0022038BD03F040FD074B103BEF
:203EA0001A68AC400121A9408A4314431C6003F031FD002038BDC046AC2B0020E020024074
:203EC00070B50E4614460546082300212422ADF1280D684603F0E2FC002006900590ADF8F0
:203EE0001000084800684FF47A716B46B1FBF0F080B2314604FB00F2284603F0CBFC28465F
:203F00000AB070BD108B0100FEB50746052400266B4697FBF2F05043381AC0B20A28ACBFB6
:203F2000372530254019187097FBF2F5AFB22FB1641E03F1010306F10106EAD1761C13F865
:203F40000109761E01F8010BF9D100200870FEBD10B50F4C94F83F00ADF1180DB0B940F05A
:203F6000010084F83F00012002F032FB02A801F0D5FF343401200090064B019403F18A0059
:203F80000388032102AA0520F3F7E2FB06B010BD38300020A81100200E4808B50178081C46
:203FA00005D0401E12D0801E01280FD908BD03F099F838B10948084900680968884238BFCF
:203FC000002004D31C20FCF797FA08BD0846F0F7C7FC08BDC6180020600D0020CC19002018
:203FE0001FB5144600900A79487940EA02208A7942EA0022C87940EA022001900A784878C2
:2040000040EA02208A7842EA0022C87840EA02200290684600F028FAB0FBF4F16143401A98
:20402000C0B200901FBDF8B5051C0E4606AF04D0012D0CBF0624002400E002240EB9A41C23
:20404000A4B2012A06D0022A0ED15889C01D04EBE00008E03878002814BF02210121002079
:20406000FAF758FE001984B22046F8BD2DE9F04115468046287840F0C000287028790C460C
:2040800004262F1D40F00200287117F801293119404689B203F038F9761EF6D52A79241D34
:2040A0004046A1B202F0FD022A7103F02DF9BDE8F08100000F4800B50068ADF1240D69467A
:2040C0006C30F8F78DF810B99DF80B0008B900200DE0684601F099FF9DF808104FF47A7385
:2040E000B0FBF1F24A43801A091A03FB01F009B000BDC046640E002070B5054602F032FD5A
:204100000D4C0221064654F80C0F58B9002025600146A0600A4603F0B9FB606038B903F0D8
:20412000E2FA04E0A84202D0491EECD10024304602F03CFF204670BDA814002038B5054671
:204140000C4600200090042C0BD3241F284604226B46A4B2214602F02CFD0098B0F1FF3F78
:20416000F1D001210A4600F0FF03FF2B18BF111C000A521C0090042AF5DD091988B238BD93
:204180002DE9F04103F016FA0D4D603D2B688046A3B105F194060024012707FA04F018EA5E
:2041A000000F07D056F8240020B1026812B1214690472B68641CE4B29C42EED3BDE8F0810D
:2041C000AC2B002010B5044603F0A8FB0C4A117819B903F09FFB822010BD11460B7884F048
:2041E000FF0213400B70097811B103F093FB05E003F090FB0348082102F0C0FE002010BDB8
:2042000016320020440B002038B50D46044603F08CFA6368A1688B4204D103F07BFB4FF0A6
:20422000FF3038BDE168491CB1FBF3F25A432368891ACD54E1606269A168491C8A42A160E8
:2042400038BF616103F066FBA06838BD0C4885460C4885446F4607208743BD460A486F4668
:2042600007600A48002803D07946491D8E460047FBF730F902F052FE03F0BCFAFEE7C04659
:20428000004B002000050000D41A0020C17501000F48B0B507680025ADF1180DADF8105051
:2042A00097B106208DF808000223ADF80A30ADF80C5004AC00943C6902AA92E803002A467C
:2042C000A04708B1ADF81050BDF8100006B0B0BDC810002010B50446012000F0F1FB2078B5
:2042E000212804BFEB2060700A4991F83F00C20824BF20F0040081F83F00800809D391F856
:204300003F0000F0FD0081F83F006078002102F069FD10BD3830002030B50E4D95F87100D5
:20432000ADF1AC0D0F280CD10B4C343C04F11400FFF7B2FAB5F8961004F1140002F0BEFB99
:2043400005E02F208DF800006846FEF76FFD2BB030BDC046A81100206C30002038B50F4CEA
:204360000546204603F0B4F8A8B9204603F0DFF90446A068054209D0E36822692846002184
:204380009847002818BF4FF0FF3005D1204603F0D0F9041CEDD1002038BDC046940F00201D
:2043A0000CB4F0B505AF061C0C4627F00303ADF1040D03F1040304D03068002818BF051C1D
:2043C00000D100253A68284602F0EEFF844238BF601E15B131684118316001B0BDE8F040EE
:2043E00002B07047D0B504463C20FCF7C9F8071C14D000213C22082303F02CFA207AB861F8
:2044000060893862E068386160683946002203F0F5F90646384601F009FB16B96FF00300FE
:20442000D0BD0020D0BD08B50B4602F0B7FC5989418199898181997B8173D97BC173197CA2
:20444000002201B10122597C417459694161197E0274002201B10122027603F119010B22C0
:204460001930FBF725F908BD416882680D4B0068C91AD21AC01A4A40A2EBB1425040A0EBFD
:2044800072504140A1EBF0114A40A2EB31425040A0EB32704140A1EBB04181EA0200A0EB0F
:2044A00031207047054152210B4A08B502F10C000068C00A01D200F0F1FB10684008FCD3BA
:2044C0000648006841680220884705490A6882420CBF0448086008BD08800240CC0100101D
:2044E0001C280020EFBEADDE10B50821ADF1180DADF800100A4C04901B21ADF80210606A13
:204500000290012101910549064803910168684688470299616206B010BDC0463D5C0100BE
:2045200064180020B014002010B5ADF1180D0C4C01900A4808210390002004902069ADF89A
:2045400000101B2102900748ADF802100168684688470299216106B010BDC046F95701009A
:20456000C8190020B01400200D4808B50068020F0C48036803F0FF03802B28BF002302F070
:2045800077F901464FF0FF30012907D1111C04D0891E04BF143358B208BD0A2008BDC0467E
:2045A00018130050A0100050D0B50E4C0646A0684FF0FF3103F09AF9277977B9E088C0F56B
:2045C000805000B2864203DC002E18BF042704D1A0780021F2F7E8FC6779A06803F082F951
:2045E0003846D0BD441A00200E4938B5CA68824210D1087801280DD103F090F90546084879
:2046000001F0ECFB0446284603F084F904F0FF00012802D06FF07F0038BD4FFAA4F038BD07
:2046200001000304700A0020B0B503F07EF805460A48017801290DD00121094F0170387852
:2046400040B1084C074620688168204688470C347F1EF8D1284603F05DF9B0BDCF1A00204F
:20466000288B0100EC8901000B4B80B51F7800227FB10A4B1B7883420BDD8A4208BF084923
:20468000084F820002EBC002B8180268D26890470246104680BDC046CF1A0020288B0100A9
:2046A00084890100EC89010030B50E4D2868ADF1240DA0B10024FFF7F7FE04EB0D02002158
:2046C000CB00491C20FA03F3042902F8013BF7DB241DE4B2202CEEDB29686846884709B0B2
:2046E00030BDC046D01A002010B50446012000F0E7F9EB200B49607091F83F00C20824BF19
:2047000020F0040081F83F00800809D391F83F0000F0FD0081F83F006078002102F062FBB4
:2047200010BDC0463830002008B564206946FFF75BFB0A490A48C1F8D8000A48C1F8DC00C5
:204740009DF8000000280CBF49F24E0047F60E20C1F88000C1F8C00008BDC046280D00200B
:20476000A431002058160020F8B5071C01D102F0A3FD0C4C201D006880473E6805465EB1BE
:2047800007498A68A6F10C00964204BF00228A600021396001F00CFEA16828468847F8BDDD
:2047A000141500208C14002038B50E4B05460C46281D03F1480102F02DFF188F2880B3F873
:2047C000460003F13E016880201D02F023FF93F83A00207300206073188F2080988F60808E
:2047E00038BDC046481300201CB50A1C17D000230124E407A04238BF041C944201D9520037
:20480000FBE790425B41904228BF801A914201D25208F6E7191C021C081C111C1CBD00B1EA
:20482000C843FBF7FEFB1CBDB0B50D46044602F07CFFA76897B121692268515C29706368BE
:204840002169A768491CB1FBF3F25A43891A2161791EA16003F05EF8A068B0BD03F05AF86C
:204860004FF0FF30B0BD00000D4910B509780446A1B1617871B9217839B194F8201021B909
